:020000040800F2
:100000000000012015D50408B1D50408C1BC0108C1
:1000100019BB0108B1D50408B1D5040800000000DF
:10002000000000000000000000000000B1D504083E
:10003000B1D5040800000000B1D50408A975010875
:10004000B1D50408B1D50408B1D50408B1D5040868
:10005000B1D50408B1D5040839A1000841A10008B0
:1000600049A1000851A1000859A10008459F0008B6
:10007000599F00086D9F0008819F0008959F000808
:10008000A99F0008BD9F0008B1D50408B1D5040898
:10009000B1D50408B1D50408B1D5040861A10008A0
:1000A000DDC80008C9C70008EDC80008B9C70008C6
:1000B000F1C7000801C8000811C80008559A0008D7
:1000C000499A0008899A00087D9A0008B1D5040869
:1000D000B1D50408F5740108017501080D75010812
:1000E00069A10008B1D50408B1D50408FDC800080D
:1000F000B5C80008B1D50408A5C80008D19F0008FC
:10010000B1D50408B1D5040821C80008B1D5040848
:10011000197501082575010831C80008A95304089C
:10012000E59F0008F99F00080DA0000821A0000825
:1001300035A00008000000000000000000000000E2
:100140000000000000000000000000002D4904082D
:1001500049A000085DA0000871A0000831750108E1
:10016000BD9A0008B19A0008B1D50408B1D50408B9
:10017000B1D50408B1D5040800000000000000005B
:10018000B1D50408B1D50408B1D50408B1D5040827
:10019000B1D50408B1D5040800000000B1D50408A9
:1001A000000000000000000000000000B1D50408BD
:1001B000B1D50408B1D5040800000000000000001B
:1001C000000000000000000000000000000000002F
:1001D000000000000000000000000000B1D504088D
:10800000084A0346D0F8E4005268D3F8F010121A78
:1080100000209142B8BFC3F8F020012283F81C2150
:10802000704700BF001000E01B4B1C4A03F5727C38
:10803000016803E063452BD053F82C2F9142F9D10E
:1080400070B593F804E0427996450AD0634505D0AF
:1080500053F82C2F9142F4D06345F9D14FF0FF3003
:1080600070BD9E4684680022DEF80C50A54208D000
:1080700001320EF10C0E032AE8D0DEF80C50A542B6
:10808000F6D1DEF81050C668B542F1D150B270BDDD
:108090004FF0FF30704700BF28F004080000014097
:1080A0004368426D30B49A61EFF31182502383F339
:1080B00012884168D2B2856C0B68046D23EA05030F
:1080C00023430B6082F31188436981681A68096849
:1080D00022F00102D0E908541A60826A1D605C61D6
:1080E0005A60D0E90B429C60DA600023B0F86C2043
:1080F00030BCCA620377704730B5FAB18E464FEA9A
:10810000014C034600F1C005002419680C3353F8F4
:10811000042C43F8084C41EA0C0142EA0E02AB423F
:1081200043F80C1C43F8042CEFD1D0F8C03043EADC
:108130000E03C0E93144C0F8C03030BD4FEA014EF3
:108140008C46DEE783695969B3F810C00A6830B419
:108150009C6822F0010224680A60E26822EA0C02AC
:10816000E260027D04681F2A06D9203A082065686B
:108170009040284242D0FEE70820256890402842DF
:10818000F9D1202000FA02F2A260254A1278002AD2
:1081900032D01A7F012A36D0D3F800210132C3F839
:1081A0000021EFF31181502282F312885868C9B27E
:1081B0009D6C0268DC6C22EA05022243026081F3B6
:1081C00011885A699968D3E90D40096814605061B3
:1081D000D3E90F40546090605C6CB3F8B400D46095
:1081E0000124C8621068204310601A8A1C7783F843
:1081F000FD40CB681343CB6030BC7047202000FAB1
:1082000002F2E260C1E70022D3F8040183F8FD2006
:1082100001300A68C3F8040122F001020A60EBE7AA
:10822000C801002010B40C4C6368002B11DD002045
:1082300004F1080C0146DCF8AC3003F1C0025960CF
:108240000C339342FBD1013063680CF5867C83428A
:10825000F1DC5DF8044B7047C8010020704700BF97
:10826000024B03EB401090F855047047C801002002
:10827000014B53F82000704750280040704700BF62
:108280000B4890F86C1589B101EB4101002300F215
:108290007450490010B41C4650F82320063302B134
:1082A00014608B42F8D15DF8044B7047704700BFF3
:1082B000C80100200B4890F86C1589B101EB410111
:1082C000002300F27450490010B41C4650F82320DB
:1082D000063302B114609942F8D15DF8044B70473F
:1082E000704700BFC801002001207047034B00EB1E
:1082F000400003EBC00090F885057047C8010020DE
:10830000204890F86C35002B3AD0002200F27453CC
:108310004FF02C0C2DE9F0434FF0500E1A4E1B4D30
:10832000144607E053F8181B01320C6090F86C15E6
:10833000914223DD197C0029F4D05F684FF0FE08DC
:10834000B90AA1F580115229294498BF91F8F48304
:10835000EFF311818EF31288D7F824900CFB086894
:10836000C9B209F10109C8F82890D7F8148048F07B
:108370000108C7F8148081F31188D3E7BDE8F083C2
:10838000704700BFC80100202018012028F0040811
:1083900007EE900AB8EE670A704700BFBCEEC00A4D
:1083A00010EE103A98B270470346012200205A7727
:1083B000704700BF08B5D0E90B2183690B44836186
:1083C0000AB108469047002008BD00BF436A024634
:1083D0001B681B6A5B685B7813F0010008BF50776D
:1083E000704700BFC2628161704700BF704700BF25
:1083F000043070470C4B93F89822D3F8941202443F
:108400000844D2B2C3F8940283F8982293F89822D1
:10841000120605D593F8982282F0800283F89822FC
:10842000024B01221A707047201801200000012021
:108430002DE9F84F154FD7F89C52ED0A20D00026B1
:10844000DFF84CA007F52879B046AC19D7F8A01290
:10845000102352466410D1F828B04846C7F8CC82A1
:10846000E102D8470F280BDD094B03F1100253F846
:10847000041B013107D19342F9D12546B542E4DC12
:10848000E802BDE8F88F661CF8E700BF201801205D
:1084900000000020184BD3F8D412D3F8D8228A1A3F
:1084A000322A15D8D3F8EC228A4200D37047D3F889
:1084B000DC22E2B110683231928810B44469C3F80A
:1084C000EC1222425DF8044B18BF1204826170471F
:1084D000D3F8DC223AB193F8E8021168C007928819
:1084E00048BF12048A610022C3F8EC22704732317F
:1084F000C3F8EC12704700BF20180120064AD2F8DA
:10850000DC323BB192F8E8121A68C9079B8848BF71
:108510001B0493610020704720180120044B4FF486
:10852000007C0020D3F8F832A2F800C00B6070473E
:10853000201801200020704701207047012070475B
:1085400000207047134BD0F8D8105B68D0F8E020BB
:1085500010B50446581A824200DC22B9D4F8E4204F
:108560000A44C4F8DC2094F8D020C4F8D830012A9A
:1085700005D0D4F8D4300133C4F8D43010BD04F1A0
:10858000E801201D0EF04CFAD4F8D4300133C4F8C1
:10859000D43010BD001000E0CB070AD490F828308A
:1085A000012B08D0C368B3F1807F03D9012303777F
:1085B0007047704770471B4AD2E9CA1310B5B1EB38
:1085C000930F8CB04FEA9302446A4FF0020306D235
:1085D00052085B0091429BB201D2FF2BF8D9C268CE
:1085E000A380B2F1807F1BD90122002301A94FF0A3
:1085F000B70C0277204604928DF814208DF82820BD
:108600008DF804C00B93CDE9021302A9CDE906331E
:10861000CDE908330EF004FA2268136A002BFCD16E
:108620000CB010BD2018012030B590F828308BB068
:108630000446012B05D0407F48B1002363770BB07F
:1086400030BD456A2B681A7B22BB637F13B90120BA
:108650000BB030BD12490220002301220290081FF6
:108660008DF80C208DF820200993CDE90010694683
:108670002846CDE90433CDE906330EF0D1F92A6856
:10868000136A002BFCD1074B5B7C03F0010383F0E2
:108690000100D3E71B6A002BD7D00020CFE700BF33
:1086A00014000020000000202DE9F0411F4F8AB087
:1086B000044690F82820A7F10408A7F11406437F88
:1086C000012A06D00BB10023637701200AB0BDE870
:1086D000F081656A2A68117B09BB002BF5D0002365
:1086E000694628460993CDE90433CDE906330123D1
:1086F0008DF80C308DF820300223CDE900780293FC
:108700000EF08EF92A68136A002BFCD1737C03F0FB
:1087100001036377002BD8D094F82820D0E7126AA1
:10872000002AD7D1002BD0D0D9E700BF14000020F9
:10873000244A002330B5044695B0101D224D0693FF
:10874000019002200B931093139311930290207FBA
:10875000009200280495CDE90E334FF001038DF807
:108760000C3007938DF820308DF834308DF8483078
:1087700002F10803A2F10802059314BF05230423A4
:108780000A920C93114B0993636A1A68136A002BBF
:10879000FCD1A0B10E480A0E00F11A0342760A0A73
:1087A0009970080C69465A701870606A0EF038F9B2
:1087B000636A1A68136A002BFCD115B030BD054BF3
:1087C000EDE700BF20000020CD830008A98300084A
:1087D000000000201900002010B594B0044650227B
:1087E0000749684646F0DEF96946606A0EF018F9F6
:1087F000636A1A68136A002BFCD114B010BD00BF65
:1088000070F40408F8B50546406A0068046A002C54
:10881000FCD1287F002839D0A8690527254E4FEACA
:10882000106C254C2E3606F801CC6763B0704FEA09
:10883000104C000A012B86F800C070704FF0000049
:108840000E6826641668A6642E63A06524D0022BE9
:108850001BD15368012220651E444968E365174B0C
:1088600084F84C0061652E6384F860206366144BC5
:10887000697F03F11402686A002914BF1946114682
:108880000EF0CEF8EB6A73B1286BF8BD04200A4CE9
:108890000C4E6063A869C9E7084A84F84C306065EB
:1088A000E0652265E3E76B6A1A68136A002BFCD166
:1088B000EAE700BF0000002000000120B5830008A7
:1088C000040001202D00002000B583B081610192D9
:1088D00001A9049A00930123C2626A46FFF792FF3E
:1088E00003B05DF804FB00BF70B51D46436A94B049
:1088F00006461B681C6A002CFCD13A4B02204FF044
:10890000010C0694029003F13C008DF80CC000901D
:1089100003F1400001903448049003F134000590C5
:10892000307F00284BD00B920A0E36338DF8204052
:1089300003F8012C05220C958DF834C08DF848C041
:1089400013940792CDE90944CDE90E44CDE91044D2
:108950000A0C9970254C090A1A705970706AD4E98A
:10896000CA32B3EB920F4FEA92014FF0020206D2E5
:10897000490852008B4292B201D2FF2AF8D9737F84
:108980008280D3B905A90EF04BF8706A03681A6AA1
:10899000002AFCD10222D4E9CB34B4EB930F4FEA86
:1089A000930106D2490852008C4292B201D2FF2AAA
:1089B000F8D98280284614B070BD6946E3E70B926F
:1089C000042235338DF820000C958DF834C08DF8D5
:1089D00048C013900792CDE90900CDE90E00CDE91A
:1089E0001000B5E700000020CD830008201801200A
:1089F0000C4AF8B5136855692B4003EA0005556128
:108A00007DB1094F0126B5FA85F4C4F11F0407EBC7
:108A1000840306FA04F4D3F8340303689847A543A3
:108A2000F1D1F8BD003C0140201801200269C36863
:108A30002DE9F04712EA03092AD005460E464FF009
:108A400000474FF00008B9FA89F327FA03F21B3BFD
:108A5000D24309EA02092A61042B16D8DFE803F0A1
:108A60003B30251A0300B36A002B3FD003F1FF3AD5
:108A7000C6F828801FFA8AFA746A34B1236820463F
:108A8000514698476468002CF8D1B9F1000FDAD14B
:108A9000BDE8F08770680028F7D0696B036889B279
:108AA0009847B9F1000FCED1F2E7B0680028ECD0BA
:108AB000A96B036889B29847B9F1000FC3D1E7E702
:108AC000F0680028E1D0E96B036889B29847B9F1F2
:108AD000000FB8D1DCE730690028D6D0296C0368D4
:108AE00089B29847B9F1000FADD1D1E7E96A1FFA11
:108AF00081FAC1E78369F0B593F8DC208BB00546B5
:108B0000012A27D0023A012A2FD893F84C21EC46AB
:108B1000D3F89C1062F07F03154C0B708669D6F871
:108B2000A0305F1C0FCCACE80F00D6F89C30CDE92C
:108B300000370FCCACE80F0094E803008CE803008A
:108B4000694606F110000DF06BFFAB6919690A6AFE
:108B5000002AFCD1D3F8A0305A8852BAEA819A8808
:108B600052BA2A82DB885BBA6B8201200BB0F0BD5F
:108B7000C0F40408F0B590F8DC308BB00446D0F8AF
:108B8000A060012B4BD015D8D0F89C304FF0FF32AD
:108B900005211A605A609A60DA60D0F8E030C0F8B7
:108BA000F010B3F57A7F54D8032380F8DC3001202D
:108BB0000BB0F0BD023B012BF9D890F84D31EC46DB
:108BC000D0F89C2063F07F03384D1370D0F8A030AC
:108BD0005F1C0FCDACE80F00D4F89C30CDE9003716
:108BE0000FCDACE80F0095E803008CE80300694660
:108BF00004F110000DF014FF2269136A002BFCD160
:108C0000738801205BBAA4F8D030B3885BBAA4F8AB
:108C1000D230F3885BBAA4F8D4300BB0F0BD90F832
:108C20004C2190F84D319B1A5B100133DBB236F8C2
:108C3000132006EB430653BAA0F8D03073885BBA12
:108C4000A0F8D230B3885BBAA0F8D43001200BB0C2
:108C5000F0BD03691A7B2AB35B691BB390F89830A7
:108C600003B390F84C310122D0F89C0063F07F03ED
:108C7000C4F8A4400E49037094F84D3194F84C01A7
:108C800084F800211B1A84F8DC20D4F8A0200733D4
:108C9000C4F804110132D4F89C10C4E93E23C4F88E
:108CA000F41084E7022384F8DC3080E7C0F4040881
:108CB000018000082DE9F041304F07EB401898F88B
:108CC00054340BB9BDE8F08100EB80030E4600215F
:108CD000044607EB4313450193F8362683F836160E
:108CE00088F83A2446F048F9B8BB3D442448A5F832
:108CF000386400EB441046F03BF93B78D5F850243B
:108D0000A3B1D5F83C140124D2F8AC308C4003F167
:108D1000C001420010F4004F90B202D15A682243C1
:108D20005A600C339942F4D1BDE8F081D5F83C1477
:108D30000124D2F8AC3001F1100203F1C0019440DB
:108D4000420010F4004F90B202D15A6822435A6098
:108D50000C339942F4D1BDE8F0810A4B93F8EC232F
:108D600002EB420203EBC203234493F89963002E03
:108D7000BBD0012388F83A34B7E700BFC801002010
:108D800000060020201801202DE9F84F374D2B78E0
:108D900013B90120BDE8F88F354F05F5876A05F650
:108DA00034360024D7F8D4B24FF6FE794FF6FF7868
:108DB00015E0B0F5606F4AD0B081B0EB08012D4BE3
:108DC0004FF05C005A4618BF012100FB04300DF043
:108DD0003DFC01340AF1200A1436082C31D0D5F8B4
:108DE0001C2FA2422DDDDAF81800DAF80420D0E9B1
:108DF0003D0146F011F9484597F8752314D0542ADF
:108E000004D1B7F878230132A7F87823D5F83C2BA2
:108E1000404502F10102C5F83C2BCAD1D5F8382BE8
:108E20000132C5F8382BC8E7542AD2D1B7F87A23D3
:108E300001340AF1200A14360132082CA7F87A23EB
:108E4000CDD10123012085F8383CBDE8F88F97F893
:108E5000EC2302EB420207EBC202224492F8992370
:108E60000D2AA9D18022B277A7E700BFC801002050
:108E700020180120040E00202DE9F8430EF0EAFC32
:108E80002F4E4FF0000C0746DFF8BC802D4C716868
:108E900000294ADD00234FF486701D4600FB036263
:108EA000013392F80521994245EA0205F6D145EAD7
:108EB0000C0C5FFA8CF9D8F80430C3F308038BBBB1
:108EC000EFF3118373BB4FF0E02CD4F8D432DCF80D
:108ED0001810D4F8D4229342F7D1D4F8F023914259
:108EE000F3D8D4F8F4C34FF47A7202FB0CF0401AB2
:108EF000B0FBFCF002FB0300C31BB3F5FA6FCCBF61
:108F00004FF0000C05F0010CBCF1000FBFD1B9F11E
:108F1000000F04D00B4B93F87523542A08D0484611
:108F2000BDE8F8830EF066FBE6E7E1460025C2E700
:108F3000B3F87C2348460132A3F87C23BDE8F883CC
:108F4000C80100202018012000ED00E010B5044603
:108F500045F0B0F80146204689B2BDE81040A9E6C8
:108F600038B50B4D00EB400005F27453C40003EB21
:108F7000C0032C4493ED027AD3ED037AE7EE007A36
:108F8000B0EE670A45F096F8D4F87435186038BD2D
:108F9000C80100202DE9F04146F026F880B31B4FB0
:108FA0007D68002D12DD3846002410F8086BA046BD
:108FB000013416B1037F012B1DD04269AC4200F58C
:108FC0008670136843F001031360F1D10EF042FC88
:108FD000D7F8204F002C0CDD0D4B03EBC4041968AF
:108FE000083333F8042CC8689C4242EA0002CA6085
:108FF000F5D1BDE8F08180F8FC80FFF751F8DCE79F
:109000003FF092F90028CAD1BDE8F081C8010020E4
:10901000EC100020836910B51A4C04EB8303D3F8DD
:109020001C043AF09FFBB4F83C340C2B0ED8DFE85C
:1090300003F0070D0D0D220D0D0D1B0D0D0D140070
:10904000D4F8FC23D36823F40073D36001220023F7
:1090500084F8392484F83E3410BDD4F8FC23D36856
:1090600023F48053D360F1E7D4F8FC23D36823F4CE
:109070000063D360EAE7D4F8FC23D36823F4806369
:10908000D360E3E72018012080699C303AF06ABB86
:10909000830AA3F58013522B52D8F0B504466A48D0
:1090A00085B0034493F8F4030D2847D8674D860133
:1090B00005EB8013D3F84074A7423FD00139C3F8C1
:1090C000404489B2C3F84C14D5F82C13B1FBF2F22A
:1090D000013AC3F844240022C3F85024C3F84824BA
:1090E000C3F8542493F87D2402F0FF014AB3584991
:1090F0000223AF1901EB8011204687F87D3404313B
:109100003BF0C0F8012387F87D34524B9C421BD0C2
:10911000B4F1804F18D0A3F57C439C4275D003F581
:1091200080639C4271D04C4A03F57C439C4218BF3B
:10913000944249D003F570539C4245D005B0F0BD30
:10914000704783F87C14D2E700234FF48051AA19AA
:10915000CDE9001392F87C140129CDE90233EDD05A
:109160000221D2F84004012482F87D143B4987682B
:109170003940816082F87D4482F87C340023AA194A
:10918000CDE90033029392F87C34012BD6D0D2F88B
:10919000403402212F4882F87D1483425A6899682E
:1091A0004ED000F5806083424AD022F0700221F058
:1091B0008001354401205A609960002385F87D04C0
:1091C00085F87C3405B0F0BD00214FF48053CDE923
:1091D0000031AB1993F87C24012ACDE90211ADD0FE
:1091E000D3F84004022283F87D241C4A87683A4061
:1091F00082601B4A83F87C140121944283F87D1419
:10920000BCD0154B9C4299D1B8E700224FF4805155
:10921000AB19CDE9001293F87C140129CDE90222A3
:109220008CD00221D3F84004012483F87D140B492B
:1092300087683940816083F87D4483F87C249DE70A
:1092400022F47002B1E700BF28F0040820180120C2
:10925000601C012000000140000C00408800FEFF5F
:10926000000401402DE9F843DDF820800F46164642
:109270000021202204461D4645F008FDB8F1000FEC
:109280000CD0D8F80030B8F80A20E3811B0C2382F8
:10929000D8F804306282E3821B0C2383384643F003
:1092A00039FAF30619D4431EB8B107EB000C01E0FC
:1092B000013B12D31CF801EDBEF12E0FF8D1C01AFC
:1092C00003F10109421EB944032AA8BF0322082B57
:1092D000A8BF082390461A4606E008280246B94669
:1092E0004FF00008A8BF08224FF02033394620462F
:1092F0002360636045F056FC04F1080317484246BA
:1093000049462081A072184645F04CFC04F1FF3C10
:109310000346E21D1CF8011FA1F1610E2039BEF1C8
:10932000190F98BF8CF800106245F3D1184604F16C
:109330000B0110F8013BA3F16102203B192A98BFF1
:1093400000F8013C8842F4D1182365832D0CE672A5
:109350002373099BA582E361BDE8F88320202000E8
:109360002DE9F04FDFF88C9487B0D9F8D402C9F812
:10937000D802002B00F0DA801344154601F12006D4
:1093800001F5FE77DFF870A403931FE0002D63D092
:10939000D9F80423AA4200F0CD80D9F80023AA42CC
:1093A00000F00281D9E9C221AA424CD8A94200F2B8
:1093B000CF81691A18463EF0E3FA0135039B06F5A2
:1093C000007607F500779D4200F0B080D9F8104391
:1093D000A6F12003AC42D9D82C1BD9F82083E2088F
:1093E000D8F8301004F0070402328A4203D3D8F8C8
:1093F00038108A420DD941461046059304923EF03A
:109400008FFA8046DDE90423002800F0C181C9F805
:10941000200398F80410002940F03F81D8F828B0C4
:10942000BBF1000F00F0AD811846D8F830304FF492
:109430000071D21AD8F80C3004EBC20203EB4222BE
:109440004346D847B9E7A942B3D918464FF400724A
:10945000002145F01BFCB0E74FF400722946184686
:1094600045F014FC80220346D94886F89E210C2240
:1094700086F8A221D9F80013D9F8F8228142C3F85E
:10948000C611C3F8CA2100F36881D24B013AD24C0D
:1094900083FB0103C81784FB01C40B44C0EB6313B7
:1094A000C0EB2430CD4C84FB03C4C3EB831C86F893
:1094B000A1018010A1EB0C011C4420F03F00013100
:1094C000014386F8A011D917C1EBE4110B4486F8CB
:1094D0009F31BF4B9A4200F34C81BE4BBE4883FB89
:1094E0000213D11780FB02401344C1EB6313C1EB9D
:1094F0002031BA4880FB0340C3EB831486F8A511E2
:109500008910121B184421F03F0101320A4386F8EA
:10951000A421DA17C2EBE010034486F8A3315523E7
:1095200086F8DE31AA2386F8DF3146E7002007B04F
:10953000BDE8F08F4FF0FF320024A6F11C00049329
:1095400083F8EC21214683F8ED2183F8EE2183F89E
:10955000EF2152221A705A7061229A7083F8E72123
:109560004122DA7083F8E621722283F8E42183F83D
:10957000E521D9F81823C3F8E8214FF4F07245F03B
:1095800085FB049B5522C6F8D041C6F8D441C6F8E5
:10959000D84183F8FE216FF0550283F8FC4183F82F
:1095A000FD4183F8FF2108E78D4C00214FF4007244
:1095B000184645F06BFB03464FF0000C022203CC2B
:1095C00046F8191CEB2146F81D0C082006F8201C53
:1095D000582106F81F1C902106F81E1CF8211A734A
:1095E00083F80BC006F8130C9A7383F80FC006F8C3
:1095F000102C06F80B1C83F82C20D9F80013D9F88E
:10960000F82283F819C0521A83F81BC083F81DC0D2
:109610001A6283F81EC083F81FC083F82DC083F838
:109620002EC083F82FC0D9E9C212521A80215A6283
:109630003F221A764FF0FF329A763E221A770122A5
:1096400083F8302083F831C086F820102921654B3B
:1096500086F82210942186F8260086F823100E2121
:10966000614A86F824100D2186F82510552186F8C8
:10967000DE11AA2186F8DF1103CBC6F82B1019885A
:10968000C6F827009B78A6F82F1086F8313003CA59
:10969000C6F83200C6F836108FE64FF4007218464E
:1096A000002145F0F3FAD8F840200346002C76D18B
:1096B000002A00F0A380D8F8303011224B49CDE9C0
:1096C0000044FFF7CFFDD8F840301A6C002A00F0B4
:1096D000A1801B6BCDE900441122454930464FF46F
:1096E000E07BFFF7BFFD06F12003D8F84480B8F116
:1096F000000F3FF462AE03F120049B44049523461F
:109700004446984610E05CF81C1B0025236BCDE90D
:1097100000C5FFF7A7FDABEB0803A46C08F1200818
:10972000002C18BF1F2B51D92379A44604F11C0E1D
:109730001122A8F12000002BE5D162792569236B65
:1097400042F021022168CDE900E5FFF78BFDE2E759
:10975000A91A18463EF014F92FE6FF23013A86F8BD
:109760009F3186F8A13186F8A031194B9A427FF7D4
:10977000B4AEFF2386F8A33186F8A53186F8A4316C
:10978000CDE6594618464FF4007245F07FFA14E6CC
:10979000A6F1240343F804AF9F42FBD10DE6002A53
:1097A000D8F844800CBF01220222C2EB0414B8F1A5
:1097B000000F3FF402AE4246013C926C002C01DDEA
:1097C000002AF9D190464FF4007B90E7049DF4E520
:1097D000FF03FB00832008829755454181808080EC
:1097E000946A0508A06A0508AC6A05088C6A050831
:1097F000906A050820180120DEADBEEF234608223E
:10980000D9F8FC124FF4F07BCDE90044FFF72AFDB4
:1098100033466AE72346CDE900445DE7F0B50446E8
:1098200090F8210187B008B907B0F0BD0DF0BAFC7F
:109830000546002852D0818826222A4BC280E36048
:10984000B1FA81F3202BC3F11F02EDD026480C346E
:10985000264E104406EB820290F84075C2F834435D
:109860004FF0004232FA03F305D0214A106820EA93
:1098700003001060536100233E44019101A9059348
:109880002868CDE903331B4B02933AF05BF896F856
:109890000038F02B0CD8AA884FF00043B2FA82F2BD
:1098A000D340C1D012490A6813430B6007B0F0BD22
:1098B000114BF0220321DC5786F800282046DE5D9C
:1098C0003EF088FF002CE6DB06F01F06012364094A
:1098D0000A4A03FA06F642F82460DCE7014BE3602B
:1098E000A2E700BF4585000828F0040820180120E1
:1098F000003C014000001110546B050800E100E03D
:1099000030B490F8443000F10801484A012BC2F805
:1099100008186ED083684649DC68464D24F460041C
:10992000AB42DC60DC6844F46004DC609C6B24F4D3
:1099300040149C639C6B44F480149C639C6B24F4E3
:10994000F8449C639C6B44F488449C639C6824F4B6
:1099500070249C609C689C609C6824F440149C600B
:109960009C689C605C6824F480645C605C6824F49F
:1099700080545C605C6901EA04015961596959616C
:1099800047D0DC682A4924F0E064DC60DC6844F0FD
:10999000E064DC609C6B24F440149C639C6B44F496
:1099A00080149C639C6B24F478249C639C6B44F42B
:1099B00010249C639C6824F470249C609C689C60C8
:1099C0009C6824F440149C609C689C605C6824F44F
:1099D00080645C605C6824F480545C609C69214015
:1099E000144C9961A3429969996118D0002380F8B9
:1099F00044301148114B848DC18D408D091BC2F834
:109A00001048C2F80C0893FBF1F330BCC2F81438CC
:109A100070470B4C616841F400016160B1E708498F
:109A20004B6843F400034B60E0E700BF20180120BF
:109A300000F0FFFF00200140007AF01F8038010095
:109A400000230140704700BF01483AF09BB800BFB7
:109A50004C200120084810B4D0F82C38D0F86048C9
:109A600099691A682CB1234600F62C005DF8044B66
:109A700018475DF8044B70472018012001483AF060
:109A800081B800BFAC200120084810B4D0F88C3851
:109A9000D0F8C04899691A682CB1234600F68C00AA
:109AA0005DF8044B18475DF8044B704720180120FF
:109AB00001483AF067B800BF0C210120084810B4F3
:109AC000D0F8EC38D0F8204999691A682CB12346AF
:109AD00000F6EC005DF8044B18475DF8044B704746
:109AE0002018012030B40469002341684025E4684F
:109AF00082690C31546244699560536093631160CC
:109B0000C2E90333C2E90533C2E90733C2E90A33C4
:109B1000C2E90C3384B1C269E0689363506211609A
:109B2000C2E90133C2E90333C2E90533C2E90733AD
:109B3000C2E90A33C2E90C3330BC7047114A037AD8
:109B40000168D35C10B4CC58CA1824F00104CC507E
:109B50001368DB07FCD4037D1F2B09D9203B20228F
:109B60005DF8044B02FA03F343F01803CB6070472F
:109B700020225DF8044B02FA03F343F018038B60D4
:109B8000704700BF486B0508F0B50668356A0029C4
:109B90005CD12F68AC68D6F818E0002F5FD0364B48
:109BA0003B40B3F1005F61D007F01F0104F11F03D8
:109BB00027F01F02194421F01F01BFF34F8F002926
:109BC0000BDD114402F12003DFF8B0C08B42CCF86A
:109BD00068221A4603F12003F8D1BFF34F8FBFF379
:109BE0006F8F03684FF48062CEF80470CEF81420B3
:109BF0005B69CEF8204043B36868F669002837D027
:109C00001D4B0340B3F1005F1AD000F01F0220F09B
:109C10001F011F32224422F01F02BFF34F8F002A80
:109C20000ADD0A4401F12003144D9A42C5F870126E
:109C3000194603F12003F8D1BFF34F8FBFF36F8FA5
:109C40004FF48063706073613462F0BDEC69002C86
:109C5000FBD06F691435D6F818E0002F9FD1084A61
:109C60003346CEF81470CEF80420C1E73346B9E786
:109C7000044B70617360E7E70000FFFF00ED00E058
:109C80004400002048000020F8B507680646D7E9E0
:109C90000454002C50D0A0612B7D1F2B39D82022DA
:109CA000286802FA03F343F018038360237D1F2B17
:109CB0003AD92022203B02FA03F3226843F018032A
:109CC000D3606368002269680A601A601A6842F00B
:109CD00010021A60BA69297A40F0BAFEFA69217A4C
:109CE000206840F0B5FE2A7A2A492F6833688D5CD7
:109CF0005A687B59206843F001037B51237AC95C81
:109D0000435843F001034350536843F00303536047
:109D1000F8BD203B2022286802FA03F343F0180321
:109D2000C360237D1F2BC4D8202202FA03F32268CC
:109D300043F018039360C4E72A7D6B681F2AA8616B
:109D40001FD82021286801FA02F242F0180282602E
:109D50000021BA691960196841F010011960297A67
:109D600040F076FE2A7A0B4933682868895C5A6885
:109D7000435843F001034350536843F002035360D8
:109D8000F8BD203A2021286801FA02F242F01802B8
:109D9000C260DDE7486B050810B1036882889A61EC
:109DA000704700BF18B1838802681B049361704735
:109DB00008B51D200DF0F6F908B183794BB11E20CE
:109DC0000DF0F0F908B1837903B108BD5523C380C4
:109DD00008BD5523C380F2E7D3B2012B23D802EB91
:109DE00042024FF0000C70B54FEA820E0F4C6346F2
:109DF00022460EF1080504E00133172B11D012F8AA
:109E00001CCF6045F8D192F801C08C45F4D1565969
:109E1000002EF1D0C3EBC3030EEB83030433E01831
:109E200070BD002070BD0020704700BF78F50408A9
:109E300010B40C4C002304F6981C01E0152B0CD038
:109E400003EB430201331CF802108142F6D1224495
:109E50005DF8044B92F99A0970474FF0FF305DF8B6
:109E6000044B704720180120D3B2022B21D802EBFB
:109E70004202002330B54FEA820C0F4D0F4C2A46A8
:109E80000CF10C0E04E00133172B10D052F82C4FBC
:109E9000A042F8D114798C42F5D152F80E40002C32
:109EA000F1D02C2202FB03C30833E81830BD002098
:109EB00030BD0020704700BF28F0040800000140BA
:109EC000002838D0002330B51B4D90F804C005F6AB
:109ED000981401E0152B2CD003EB43020133A15C55
:109EE0006145F7D12A44046890F805E092F99A395F
:109EF000DAB2022A1DD803EB4303104810494FEA97
:109F0000830C024600230CF10C0504E00133172BEF
:109F10000FD052F82C1F8C42F8D111797145F5D130
:109F200051590029F2D02C2202FB03C308331844F4
:109F300030BD002030BD70472018012028F00408F3
:109F4000000001400348D0F890300BB18030184732
:109F5000704700BF000001200348D0F8B4300BB1B7
:109F6000A4301847704700BF000001200348D0F814
:109F7000D8300BB1C8301847704700BF000001202F
:109F80000348D0F8FC300BB1EC301847704700BFE5
:109F9000000001200348D0F8203113B100F588708B
:109FA00018477047000001200348D0F8443113B12E
:109FB00000F59A7018477047000001200348D0F858
:109FC000683113B100F5AC701847704700000120EC
:109FD0000348D0F88C3113B100F5BE7018477047B4
:109FE000000001200348D0F8B03113B100F5D07063
:109FF00018477047000001200348D0F8D43113B14E
:10A0000000F5E27018477047000001200348D0F8BF
:10A01000F83113B100F5F4701847704700000120C3
:10A020000348D0F81C3213B100F50370184770478D
:10A03000000001200348D0F8403213B100F50C7045
:10A0400018477047000001200348D0F8643213B16C
:10A0500000F5157018477047000001200348D0F83C
:10A06000883213B100F51E701847704700000120B8
:10A070000348D0F8AC3213B100F527701847704789
:10A08000000001200138074B074A00EBC00003EB3A
:10A090008000D0F8800090420CBF952096203EF0C2
:10A0A000C9BB00BF000001200060024001382DE95B
:10A0B000E84100EBC000134D1E46134B05EB800535
:10A0C00090460F46D5F8800098420CBF9520962008
:10A0D0003EF0B0FB95F995004FEA9811C5F89070E5
:10A0E000C5F898603EF076FB95F99530002B07DBBC
:10A0F00003F01F0001225B090449824041F823203C
:10A10000BDE8E881000001200060024000E100E0BD
:10A11000800AA0F58010522808D8054B184490F802
:10A12000F4330D2B02D8034AD056704700207047F5
:10A1300028F00408386B05080120FEF759BC00BF61
:10A140000220FEF755BC00BF0420FEF751BC00BF43
:10A150000820FEF74DBC00BF1020FEF749BC00BF31
:10A160004FF47870FEF744BC4FF47C40FEF740BCDF
:10A1700030B1036882881B691A4214BF0120002095
:10A18000704700BF2DE9F04F884683B0044617465C
:10A19000002800F0BC8002685E4B13449B0A5E4AB4
:10A1A000C8F3411B134493F8D4073EF043FBC8F3B4
:10A1B0008103B4F804E008F00302256801939EFAD5
:10A1C000AEF0B0FA80F002F1FF3A3EFA00F35ED052
:10A1D0000126032103E001303EFA00F357D006FACE
:10A1E00000F313EA0E03F6D0D5F8009093FAA3F427
:10A1F000B4FA84F493FAA3FCBCFA8CFC6400BAF1C0
:10A20000010F4FEA4C0C01FA04F402FA0CFC29EAA3
:10A21000040444EA0C042C6049D9D5F80C9093FA54
:10A22000A3F4B4FA84F493FAA3FCBCFA8CFC6400A3
:10A23000022A4FEA4C0C01FA04F40BFA0CFC29EA4E
:10A24000040444EA0C04EC60C5D193FAA3FCBCFA04
:10A250008CFC1C0ABCF1070F41DC2C6A93FAA3FCAE
:10A26000BCFA8CFC93FAA3F34FF00F09B3FA83F313
:10A270004FEA8C0C01309B0009FA0CFC07FA03F33F
:10A2800024EA0C0423432B623EFA00F3A7D1BAF16F
:10A29000010F09D86B68C8F3001823EA0E030EFB00
:10A2A00008FE4EEA03036B6003B0BDE8F08FD5F8FB
:10A2B000089093FAA3F4B4FA84F493FAA3FC64002C
:10A2C000BCFA8CFC01FA04F44FEA4C0C29EA0409AC
:10A2D000019C04FA0CFC49EA0C04AC609DE7D5F83B
:10A2E00024C094FAA4F9B9FA89F994FAA4F30F24D2
:10A2F000B3FA83F34FEA89099B0004FA09F907FAD4
:10A3000003F32CEA090C4CEA03036B6263E74FF09A
:10A31000FF3344E70000FEBF28F0040800B131E736
:10A3200070472DE9F84FC04F6023064603FB0073CA
:10A33000D3F81848002C00F06B81D3F820A8BAF1AC
:10A34000000F04D09AF80630002B40F061816023A2
:10A3500003FB0673D3F824581DB1AB79002B40F0F2
:10A360005781731CDBB2BAF1000F04D015228AF8B2
:10A3700007308AF8062015B11622EB71AA714FF04A
:10A380006009207C3EF056FA294609FB06F9504642
:10A3900041F030FE042207EB0908504698F82838AF
:10A3A000002B14BF3E211E21FFF7B8FF98F8283874
:10A3B00028469E4D002B4FF004024D4414BF3E2111
:10A3C0001E21FFF7ABFF4C220021284644F05EFC23
:10A3D000D8F818389FED967AB0EE084A5B68F7EE29
:10A3E000003AB8F82A984FF0000EC8F82C3840F21E
:10A3F0001458904B9FED905A9A68904BC2F382226A
:10A40000134493F8DC27D7F82C33D34007EE903A67
:10A41000F8EE677AC7EE275A07EE909A9FED887A92
:10A42000F8EEE77AC7EE274ADFED867AB0EE007ADB
:10A43000E5EE877AA5EE875A25EE844A37EE856ADF
:10A4400074EEE72AB9F5C87F0EF1010CD5BF64237D
:10A4500032234FF49670782007EE90CAD8BF4FF49D
:10A46000167A0344C8BF4FF4827AB8EEE77AD8BFB1
:10A47000414607EE903AC8BF4FF4FA7127EE257AAD
:10A4800001EB0A03F8EEE76A86EE873A73EE636A39
:10A49000FCEEE67A17EE902A07EE90AAB8EEE73ABD
:10A4A00007EE903AF8EEE77A23EE243AC3EE276AF5
:10A4B00036EEC53A72EEE66AC3EE077A77EEE37AD5
:10A4C000FCEEE77A17EE901AC6EE877A77EEE37A1B
:10A4D000FCEEE77A17EE903A03F1020A0AEB010B61
:10A4E000F0EE466A07EE90BAF8EE677AE7EE276A72
:10A4F000F4EEE64AF1EE10FA00F38E805FFA82FA8B
:10A50000BAF10F0F00F28A80323807EE900AF8EEA7
:10A51000E77A77EEC47AC7EE876AFCEEE67A17EE42
:10A52000900A5FFA80FABAF10F0F77D81FFA81FA12
:10A53000BAF1FF0F72D81FFA83FABAF1FF0F6DD884
:10A5400012054AEA0E7302F07F620004134300F41E
:10A550007F003D4A034302EA01210B43602000FBD8
:10A56000067600272846C6F830380123C6F8347826
:10A57000C6F83838C6F83C78C6F84078C6F8487847
:10A58000C6F84C7841F020FA96F86D38202BD9B2F5
:10A590001AD196F86C38012B16D0242386F86D3822
:10A5A000D6F82C381A6822F001021A601A6822F4D0
:10A5B00080521A601A681A601A6842F001021A6022
:10A5C00086F86D1886F86C78002194F912003EF038
:10A5D00001F994F91230A27C002B07DB02F01F0175
:10A5E00001225B098A40194941F82320002194F98E
:10A5F00011003EF0EFF894F91130627C002B07DB7C
:10A6000002F01F0101225B098A40104941F8232012
:10A61000BDE8F88FE64615E701315FE7BCF10F0FA3
:10A62000F8D100239AE700BF201801204C20012018
:10A63000286B6E4E003802400000164328F00408D4
:10A64000002474490000704200FFFF0000E100E0B8
:10A650002DE9F047814DC0EB001605EBC606D6F894
:10A66000D839002B00F0B8800446070196F8480A54
:10A670003EF0E0F896F8483A012203F01F015B092A
:10A68000013B8A40032B0AD8DFE813F0DC0004000A
:10A69000E200D60072494B6A23EA02024A623B1B7F
:10A6A00004F1010905EBC3035FFA89F993F8DC09AA
:10A6B0000CF078FD064618B1122380F807908371DC
:10A6C0003B1B05EBC30393F8DD090CF06BFD8246E1
:10A6D00018B1132380F8079083713B1B05EBC3036C
:10A6E00093F8DE090CF05EFD804618B1142380F863
:10A6F000079083713C1B50462E2105EBC40595F84D
:10A70000E029FFF70BFE95F8E1290E214046FFF7FF
:10A7100005FE95F8DF292E213046FFF7FFFDD5F81D
:10A72000D83950491A688B4222F040021A6055D03D
:10A730004D4A934269D002F58062934258D1484A0B
:10A74000116A41F400411162116A21F40041116261
:10A750005A6842F480525A601A68520634D4434907
:10A760001E68D1F8D442D1F8E002D1E9B025B0F5A5
:10A77000005F42EA0502D1F8CC5242EA0502D1F864
:10A78000D05242EA0502D1F8D85242EA040242EA23
:10A790000502D1F8DC5242EA0502354D42EA0002D8
:10A7A00005EA060542EA05021A60D1F8C8225D688A
:10A7B00042EA14422F4C04EA050442EA04025A60B9
:10A7C00002D1B1F8E4221A61DA6922F40062DA6196
:10A7D0001A6842F040021A60BDE8F087204A516AC8
:10A7E00041F480515162516A21F480515162AFE7C6
:10A7F000214A934213D11A4A516A41F400515162DD
:10A80000516A21F400515162A2E7154A116A41F4DC
:10A8100080411162116A21F48041116298E7174A60
:10A82000934295D10E4A516A41F480115162516AA6
:10A8300021F4801151628BE709490B6923EA020276
:10A840000A612CE706494B6923EA02024A6126E7BE
:10A8500003490B6A23EA02020A6220E7201801205A
:10A860000038024000300140003800400000012064
:10A870004000FFFFFBF0FFFF0034014000500140AB
:10A8800008B100227EE470472DE9F041CB781BB976
:10A8900000263046BDE8F08100F110070C46054661
:10A8A000897838460BF040FF06460028F0D0E07863
:10A8B0000CF078FCA86123780133DBB210B1C371CE
:10A8C000222383710D21FFF7DBFFA869FFF764FAEC
:10A8D0000F4AD2F8D432632BFBD90E480BF010FF8D
:10A8E000DFF838800C4BA88202E058F8043B53B1E3
:10A8F0003846984703460028F7D0286985F8D830AD
:10A9000041F042FCC5E7E0781E460CF0A9FCC0E728
:10A910002018012040420F006111040810F80408BB
:10A9200070B50E4CD4F81C6F002E15DD04F587644D
:10A93000002503E0B54204F120040DD0237F01354A
:10A94000002BF7D0E06800220028F3D0217D2034CE
:10A95000FFF718FCB542F1D1012070BDC8010020FD
:10A96000AB4B2DE9F04F91B093F8CA8BA94B002562
:10A97000A94F0093A94BA3F50D6ADFF8B892DFF851
:10A98000B8B24E46B30AA3F58013522B55D85344A0
:10A9900093F8F4330D2B50D8B8F1010FFC5640F06A
:10A9A0001E81012C3FD14FF000094946204610F08E
:10A9B00039FF10F0BFFF90F800C0BCF1000F18BFC6
:10A9C000BCF1540F14BF4FF0010C4FF0000C40F0DD
:10A9D000028109F104091FFA89F9B9F1100FE4D1D4
:10A9E000002D00F0BA808B4A00210DE0534493F80B
:10A9F000F4330D2B0FD8FB56A3420FD0013102F5D3
:10AA00008672A94280F2A580906803689B0AA3F52C
:10AA10008013522BEAD90023A342EFD143799BF84C
:10AA200005009842EAD17D4B5B4513D05BF81C6F63
:10AA3000B30AA3F58013522BA9D9B8F1010FF2D0B4
:10AA400001230024B8F1020FADD1002BABD0734B22
:10AA50005B45EBD1009B013503F58673042D009314
:10AA60008BD1DFF8D8814FF0000B08F59E77A8F561
:10AA7000876ADAF81C3F5B4568DDD8F80C60002E69
:10AA800064D098F81030B088D6F80090DAF8045006
:10AA900063490193B0FA80F34944002D0293C3F156
:10AAA0001F034FEA9121009340F3CD80594B0024BE
:10AAB00005E0013403F58673AC4200F0C1801A68EA
:10AAC0008A42F6D14FF48673524A03FB0424009A5B
:10AAD0000BF1010B019B5100C8F8042088F81030DD
:10AAE0000323C8F80C6003FA01F5C8F81840B371E5
:10AAF000012386F807B01646A26C03FA01F12A4337
:10AB0000A264226D0A4322659AF80020002A6BD0C5
:10AB100003FA06F11A46636D0B4389B26365C9F8FF
:10AB20001800D4F8AC00FDF7E7FA204608F1200839
:10AB3000FDF7B6FA0123BBF1080F07F1180708F873
:10AB4000043C08F8033C07F8073C92D111B0BDE87B
:10AB5000F08FBCF1000F7FF466AF5846FDF764FA42
:10AB60009BF80540C3B2022B00F24C83431C2D4AD4
:10AB70005BB203EB430398002B4B03F5727104E0C7
:10AB8000994200F03F8353F82C2FB242F8D11A7942
:10AB9000A242F5D11A58002AF2D094460023234A43
:10ABA00051680133614513D0102B02F12402F7D113
:10ABB0004FF0FF3303EBC3031D4A02EB830393F80B
:10ABC0009C30002B7FF42FAF009BC3F808B041E707
:10ABD000DBB2013BEEE7002D7FF405AF23E7B4F1D4
:10ABE000080318BF01232DE702990004C1F12F05C6
:10ABF000009903FA01F1AB40656D89B22B4363659F
:10AC0000C9F81800D4F8AC00FDF776FA8DE700BF5C
:10AC100020180120D0010020386B0508F8F804083E
:10AC20000000FEBF0000014028F004088000012061
:10AC3000000001200004014018F80408000600206C
:10AC4000032C00F399824FF4867303FB05A3186964
:10AC5000002800F0C18299600131CAB283F8112145
:10AC60000492542283F810216B1C0268CAF8043045
:10AC700044790392FDF7D8F9A04B864693F8E13B5F
:10AC80000593C3B2022B00F2BD8200F1010C9C4976
:10AC90009C4800234FFA8CFC039A0CEB4C0C4FEAB7
:10ACA0008C0C05E00133172B00F0AC8251F82C0F0F
:10ACB0009042F7D10879A042F4D151F80C00002855
:10ACC000F0D02C210EEB4E0E002401FB03F303EB1E
:10ACD0008E0E8B4B734419694FF4867303FB05A3E7
:10ACE000C3E90701884B9C46DCF80410884217D062
:10ACF00001340CF1240C102CF6D1844B93F87820FD
:10AD0000002A00F06282824B82488349834AC3F85A
:10AD10004804C3F84014C3F8502411B0BDE8F08FC4
:10AD2000611C7A48C9B2013901EBC10100EB810114
:10AD300091F89C0006900028E5D104984FF08C0C07
:10AD400081F89D004FF4867000FB05F420465424E2
:10AD500081F89C400446811071480394544400FBE0
:10AD600001F1C4F800C101FB0CF001EB4101C4F892
:10AD70000C9001EB011C6B4901EB4000A1F54C71FB
:10AD800001EB8C01C4F8FC00C4F8B4103321C4F802
:10AD9000B8106549039C0C195849D1F82C930599B2
:10ADA000062900F00E82072960486149DFF888E132
:10ADB0000CBF84468C465F4908BF71461046059318
:10ADC000039BB9FBF1F1B9FBFCFC4A1E4FF48679F9
:10ADD0000CF1FF3192B209FB05A9A9F8BC1003F1EF
:10ADE0005801A9F87420504B226600221944A4F897
:10ADF00058206266E2653FF0A7FDD9F81030186868
:10AE00000493026842F0800202605A79059B0C2A82
:10AE100008D8DFE802F06B070707640707075C073D
:10AE2000070754004FF4867202FB05A251694FF0E8
:10AE3000600C02684FF000094FF0020ECDF820C000
:10AE40004FF4807C22F00102CDF82890CDF838C074
:10AE50004FF0010CCDF83490CDF824C04FF00A0C1F
:10AE6000CDF83C900593CDE90BCE026008AA3FF0E7
:10AE700029FC4FF48672049B02FB05A219685269F3
:10AE8000059B012A5AD0042A58D0102A00F0A98123
:10AE9000402A53D0B2F5807F00F0A681B2F5806FD2
:10AEA00000F0A281B2F5805F00F0A481B2F5803F8E
:10AEB0004FF03C090CBF08224FF400623FE04FF412
:10AEC00086724FF4805102FB05A25161AFE74FF447
:10AED00086724FF4807102FB05A25161A7E74FF41F
:10AEE0008672102102FB05A25161A0E74FF4867221
:10AEF000012102FB05A2516199E700BF2018012042
:10AF000028F004080000014080000120000001201A
:10AF1000C0120020F1550108ED550108F95501084E
:10AF20006B4CA407501A0020D001002010552200BD
:10AF300044950800D0DD060040771B00082201F18F
:10AF4000180050F809C042EA0C0240F80920049A9F
:10AF50001079002840F01C814FF48671002201FB1B
:10AF600005A1D1F810C0C869DCF800C0DCF80010F9
:10AF700041F00101CCF8001059680132884200F01C
:10AF80000381102A03F12403F6D14FF0FF339F4AC7
:10AF900003EBC30302EB8303D3F880009C4B98427E
:10AFA0000CBF952096203DF045FC4FF4867303FBC3
:10AFB00005A31A6953790C2B00F2E380954901EB44
:10AFC0004303B3F8ECC84FF486731068924903FB4F
:10AFD00005A3A3F818C0002306E0904200F0088102
:10AFE0000133042B00F00B8151F83320002AF4D1F7
:10AFF000DAF8202F0132CAF8202F0AEBC302DB0057
:10B00000C2F8240F1944069823469022B1F804E0B0
:10B01000DFF818924CEA0E0CA1F804C07F49FFF744
:10B0200045F84FF486734FF4403C402103FB05A5DF
:10B030000023E869026842F010020260026842F0F0
:10B0400014020260C4F8A830C4E91F33C4E92833ED
:10B0500004232A6AC4F898C04FF4804CC4F89C308A
:10B060004FF48063A167C4F88430C4F89420D5F805
:10B07000B820C4F89020C2B220F0FF00103AA9FB1B
:10B080000231EA68039B1832090922674FF48052A3
:10B09000C4F8882003F17002614B1A44D5F8B4302B
:10B0A000C4F88CC063673FF0D3FCE869039B4FF49E
:10B0B0000031D0F800E04FF4006C03F1B802584BB7
:10B0C000C4F820E0D0F814E01A440023C4F824E0C7
:10B0D000D0F804E0C4F828E0D0F808E0C4F82CE088
:10B0E000D0F80CE0C4F8C830C4F830E0C4F8F03050
:10B0F000C4E93033C4E93A332B6A03930423C4F818
:10B10000E4304FF48063C4F8CC30039BC4E937319A
:10B11000D5F80031C4F8D830C3B220F0FF00103B9E
:10B12000A9FB0331EB68C4F8D0C010330909C4F897
:10B13000B830D5F8FC3003934FF48043C4F8D430D2
:10B14000039BC4F8BC303FF083FCEB69B0881A68FD
:10B15000D6F8009062635A69A2635A68E2639A68FB
:10B160002264DA6862641A6842F010021A601A688F
:10B1700042F014021A60AAE403232A4A82F8E03B50
:10B18000C1E54FF0000C1EE7D3B20693013BFEE68B
:10B19000079305910CF006F805998146079B58B175
:10B1A00005930221049BDA79FEF7ECFF049B5422FD
:10B1B000A9F806201968059B4A6C42F400424A64CB
:10B1C000CAE6DFF86CC01849F8E50499542283F800
:10B1D000791083F8782096E50223124A82F8E03B42
:10B1E00091E54FF40062AAE608224FF00409A6E6B2
:10B1F000DB0007E74FF400624FF004099FE60023ED
:10B200009B88FFDE00235B68FFDE00BF000001209B
:10B210000060024028F00408EC100020458100087E
:10B22000D001002020180120A0BB0D00ABAAAAAAC3
:10B23000882A1100F8B590F8B2311C09013C052CA0
:10B240000FD81B4E054603F00F0306EB4402B2F87D
:10B25000080940FA03F2D20703D595F8BD71012F12
:10B2600001D00120F8BD07FA03F33444013B184034
:10B2700041F07CFF94F8142913180E4A02EBC30125
:10B2800052F833208B8810691840EBD0002395F8D2
:10B29000B3210846022185F8BD31FEF773FFD5F8CA
:10B2A00020213846136843F008031360F8BD00BF3F
:10B2B00028F00408042401202DE9F04F00228DB06D
:10B2C0002F21074610F08EFBD0B19B4E05464379E7
:10B2D000D0F80080A6F83C34FEF7F2FD80B1446857
:10B2E00074B1DFF88CB2002259464B680132243128
:10B2F0009C4210D0102AF8D1904B93F878201AB1C4
:10B3000000200DB0BDE8F08F2F21104683F8792082
:10B3100083F87810F5E7D2B2DFF820A2013A02EB09
:10B32000C2020AEB820292F89C90B9F1000FE7D1B9
:10B330002F218368C6F8FC83A2F89C10D6F82C2332
:10B340007F4901938A4280F0D8804946120AC6F8A4
:10B3500000147C490020A1FB02317B4BC6F80C0491
:10B360000A09C6F804040909A3FB0232C6F8081446
:10B370005208A6F8E62E5200A6F8E42E96F83924D4
:10B3800002F0FF01002A00F0C480022240466F490B
:10B3900086F8392438F076FF0122384686F83924B9
:10B3A0000BF000FFC6F8E80E28B12F21C1804E2116
:10B3B000EA79FEF7E7FE664A0021019BC6F8F81E0F
:10B3C000C6F8F03EC6F8081FC6F8101FC6F8181FCA
:10B3D000C6F81C1F106BC6F8EC4E40F4001010634A
:10B3E000106B00F4001003900398106B40F4800081
:10B3F0001063126B02F480020492049A4022C6F891
:10B40000F42E4FF48062C6F8FC2E4FF48052C6F83A
:10B41000002F4FF48042C6F8042F4FF40032C6F8D4
:10B420000C2F0322C6F8142F96F83C240C2A73D84C
:10B43000484901EB4202B2F81C79B8460837464841
:10B440005946002206EB870CCCF8FC03A0F52F60D0
:10B45000C6F8240F486801322431844262D0102A91
:10B46000F8D14FF0FF3202EBC2020AEB820A3B4AEC
:10B47000DAF8800090420CBF952096203DF0DAF972
:10B480000022DBF8041001320BF1240B8C4246D071
:10B49000102AF6D106EB870748464346602230491A
:10B4A000FEF704FED7F8FC0338F076F800287FF4A6
:10B4B00027AF60210A90AB79059159000B90DB0012
:10B4C000069001F00201099003F00803B6F83C244D
:10B4D0002448CDE9071305A93CF0A4FD00287FF41A
:10B4E0000FAFAB79B6F83C149B071E481DD538F05A
:10B4F000C9FFB0FA80F0400903E71B491B4811441B
:10B50000A0FB0131890D013989B2481CB2FBF0F270
:10B510001CE786F8381438E788460F468EE75FFA4E
:10B5200082F9B7E7D2B2013A9DE738F07BFEB0FA74
:10B5300080F04009E5E600BF20180120000001204E
:10B54000006CDC02598B4F01ABAAAAAA201C012077
:10B550000038024028F004080C2701200060024057
:10B56000159000081C1C012000366E01819F5E169C
:10B5700080000120014B43F8201070475028004004
:10B580001D4B1E48196C1E4A41F0805130B419649D
:10B5900082B0196CFF2401F080510191019901687A
:10B5A00041F480710160CA20196C41F48061196412
:10B5B000196C01F4806100915321009D5462506226
:10B5C00051625B6FDB000DD40E4B00210E4A43F835
:10B5D000041B9342FBD10D4B0D4AC3F8502802B017
:10B5E00030BC7047094A0A4BD2F850289A42EBD136
:10B5F00002B030BC704700BF00380240007000400D
:10B6000000280040542800406C28004000200040E2
:10B61000316665422DE9F0470646086888B00C4659
:10B620004FEA902CBDF84080ACF5801C9DF844900A
:10B63000BCF1520F64D8374FBC449CF8F4530D2D25
:10B640005ED81946FDF724FD334A2368617902EB81
:10B65000851A94F806E0B9F1000F54D1F4469B0A1C
:10B66000A3F58013522B23D83B4493F8F4030D2801
:10B670001ED84FEA4C034FF480774FEACC0CCDF83C
:10B68000088003F0020302EB80100A4601A903932D
:10B690000CF008030493602301934FF40073CDE989
:10B6A0000673002305933CF0BDFC617994F806E035
:10B6B0001EF0020F504629D038F0E4FE174BA801C7
:10B6C000022203EB8515D5F8401485F87D24144A31
:10B6D0008D682A40062A06D0B2F5803F03D00A685A
:10B6E00042F001020A600344012283F87D242168AC
:10B6F000637901F1340271600021D0183060D150BB
:10B7000008B0BDE8F0878EF0010CA8E738F08AFD9C
:10B71000D4E700BF28F00408601C01202018012095
:10B7200007000100F0B50446D0F89400434B83B005
:10B73000A16804F1640204F118070E68C1B220F098
:10B74000FF0001921039A3FB013109093FF0CAF94A
:10B75000616D0023019A012984F8583018D004291A
:10B7600016D0102955D0402912D0B1F5807F53D082
:10B77000B1F5806F50D0B1F5805F55D0B1F5803F05
:10B780004FF03C030CBF6FF0080C6FF4006C01E04D
:10B790006FF0080C06F118053046E95801EA0C0173
:10B7A000E950616D3EF08EFF636D012B16D0042BC6
:10B7B00014D0102B0FD0402B10D0B3F5807F2FD09A
:10B7C000B3F5806F2CD0B3F5805F31D0B3F5803FF7
:10B7D00006F1540502D04FF4006100E008212B6807
:10B7E0003A46D4F894000B4340212B602162C1B249
:10B7F000124B20F0FF001039A3FB013109093FF083
:10B8000027F9D4F89420136843F01003136003B0B1
:10B81000F0BD6FF4006CBDE76FF0080C0423B9E7CE
:10B8200006F11C050821DAE76FF4006C0423B1E788
:10B8300006F11C054FF40061D1E700BFABAAAAAA2C
:10B840002DE9F04FDFF85CB29BF800402DED028B44
:10B8500087B034B90124204607B0BDEC028BBDE8A7
:10B86000F08F8B4BDFF840A2D3F8D43208EE103AB9
:10B870000BF0F0FF9AF8243C0390002B00F00181BC
:10B880000BF234670BF634330BF63C4400263D468E
:10B8900001930597DAF81C34039AD31A03D4EA6D9E
:10B8A0009A4200F3D08006EB86030BEB431393F828
:10B8B0008C3603F0FF020292002B00F08D80D5F849
:10B8C0009410AB6873481A68CBB221F0FF01103BAB
:10B8D000A0FB030370481B09C35C19444B68A9898A
:10B8E0001FFA83FCD368CCF1160C23EA0103BCF1E8
:10B8F000070FD36070D9DBF83C3B002201210133F4
:10B9000096468946CBF83C3BD5F89C301F460493BD
:10B9100057F8048B40461CE0D7F80080BEF1140FA6
:10B92000A8EB000340461CDC13F1080848BF03F1F4
:10B9300017084FEA28130EEB281E03F1FF380131D8
:10B9400002FA03F3043709FA08F28C4542EA0302CB
:10B9500007D38C45E0D8CEF1150338684FF0150EAB
:10B96000EBE7BEF1150F65D14C49C2F38423C2F356
:10B97000441001EB830301EB8000D3F83839D0F891
:10B9800038091B0243EA001302F01F00C2F3C4325D
:10B9900001EB800001EB8202D0F83819D2F8382987
:10B9A0000B4343EA023383EA132282EA121202F0C3
:10B9B0000F020F2A3ED1C3F30F134FF6FF729342CB
:10B9C00038D0B3F5606F45D0019A9381029918EE93
:10B9D000102A20460AF03AFE019B284601365C34C4
:10B9E0001433A0350193FFF79DFE9AF8243CB3422F
:10B9F0003FF750AF0122059F8BF8382C0022CAF880
:10BA00001C24002B3FF426AF03EB830307EB431307
:10BA10003A7CA03757F84C0C12F0020F57F8982CCC
:10BA200011680A6A14BF42EA80020243BB420A62FA
:10BA3000EED10FE7DBF8383B0133CBF8383BCEB122
:10BA400000230293C2E70024204607B0BDEC028B1E
:10BA5000BDE8F08F0E4991F8EC2302EB420201EBB6
:10BA6000C202324492F899230D2AADD18023019A63
:10BA70009377ABE704995822094843F093F802966C
:10BA8000A4E70122CAF81C348BF8382CE3E600BF87
:10BA900020180120ABAAAAAA486B050828F00408C0
:10BAA000A80D0020C8010020C0120020D0F82011ED
:10BAB000242200232DE9F041C0F8942104460A68AD
:10BAC000806804F5907522F001020A600B604B60FB
:10BAD0008B6094F805C0C4F89C314FEA8C22C4F8FE
:10BAE000943184F8903102F48052C4F89831C4F84B
:10BAF0003831C4F828214FEA0C32C4F8403102F43E
:10BB00000052C4F834312379C4F82C214FEA0C22B6
:10BB1000C4F8240113F0010002F48062C4F830215B
:10BB200002D00422C4F8342113F0020305D0D4F863
:10BB3000342142F00802C4F834211CF0010F0DD06A
:10BB400048B1D4F8442142F00202C4F844214FF431
:10BB50008032C4F84C21002B40F0FF80A84B03F149
:10BB6000200053F8042F944200F0BD809842F8D191
:10BB70001CF0080F40F0CD80D4F89431002B00F079
:10BB8000168124232846C4F894310B6823F001035E
:10BB90000B6038F09BFC012815D0D4F84431002B01
:10BBA00040F01881D4F8203128465A6822F4904297
:10BBB0005A609A6822F02A029A601A6842F00102DA
:10BBC0001A603FF0D5FE2379DA0761D5D4F8FC205E
:10BBD000002A00F0D9800023D4F8041104F13C06B7
:10BBE000E263A3644FF480623046E264C4E9101358
:10BBF000C4E91433C4E91833C4E91A334FF4803369
:10BC0000E3654FF48073A3653FF02CFF304637F0B7
:10BC1000C3FCD4F89881C4F88C61B8F1200F656733
:10BC200031D1E368626999B26AB3B1FA81F77F09E9
:10BC300049B394F89001012825D030460126C4F874
:10BC40009C710B4684F890612226A4F87811C4F800
:10BC500098616C4ED4F82011A6676B4E2431C4F85D
:10BC60007421E667694EC4F88C70C4F8886037F0B8
:10BC700031FD002800F0B280102384F89071C4F8E0
:10BC80009C31C4F89481E26B23795268C4F8142182
:10BC90009B0777D5D4F80021002A69D00023D4F877
:10BCA000081104F19C06C4F89C20C4F8A830402276
:10BCB000C4F8B8303046C4E92C33C4E93033C4E9A1
:10BCC00032334FF48033C4F8BC304FF48063C4E99E
:10BCD0002812C4F8AC303FF0C5FE304637F05CFCAB
:10BCE000002867D0FEE7002C3FF442AF94F8BC3147
:10BCF000002B3FF43DAFD4F844311CF0080F43F063
:10BD00000803C4F844314FF40043C4F854313FF4FD
:10BD100033AFD4F89431002B55D024232846C4F8EF
:10BD200094310B6823F001030B6038F0CFFB01283E
:10BD30003FF449AFD4F84431002B47D1D4F8203137
:10BD400028465A6822F490425A609A6822F02202E9
:10BD50009A609A6842F008022EE7D4F8443143F022
:10BD60000103C4F844314FF40033C4F84831F5E618
:10BD7000D4F8A0311A6842F080021A601A6842F0C2
:10BD800040021A60BDE8F081D4F8A021116841F4A6
:10BD900080711160916841F001019160116841F07A
:10BDA00020011160116841F01001116070E784F802
:10BDB0009031E6E6D4F89C30C4F88861C4F8D450D9
:10BDC0005860BDE8F08184F89031A6E7284638F045
:10BDD00037FDB3E7284638F033FDE3E6D4F82031E9
:10BDE00084F890011A6842F480721A609A6842F0EE
:10BDF00001029A609A6842F040029A6043E700BFED
:10BE0000E81E0020D10704080108040805080408FA
:10BE1000F8B5EFF31185502383F31288D0F8003181
:10BE20001B6813F0010303D0EDB285F31188F8BD50
:10BE3000D0F894210446D0F898110A4302F0210268
:10BE4000212AF1D0D0E90901884253D043D8226990
:10BE50001846531A9BB2D4F894710022A062202F86
:10BE600084F8A421E0D1A2695118DDD0B3FA83F699
:10BE70007609002BD8D094F89021012AD4D0012241
:10BE8000D4F88801A4F8723184F890212122C4F8F2
:10BE90009C61C4F86C11A4F87031C4F89421E8B125
:10BEA000DFF858C0D4F82021C0F83CC0DFF850C0FB
:10BEB00028320665C0F840C0DFF848C0C0F84CC062
:10BEC00037F008FC50B1102384F89061C4F89C311D
:10BED000C4F89471A8E7431A9BB2BCE7D4F82031A8
:10BEE00000224021196284F890219A6842F0800271
:10BEF0009A6099E7012384F8A43195E7A90704081B
:10BF0000CD0704080508040870B5D0F8204105469F
:10BF1000E369990614D5606AEB6AC0B2002B74D04D
:10BF2000296B9847D5F82041236823F48073236058
:10BF3000A36823F00103A360A36943F00803A3618E
:10BF4000E369DA0701D501232362E3699B0701D581
:10BF500002232362E3695E0701D504232362E369B8
:10BF6000180701D508232362E369590614D5402335
:10BF7000236295F8BD61002E31D0D5F80031CBB1E8
:10BF80002846FFF745FF95F8A4311BB195F8BD6130
:10BF9000002E4BD0D5F82041D5F8003163B1E369CC
:10BFA000DB0606D56B6B13B19847D5F820411023FB
:10BFB000236270BDD5F82041E3691A06EFD5D5E9B3
:10BFC000092393422DD0AA69D25C0133D2B2A26276
:10BFD0002A69B3FBF2F102FB1133AB62DFE795F89C
:10BFE000B2010BF0DFF8236823F00803236001237C
:10BFF00085F8BD310028C0D032462021FEF7C2F8B6
:10C00000D5F80031002BBBD1D4E7EB696A69D05475
:10C01000EB69EA680133B3FBF2F102FB1133EB6128
:10C0200080E7236823F080032360B8E795F8B20126
:10C030000BF0B8F8D5F820410122236823F008035B
:10C04000236085F8BD210028A6D032462021FEF7C6
:10C0500099F89FE72DE9F04FAF4C83B004EB8004D3
:10C06000D4F82C4C002C6BD0D4F8AC511F46DFF820
:10C07000C4B290466B680646A84AC4F8A0316B6B00
:10C08000DFF8B49263612B6BA160A3616B8FE360F7
:10C090002B8FC4F8A82123610BF6B81323602A78EC
:10C0A00009EB420393F94C0F53000193C3B2012BE8
:10C0B00040F28680D4F8003183B1994900209C4633
:10C0C0004B68013024319C4500F0F6801028F7D1F0
:10C0D000944B93F87810002900F05381D4F8FC00B9
:10C0E000002840F0C2806B68C4F8203195F8280021
:10C0F000002840F0D28094F8B2010BF053F80221EE
:10C100003A07034694F8B09184F8BD111CD558B392
:10C1100017F0510F4FF00B0206F1010614BF0A2170
:10C120001A2117F0410FC671827114BF40232023DA
:10C1300094F8B3211943FEF725F8D4F8FC3043B343
:10C14000204603B0BDE8F08F18F0020F0CD058B1B4
:10C150000B223B06827106F10102C27100F11881C7
:10C1600094F8B321FEF70EF848460BF01BF80028B0
:10C17000E3D018F0010FE0D00C2201360221C67185
:10C18000827194F8B121FDF7FDFFD4F8FC30002B4B
:10C19000D6D195F82C1095F92A0089093CF01AFBA4
:10C1A00095F92A3095F82A20002BC9DB02F01F02EE
:10C1B00001215B095C4801FA02F240F82320BFE745
:10C1C00008234FF00C0A0BF5AA6C1AFB003A002367
:10C1D000E64619460131172962D01EF81C3F042B90
:10C1E000F8D19EF801309342F4D15EF80A30002B6A
:10C1F000F0D08E460199C4F800318944CEEBCE01CF
:10C2000099F94DEF890000EB4009BEF1FF3F01EBCA
:10C2100089015944D1F85C15C4F808113FF44DAFB9
:10C220000021013117293FF447AF1CF81CEFBEF184
:10C23000050FF6D19CF801E09645F2D15CF80AE0D2
:10C24000BEF1000FEDD0C1EBC101C4F8FCE000EB82
:10C250004000890001EB80008344DBF85C15C4F8E2
:10C260000411002B7FF429AF70462D4A002351683A
:10C2700001332432814261D0102BF8D1294B93F83D
:10C280007820002A7FF42FAF2A78013283F87920B2
:10C290000C2283F878206B6826E73CF0CBFA2AE77B
:10C2A000019B9944D4F8003199F94D1F0131B7D160
:10C2B000002B7FF402AF11E75FFA80F9194B0132CE
:10C2C00009F1FF31D2B201EBC10103EB810393F815
:10C2D0009C1000297FF402AF83F89D201348D3F807
:10C2E000802082420CBF952096200B2283F89C2050
:10C2F0003CF0A0FA2346484695F82B200C49FDF760
:10C30000D5FE6B68D4F8FC002833C4F81831002837
:10C310003FF4E9AEA9E700BFC012002035B2000823
:10C32000800001200000012000E100E000600240E8
:10C330008990000828F0040820180120DBB2184A70
:10C34000013B03EBC30302EB83032A7893F89C10B1
:10C350000132D2B200297FF4C6AED3F8800083F850
:10C360009D20104A90420CBF952096200C2283F805
:10C370009C203CF05FFA6B6803F12402C4F81C2196
:10C38000B2E6013283F879200B2283F87820A5E603
:10C390000123204684F8BD31FEF74CFFE4E600BFE0
:10C3A0000000012000600240BFF34F8F0549064B9B
:10C3B000CA6802F4E0621343CB60BFF34F8F00BF43
:10C3C000FDE700BF00ED00E00400FA0508B572B615
:10C3D000FFF7EAFF30B583B0FFF7D2F80320FBF791
:10C3E00047FF01284BD0324C0025324A0523C4F8C0
:10C3F0009850C4F89C50C4F8A020C4F89430BFF3FF
:10C400004F8FBFF36F8F4FF6FF01E2682A4B0A4050
:10C4100013432A4AE360536F37F06AFC284B2949DB
:10C42000A3FB0023D4F8FC209B0C42F08072C4F8DC
:10C43000FC20C1F8F433D1F82C332349234AA1FB63
:10C44000031323499B09C2F8B01F5560013B1168D3
:10C45000B3F1807F41F00101116008D24FF0E0227A
:10C46000F0215361072384F82310956113614FF085
:10C47000E022136943F00403136103B030BD0221CD
:10C480000320FFF777F80D4B12485A6C124942F41B
:10C4900080425A645B6C03F480430193019A026802
:10C4A0000B68026083F308884B689847FEE700BF7B
:10C4B00000ED00E01B0000060005FA050038024010
:10C4C00083DE1B4320180120D34D6210001000E0D2
:10C4D00055CEACC5003801400000F01F800AA0F521
:10C4E000801052281CD80F4B184490F8F4330D2BB1
:10C4F00016D8013910B40C4C04EB831CD4F82C432F
:10C500008BB2DCF840040CF24441CCF84C34B4FB60
:10C51000F2F2013A5DF8044BCCF8442437F0B2BE95
:10C52000704700BF28F004082018012070B50446A9
:10C530000068830AA3F58013522B05D82E4E33448E
:10C5400093F8F4530D2D00D970BDFCF7A1FD2B4BD2
:10C55000A801022203EB8515D5F8401485F87D2447
:10C56000274A8D682A40062A06D0B2F5803F03D0BC
:10C570000A6842F001020A60034401202168214A4E
:10C5800083F87D040023204801E050F833209142D5
:10C590000AD001330E2BF8D1012100203CF01AF90A
:10C5A0001A4B01221A6070BD06EBC303012193F9F7
:10C5B000ED4993F8ED6920463CF00CF9002CC3DB03
:10C5C00006F01F0301216409104D01FA03F31B2E2D
:10C5D00045F8243008D02E2EB6D12C203CF0FAF8A5
:10C5E0004FF480536B6070BD19203CF0F3F84FF0AE
:10C5F00000732B6070BD00BF28F0040820180120D4
:10C60000070001000000014010FA040800E100E00A
:10C6100003689B0AA3F58013522B56D870B53B4C88
:10C62000234493F8F4C3BCF10D0F4DD8407985082D
:10C6300000294ED00CEB8C034FF0020E84083448D6
:10C640000CEB43030EFA04F42B4400EB8C15D5F8E5
:10C65000405400EB830EEE68CEF804103443CEF85D
:10C660001420EC604FEA8C14EFF3118E502383F307
:10C6700012882C2303FB0CF3C258C11832B3131DCC
:10C680004A622C22234D02FB0CF215441432024460
:10C6900052F8041B19B1196052F8043C0433954256
:10C6A000F6D100225FFA8EFE1A608EF311882C23D9
:10C6B00003FB0C0C2044DCF82430D0F8402403B3F6
:10C6C000D36843F00103D36070BD70472433034443
:10C6D000D7E70CEB8C030E482C460CEB43032B44A2
:10C6E00000EB8C15D5F840640225A540F46824EAD7
:10C6F0000504F46000EB8304616062614FEA8C140E
:10C70000B2E7D36823F00103D36070BD28F00408BA
:10C71000201801204418012003689B0AA3F5801308
:10C72000522B00D97047144A134493F8F4330D2B5D
:10C73000F8D810B4114C79B94179022204EB831076
:10C740005DF8044B21FA02F3D0F840149A40CB680C
:10C7500023EA0203CB6070474179022204EB831085
:10C760005DF8044B21FA02F3D0F8401402FA03F307
:10C77000CA681343CB60704728F0040820180120D2
:10C7800003689B0AA3F58013522B10D8084A134460
:10C7900093F8F4230D2A0AD8407902230549D8409A
:10C7A00001EB82128340D2F84024DB4313617047CF
:10C7B00028F004082018012001490248FCF736B986
:10C7C000201801200000014010B5064C0648214603
:10C7D000FCF72CF904F5C6710448BDE81040FCF7DD
:10C7E00025B900BF2018012000000140004401408D
:10C7F00002494FF08040FCF719B900BF4C180120E6
:10C8000001490248FCF712B97818012000040040E1
:10C8100001490248FCF70AB9A418012000080040A9
:10C8200001490248FCF702B9D0180120000C004071
:10C830002DE9F843194E3569F3681D4010D04FF0CB
:10C840000047DFF85C80B5FA85F227FA02F31F2A69
:10C850006FEA030305EA0305336103D0002DF2D12B
:10C86000BDE8F883D8F80431A3B103F1FF39002300
:10C870001FFA89F9C8F80431D8F80041002CEDD02E
:10C8800023682046494698476468002CF8D1002D5B
:10C89000D9D1E5E7F16A1FFA81F9EDE70010004010
:10C8A0002018012001490248FCF7C0B854190120A2
:10C8B0000004014010B5064C064804F59A71FCF7D7
:10C8C000B5F804F504710448BDE81040FCF7AEB8B3
:10C8D0002018012000040140001C004001490248CA
:10C8E000FCF7A4B88019012000400140014902482A
:10C8F000FCF79CB8D81901200048014001490248C2
:10C90000FCF794B8041A0120001800402DE9F0410A
:10C910004FF425728EB00021664842F0B7F9664B9D
:10C92000664E4FF080415A6C06F68805374642F055
:10C930000102DFF89081A6F18C045A645A6C02F06F
:10C9400001020092009A1A6C42F001021A641A6CF9
:10C9500002F001020192019A1A6C42F002021A647A
:10C960001A6C02F002020292029A1A6C42F004025D
:10C970001A641A6C02F004020392039A1A6C42F0D1
:10C9800008021A641A6C02F008020492049A1A6CE3
:10C9900042F010021A641A6C02F010020592059A15
:10C9A0001A6C42F020021A641A6C02F020020692FD
:10C9B000069A5A6C42F002025A645A6C02F0020261
:10C9C0000792079A5A6C42F480325A645A6C02F405
:10C9D00080320892089A5A6C42F400325A645A6CB7
:10C9E00002F400320992099A5A6C42F480225A6485
:10C9F0005A6C02F480220A920A9A1A6C42F040029F
:10CA00001A641A6C02F040020B920B9A1A6C42F0F4
:10CA100080021A641A6C02F080020C920C9A1A6C52
:10CA200042F480721A641B6C03F480730D930D9BA7
:10CA30004246002301E054F8332091420BD00133E9
:10CA40000E2BF8D11C3700203BF0F4FEAF420CD087
:10CA500057F81C1CECE71A4A1C3702EBC30393F887
:10CA6000EC093BF0E7FEAF42F2D14FF08041154FA9
:10CA7000154C3A46002301E054F8332091420BD084
:10CA800001330E2BF8D11C3600203BF0D3FEAE4212
:10CA90000CD056F81C1CECE7094A1C3602EBC30309
:10CAA00093F8EC093BF0C6FEAE42F2D10EB0BDE801
:10CAB000F08100BF20180120003802409CFA0408D1
:10CAC00028F004080000014010FA0408800AA0F5CC
:10CAD000801052280ED8084B184490F8F4230D2AE1
:10CAE00008D8064B03EB8213D3F84024136843F0B5
:10CAF00001031360704700BF28F0040820180120CC
:10CB0000F0B5A24CA5B0E368022B00F03A82A04831
:10CB1000A04AA149121A42F045F8A048A04AA149EA
:10CB2000121A42F03FF8A368012B00F2C28003EB17
:10CB300043039D4A9D4D02EB430032F81320418888
:10CB40008388C5E9BA21C5F8F032994C994E9A4BC1
:10CB5000B2FBF1F2994901FB02F20021C6F82C2345
:10CB6000D4F8882042F47002C4F888201A6842F091
:10CB700001021A609960924A1868024091481A604E
:10CB8000C0F30807904A5A601A6822F480221A609B
:10CB9000D96007B1FEE78D49A0604FF6FF000A6833
:10CBA0008B4B42F400720A60E26802401343E36078
:10CBB0003CF03CF9BFF34F8FBFF36F8FC4F8507256
:10CBC000BFF34F8FBFF36F8F636943F4003363612B
:10CBD000BFF34F8FBFF36F8FC4F88470BFF34F8FD5
:10CBE000D4F8803043F6E07CC3F3C90EC3F34E3370
:10CBF000580100EA0C01734641EA8372013B5F1C55
:10CC0000C4F86022F8D1203810F1200FF1D1BFF321
:10CC10004F8F636943F480336361BFF34F8FBFF37A
:10CC20006F8F6A49644B0A6842F480720A60196C1B
:10CC3000684A41F080511964196C01F080510291E9
:10CC40000299116841F4404111601268D5F8E80278
:10CC500002F44042D5F8EC42D5F8F0120192019A64
:10CC60009A6802F00C02042A00F08D809A6802F0A3
:10CC70000C02082A00F083804F4A136843F4803383
:10CC80001360D6F8647F04E0D6F8643FDB1B642BA6
:10CC900074D813689B03F7D5474A936803F00C03D5
:10CCA000082B6BD0136823F080731360D6F8647F71
:10CCB00008E03E4DD5E9BA2147E7D6F8643FDB1BD3
:10CCC000022B5BD813689B01F7D40B06640843EA78
:10CCD0008013611E43EA01433F491943364B5160BB
:10CCE000116841F080711160D6F8641F04E0D6F835
:10CCF000642F521A022A41D81A689201F7D5196C8A
:10CD0000344A41F0805119641B6C03F08053039343
:10CD1000039B136843F480331360D6F8641F06E066
:10CD2000D6F8643F5B1AB3F57A7F00F2CB80536884
:10CD3000DF03F5D51368274943F400331360D6F8B1
:10CD4000642F06E0D6F8643F9B1AB3F57A7F00F2B1
:10CD5000B9804B689C03F5D54FF400124FF0006387
:10CD600004A804924FF4C07221930723CDE908234D
:10CD700003230A9336F0F0FF80B3FEE7FEE75B681B
:10CD80005A027FF579AF0C4B1B6885E750280040AD
:10CD9000000000008838000028F20508000000208C
:10CDA000C8010020B74C0608080305080000012050
:10CDB00000ED00E0201801200038024040420F0042
:10CDC000FFFFF6FE0000000810300024003C024087
:10CDD0000003FA0500700040080040206C4A136808
:10CDE00003F00F03062B0AD8136823F00F0343F058
:10CDF00007031360136803F00F03072B63D1654B20
:10CE00009A6842F4E0529A609A6842F460429A60EA
:10CE10009A6822F0F0029A601A68900153D59A68D5
:10CE200041F2883122F0030242F002029A60D6F801
:10CE3000640F04E0D6F8642F121A8A4243D89A6825
:10CE400002F00C02082AF5D1514A136819070AD5D5
:10CE5000136823F00F0343F007031360136803F014
:10CE60000F03072B2FD14B4C4B4FA36823F4E053F8
:10CE700043F4A053A360A36823F4604343F4004346
:10CE8000A36036F035FFA368C3F303133B4493F864
:10CE9000F431D840C6F82C033BF0C8FF002304A8A7
:10CEA000CDE91333CDE91533CDE91733CDE9193386
:10CEB000CDE91B33CDE91D33384B049336F04CFFDD
:10CEC00010B1FEE7FEE7FEE702234FF0007204A870
:10CED000CDE90633D823CDE9042301230B9336F0A3
:10CEE0003BFF00B1FEE7D4F88C3023F08073C4F828
:10CEF0008C30D4F88C3043F08073C4F88C30A36845
:10CF000003F00C03042B36D0082B18D0244BC6F8A2
:10CF10002C33204AD5E9BA31B3FBF1F39168D6F846
:10CF20002C23C1F303110F4497F8F411CA401D4993
:10CF300001FB03F3C6F82C23934220D0FEE763687D
:10CF4000626813F4800F636802F03F0218BF16494D
:10CF5000C3F3881308BF1249B1FBF2F202FB03F3DB
:10CF60000C4A5268C2F3014201325200B3FBF2F3A1
:10CF7000C6F82C33CDE70C4BC6F82C33C9E725B0E7
:10CF8000F0BD00210320FEF7F5FAFFF70DFA00BF10
:10CF9000003C02400038024020010508C0FF0300A9
:10CFA0000024F40040420F0000127A000548D0F837
:10CFB000A03223B1DB6A13B100F52870184702488C
:10CFC000704700BF201801202403050810B5174C36
:10CFD000D4F8683F1B883BB9002384F8743F84F879
:10CFE0009832C4F8943210BDD4F86C2F002AF3DDC7
:10CFF000012A08D0D4F8703F59880123A4F8761F7D
:10D0000084F8783FE8E7D4F8701F8A8849880132AD
:10D01000521A9A42F1D10022D4F8A03204F52870B5
:10D020001B69C4F8CC229847D6E700BF201801201E
:10D030000748D0F89C3213B190F8783F0BB100202C
:10D040007047D0F8A03200F528705B68184700BF21
:10D0500020180120174B10B4174C93F89822224443
:10D06000C0E9002493F8980293F8742F824217D8ED
:10D0700093F89802824206D300235DF8044B1846C9
:10D08000C1E90033704793F89832002A5DF8044BE9
:10D09000C3F180030CBF012002204A600B6070477F
:10D0A00093F8984200230120121B5DF8044BC1E95C
:10D0B00000237047201801200C1F00200F4B93F80D
:10D0C000982293F8740F93F89822904293F898223C
:10D0D0000FD8904204D3D3F89432002018447047FC
:10D0E00093F89822D3F89432C2F180021044184485
:10D0F0007047801AD3F894321844704720180120E2
:10D1000010B51B4C84B01B4B94F898220393134426
:10D1100094F8741F029394F89832994294F89832D4
:10D1200014D899420AD294F898320191C3F180033D
:10D130000093C9B901223F2B0ED868B994F8980220
:10D14000401AB0FA80F0400904B010BD0022CB1A9A
:10D15000019201220093EEE76946002302A83FF006
:10D1600029FA94F8741FE9E70B440222E3E700BFB1
:10D17000201801200C1F00202DE9F043164685B031
:10D1800000293CD0451E284CDFF8A4804FF0000950
:10D190006F180DE094F8983208468B4294F8983254
:10D1A0001DD9C3F1800318443F281BD8AF4226D0B5
:10D1B00094F8740F15F8013F411C4044C9B280F83F
:10D1C0004C3C0B0684F8741FE4D5002094F8983288
:10D1D00084F8749F01468B4294F89832E1D8C01AC3
:10D1E0003F28E3D994F898328B42DFD00F4B1B785D
:10D1F000002BDBD00020FFF783FFAF42D8D1694678
:10D2000002A8FFF727FFDDE9003213443F2B00D9C6
:10D2100010B905B0BDE8F0830246334602A83FF0DE
:10D22000C9F905B0BDE8F0832018012000000120F5
:10D23000C012002030B585B0694602A8FFF70AFF8A
:10D2400058B9094C04F52875D4F8A03228465B6813
:10D2500098470028F8D005B030BD0246012302A847
:10D260003FF0A8F9EDE700BF2018012070B5114C80
:10D2700016460A4682B0D4F89C3281190546994276
:10D2800094F8741F88BF1E1A94F89832994203D0FC
:10D290000192FFF7CFFF019A002033462946C4F8D8
:10D2A000CC02D4F8A002846A0348A44602B0BDE8C8
:10D2B0007040604720180120C01A01208C46134698
:10D2C000014662461846D1E738B5244C002204F6E0
:10D2D0007C701346C4F89C2202461178063202295B
:10D2E0002BD00133062BF8D10022D4F8A032C4F899
:10D2F000702FF3B1DA6AE2B119489047D4F8703F61
:10D30000C4F8680FA3B159889A884368521A02FB7F
:10D310000333C4F89C32FBF78BF894F89832054637
:10D3200094F8742F9A4201D0FFF784FFC4F8945206
:10D3300038BD0C4BC4F8683F38BD03EB4303D4F849
:10D34000A02200EB4303C4F8703F12B1D26A002A56
:10D35000D2D1044A1046C4F8682FD4E7201801201F
:10D36000C01A01202403050810B50A4CD4F8A032D5
:10D370005B6A13B104F528709847D4F89432D4F856
:10D38000682F013B5288134452421340C4F8943230
:10D3900010BD00BF201801202DE9F043384E93B096
:10D3A000FFF714FEFFF790FF96F8983296F8742F67
:10D3B0009A4201D0FFF73EFF0025D6F89C72C6F8CE
:10D3C000945297B16C46DFF8BC802A46414620460D
:10D3D000203501F003FE20463FF09CF90122014672
:10D3E0002046FFF7C9FEAF42EFD896F8983296F87C
:10D3F000742F9A4201D0FFF71DFFD6F8683F9B7B40
:10D40000012B36D096F8983296F8742F9A4201D0B4
:10D41000FFF710FF0020C6F894026FB380466C46F9
:10D42000DFF86090054601E0AF421CD92A46494624
:10D4300009A801F0D3FD21220021204641F026FC5D
:10D44000202221462846FFF711FF2022064609A97F
:10D450002046203541F047FD08B9202EE4D0AF42E8
:10D4600008F10108E2D8B8FA88F0400913B0BDE825
:10D47000F083FFF779FFC5E7012013B0BDE8F08323
:10D4800020180120B86A05080A4B93F8F40218B96D
:10D49000094B93F8A00F7047084AD1680329F7D1C8
:10D4A00005494FF0010C81F8A0CF0021D16083F82D
:10D4B000F41270470000012020180120502800407D
:10D4C0000321044608B50846FEF754F872B6104921
:10D4D000D1F8A80FD1F8AC3F50EA03020AD10022DC
:10D4E00011460420FEF746F811460520FEF742F8E3
:10D4F000FEF75AFFD1F8D42221B24EF6602412185A
:10D5000004FB01F143F100038A1843EBE171E8E702
:10D51000201801200021032008B5FEF72BF872B671
:10D52000FEF742FF184CD4F8B02F94F8B60F08B5A8
:10D530004AB11168938809690B40F8B9003B18BFDC
:10D540000123002BF4D114200DF034FB00BFD4F8DC
:10D55000B03F63B1196894F8B62F9B8809690B40F6
:10D5600042B9003B18BF01230BB1FFF7D3FFFAF715
:10D5700091FFEBE7B3FA83F35B09F5E7B3FA83F3C3
:10D580005B09002BD4D1DEE720180120F8B51C2060
:10D5900009F008FE04461121FDF772F97CB3A38857
:10D5A000C82022681B0493610DF004FB2368A28845
:10D5B0001B209A6109F0F6FD08B12923C3802923B5
:10D5C000E380264CD4F8443213B10023C4F844322B
:10D5D0000023234E0125234FC4F8406287F8B83F4B
:10D5E00084F82C523BF03AFD06F11C03C4F8443297
:10D5F0001D4B93F87131AB420CD02846F8BDC820C2
:10D600000DF0D8FA1B2009F0CDFD0028D9D0292330
:10D61000C380D6E7D4F86002543690F8BC33C4F81F
:10D620005C62AB4214D00168D1F8043823F00203E5
:10D63000C1F80438D7F8642FD7F8643F9B1A032B3E
:10D64000FAD98B68002243F001038B6080F8BC2379
:10D650000023064A184682F82330F8BD202801200E
:10D66000F8020120201801201829012000ED00E017
:10D670002DE9F04F00218BB041F69462BD4841F096
:10D6800005FB0420FAF7F4FD01460520FAF7F0FD4A
:10D6900051EA000340F05E81B74B03934C22002116
:10D6A000B448012441F0F2FA00214C22B14841F083
:10D6B000EDFA039BAF4AD3F89C33B04D147115605B
:10D6C0005362C2E907333BF0D1FBFFF7FDFD0021B8
:10D6D000084609F0F5FDFAF7ABFEB0F1000B40F398
:10D6E0000981A44B0024A64D03F14C0AA54B274603
:10D6F000A04605F5BA79A44ECDE9013404E008F559
:10D700000068C34540F3AC80019AD2F8D432C2F825
:10D71000D832FAF7BFFE202249464046FFF7A6FD61
:10D7200012229A49484641F0DEFB0028E7D14745DE
:10D7300021D0029B5A1C03EB4301954B029203EB51
:10D74000810394491846049301F048FC5246049B17
:10D7500042F84C3BDAF81C30CAF80C70A8EB07070B
:10D76000CAE908330123CAF808308B4BCAE90477A9
:10D77000CAF828309246039B47461222D3F89C33BE
:10D78000CAF81C30A918335D013291F8741199421E
:10D790000BD00024202AF5D120374946BB45384616
:10D7A00054DBFFF763FD0022ECE70134152CF1D1C7
:10D7B000D0197A492022FFF759FD00230A2209A92E
:10D7C0007648CDF8249001F0A3FD07460998002380
:10D7D0000A22013009A9099001F09AFD079000235F
:10D7E00009980A2209A90130099001F091FD0690DB
:10D7F000002309980A2209A90130099001F088FD47
:10D80000059009A9099800230A220130099001F026
:10D810007FFD0490002309980A22194601300990DF
:10D8200001F076FD97B1DDE9063243EA4211049B2F
:10D830005A01059B42EAC32242EA6003A7F2BC7286
:10D8400041EA422243EA0243CAF81C30029B642B9D
:10D8500000F0F380474608F50068C3453FF754AF32
:10D86000029A642A00F0E280B84500F0DF800C23C1
:10D87000474DA8EB070602F1010803FB0255454995
:10D880004246454C284601F0A9FB029ADAF81C30C2
:10D89000CAF80050951CCAF80C70CDF80880CAF878
:10D8A0002840CAE908330123CAE90466CAF80830E7
:10D8B0004C22304B00213A4F02FB05F501262B4448
:10D8C000184641F0E3F94C22002141F0DFF9294AE2
:10D8D0005751039A8462029CD2F89C2302348660DA
:10D8E0004262C0E904BBC0E907224FEA4B03B3F12F
:10D8F000805F1EDA4C221F4B00212A4F02FB04F4EA
:10D90000012502262344184641F0C0F94C2200218B
:10D9100041F0BCF9174A03991751CBF10062D1F8D5
:10D920009C13AA40467185604162C0E90711C0E9B5
:10D930000422104B9D6835B91A461B791BB1136838
:10D94000002B40F08380002108460BB0BDE8F04F6B
:10D9500009F0B6BC4FF47A7200233FF09FFB124BE4
:10D9600040F26D11022440F2B2720D46B0FBF3F3A7
:10D9700024E000BF083001200000012074F10508F8
:10D980001829012020180120FC6A0508D86A05081A
:10D99000AC2A0120EC6A0508BDD200088C2A0120BF
:10D9A000146B0508246B05088051010001325B1AD5
:10D9B00012F003040CBF4FF4B77129469942F5DD0C
:10D9C0007449002C3CD003910399D1F86C1399420F
:10D9D0006FDC714D01245B1A55F8041F0134994224
:10D9E000F9DD0133A2F2BC72039D43EA44133C24E7
:10D9F00043EA4223694AB0FBF2F102FB11024FF401
:10DA00006160B2FBF0F100FB11221C20C5F870032D
:10DA1000B2FBF4F004FB1022521042EA401242EA38
:10DA2000C12242EA0343C5F89C3337E6029B012436
:10DA30005D1C002B3FF459AF00E06525584C37E7DB
:10DA40000C4603911D21C4F87013BDE729462E46EC
:10DA50001564D563C2E91155D46C02F14C0354B37B
:10DA60009C68481E1E648442DE63C3E9116612D0BE
:10DA7000481C844216D08C427FF465AF08460028CB
:10DA80003FF461AF116CCC6B0134CC6319649364C7
:10DA900001461A46E0E700293FF455AF884253F8A3
:10DAA0000C2CECD1117900293FF44DAF53641A646A
:10DAB000EEE7012495E73B490222264611E0CB6BB5
:10DAC0000A635B01C1E9046657D003F6FF77531E72
:10DAD00003EB17335A1C0135C1E90D3351F84C0FD4
:10DAE000C8B10B79002BEAD108690A63002848D134
:10DAF000531E10464F694863002F40D007F6FF774A
:10DB000003EB1733201A8B635A1C0135C41851F8E4
:10DB10004C0F0028E5D124483E22013BC0F81843B1
:10DB20003F24C0F800234022990F0190C0F82453ED
:10DB3000C0F81433C0E9C1421C4AC0F8FC229A0064
:10DB40002BB340F2FF10121841F10001520A42EAD1
:10DB5000C15202F140010198124C0A44C0F80C1362
:10DB600002EBC303C0F810235902C0F8F832DA0DF3
:10DB7000C0E9C744C0E9BC12E5E61346AAE713466C
:10DB8000C0E700F6FF70531E03EB1030B2E701222E
:10DB9000DFE700BF000001206C030120805101007D
:10DBA000BDD200080830012020180120306B050884
:10DBB00043F2012243F2010C43F20111002342809F
:10DBC00041F20142A0F800C04FF0010C81804FF6F5
:10DBD0000171C280FF22438180F808C08381C38124
:10DBE00001828274704700BFFF22174B4FF0FF3C49
:10DBF000C270027102724272427382738274C27482
:10DC00000022F0B503F10C076646172516244FF0E5
:10DC1000150E02EB8202BB4200EB020100F802E0AB
:10DC20004C708D70CE7081F804C00BD093F9062033
:10DC3000063393F801E09C78DD7893F9046093F95A
:10DC400005C0E6E7F0BD00BFA80305084FF0000CD3
:10DC500001210222032380F805C08171C271037281
:10DC6000704700BF00230222037043708370C370AB
:10DC7000027170472C22022302704370704700BF6C
:10DC8000012322210022037041708370C27070470B
:10DC90004FF4F07140F22E4C0022072301804FF424
:10DCA0007A71A0F81EC04FF4FA6C41844FF4F5610C
:10DCB0008271A0F820C040F2012C428242F2201270
:10DCC000818442F22451A0F814C040F2034C018137
:10DCD00042F2267142810E22A0F816C040F2056C75
:10DCE0008181012180F8262002228370A0F818C0CB
:10DCF00083764171427400B540F2262EA0F81CE0F4
:10DD00005DF804FB8388C3F30B039342A8BF13465B
:10DD100070B51D460C461A460646806840F042FF24
:10DD20006219084B9442B56908D0074814F8011BE2
:10DD300000FB03F3A24283EA0103F7D101202B6029
:10DD400070BD00BFC59D1C819301000100230370BD
:10DD500043708370C37070470023037043708370F7
:10DD6000C3707047012300224FF0380C39218270B4
:10DD700080F800C04170C270037143718371C37138
:10DD8000704700BFFF232821292201704270837051
:10DD9000C3707047002306214FF47A720170037339
:10DDA000C0E90123704700BF0023FF22411C10B5CA
:10DDB00000F8132001F8132001330B2BF8D10B4B83
:10DDC0004FF0FF31002203F10F048C4605E093F978
:10DDD00004C093F9051013F8032F00EB420E9C4288
:10DDE00000F812C08EF80110F1D110BDBC03050877
:10DDF0004FF0240C00230122022180F800C04FF0D4
:10DE0000250C427080F803C04FF0200C837080F81E
:10DE100006C04FF0210C027180F809C04FF0260CAB
:10DE2000437180F80CC04FF0180C0372C372427338
:10DE3000837302744374FF23C274032280F812C0F8
:10DE40004FF0120CC171817201758275C37580F833
:10DE500018C04276837600B54FF0270E80F80FE0A9
:10DE60004FF0130E80F815E05DF804FB03230370F8
:10DE7000704700BF0A4491421AD001F1FF3C41F2C1
:10DE8000210100B502F1FF3E1CF8012F082380EAB2
:10DE9000022010F4004F4FEA400281EA40000CBF1C
:10DEA00090B280B2013BF4D1E645EDD15DF804FBC0
:10DEB000704700BF704700BF2DE9F047089F002B57
:10DEC0000E4605463C4614BF4FF030094FF020097E
:10DED00014F8011B41B3002A2CDD234600E0B2B147
:10DEE00013F8010B9046013A0028F8D1A8F1020876
:10DEF0006AB1C24649462846B04753460AF1FF3A3E
:10DF0000002BF7DC28EAE8723978013249B1D71BD7
:10DF10002846B047E01914F8011B0029F8D1BDE8E4
:10DF2000F0871046BDE8F087002A02F1FF38E0DCF8
:10DF30000846F4E70022EAE703685A1C02601970F9
:10DF4000704700BF024B186803681B68184700BF82
:10DF50009C4E01200378092B01D0202B05D110F80D
:10DF6000013F202BFBD0092BF9D02D2B63D02B2B7D
:10DF7000B7EE000A08BF01300278A2F13003D9B22F
:10DF8000092961D8F2EE046ADFED4D7A07EE103A06
:10DF900010F8012FB8EEC77AA2F13003D9B2A7EE7C
:10DFA000A67A0929F0EE477AF0D92E2A50D00378C4
:10DFB00003F0DF03452B3BD110B442782D2A73D0F8
:10DFC0002B2A62D0A2F130030130092B63D8002440
:10DFD000002303EB830302EB430310F8012FA2F1AC
:10DFE0003001303B0929F4D9B3F59A7F1A46B7EED0
:10DFF000007A28BF4FF49A72072B09D91346DFED38
:10E00000316A083B27EE267A072BFAD802F007027E
:10E010002AB1F2EE046A013A27EE267AFBD1002CEF
:10E020003BD0C7EE877A5DF8044B20EE270A704795
:10E0300020EE270A704742780130BFEE000AA2F1B5
:10E040003003D9B209299DD92E2ADFED1D7AAED130
:10E0500043780130A3F13002D1B20929A8D8B2EE39
:10E06000047AF0EE475A06EE902A10F8013FB8EE17
:10E07000E66AA3F13002D1B2C6EE076A092927EE9B
:10E08000257A77EEA67AEED992E782780230A2F16D
:10E090003003092B9BD9B7EE007A67EE877A5DF8DB
:10E0A000044B20EE270A704782780230A2F1300339
:10E0B000092B01D801248BE7B7EE007AB1E700BF46
:10E0C0000000000020BCBE4CF8B5164D6B78BE2B8E
:10E0D00025D1AC1C144F022229464FF6FF70FFF7E2
:10E0E000C9FE22884AB1A618BE4218D2052A16D9FE
:10E0F00021463446FFF7BEFEF3E721460222FFF732
:10E10000B9FE0222A1180634FFF7B4FE074B641BC8
:10E110009C8041F60F53C31A58425841F8BD002065
:10E12000FCE700BF00400008008000089C4E012072
:10E13000F0B5067906F0E003402B03D145794FF0A6
:10E14000FF3406E0602B4FF00105F8D1447905FA61
:10E1500004F40023012006F00706AB4200D1F0BD15
:10E16000052E0FD8DFE806F00308101D242448B15F
:10E17000C85CD75C78400FE020B1C856D756C71BA3
:10E18000784278410133E8E70028FBD031F81300EA
:10E1900032F81370784080B220420CBF012000207A
:10E1A000F0E70028EED031F9130032F91370E6E7FA
:10E1B0000028E7D051F8230052F82370DAE70379FA
:10E1C00003F01803102B1DD004D82BB1082B06D058
:10E1D00000207047182BFBD1B0F80B007047114B93
:10E1E000B0F80B0093F90030591C09D10E4B1B7A83
:10E1F00003EB830203EBC20300EB830080B27047A2
:10E20000DBB2F5E7074BB0F80B0093F901305A1C6D
:10E2100006D1054B5B7AC3EB031300EB4300EDE73C
:10E22000DBB2F8E7A00301209C4E0120114A002335
:10E230004FF0280C0360838030B54FF448744FF0E2
:10E24000290E02F10C0503EB4303AA4200EB430144
:10E2500000F813C081F801E0D3788C808B7008D06F
:10E2600092F90630063292F801C092F802E09488E2
:10E27000E9E730BDD0030508013900224B000260F8
:10E2800001F0030103F00802C1EB01119300C1EB9F
:10E290000111A3EB92038900C3EB031381809B0060
:10E2A0004380704786B04FF4E16200234FF4007C56
:10E2B000ADF80C2041F6037203994280ADF81410BA
:10E2C000BDF814200293828140F20122ADF814308F
:10E2D000A0F800C040F2333CBDF814108360C0F8D1
:10E2E00016304FF49A73C28144F20322A0F806C09C
:10E2F00041830282838206B0704700BF144B15220F
:10E30000144910B5044618681B79206204F12500F1
:10E3100084F8243040F0FBFD0F4B4FF0010E1A7EC5
:10E3200084F83AE012B984F83B2010BD03F11C0CCC
:10E33000BCE80F0020606160A260E360BCE80F00F1
:10E3400084F83BE020616161A261E36110BD00BF20
:10E350005C6B0508646B05089C4E01202DE9F843B1
:10E3600038220021064640F091FC01230222174C7E
:10E370004525B373412186F8213041F61E63DFF84D
:10E380006090671EF384124B09F108083272B36281
:10E39000104B114A336103F1C87303F2B633736152
:10E3A0000E4BC6E90623484640F077FD631E29461A
:10E3B00028B1DA1B4045A0EB090338BFF25415B170
:10E3C00014F8015FEFE7BDE8F88300BF716B050843
:10E3D0001E7D01016400DC050019750343080E0071
:10E3E00048AB0508202108B540F057FD034618B199
:10E3F0001A780130202AF9D0184608BDB5EEC00AB7
:10E40000DFED357A0023F1EE10FA70B5C8BF30EEBB
:10E41000270A86B0D8BF30EE670ADFED307A0546AE
:10E4200003A902936E4620EE270ACDE90033FDEEE4
:10E43000C07A17EE904A84EAE470A0EBE47038F0FA
:10E44000E3FB002C03A8ACBF20232D238DF8003064
:10E450003EF060F9012829D0022833D003281DD0CE
:10E4600003A9304640F00AFD30463EF053F9044619
:10E4700031462846033CE4B2224640F093FB002399
:10E4800028462B553EF046F92E22431C31192A54BA
:10E49000E81840F00FFD284606B070BD302303A9F0
:10E4A00030468DF8013040F0E9FCDDE7302303A968
:10E4B00030468DF801308DF802308DF8033040F091
:10E4C000DDFCD1E7302303A930468DF801308DF80B
:10E4D000023040F0D3FCC7E76F12033A00007A44E1
:10E4E00008F0EEB813B568B14C1E14F8011F21B93D
:10E4F00002B0BDE8104008F0F7B8019008F0E0F86D
:10E500000198F2E702B010BD10B50C4628B1C9431E
:10E51000013801F0010108F04DFFE30701D4FDF7D8
:10E5200055FF10BD2DE9F3410023124D044600EBC9
:10E530008106114F05F83C3FB44203D10F4802B0A9
:10E54000BDE8F081394628464FF0000840F096FCBF
:10E550002146684640F0AEFC2021684640F09DFC14
:10E5600028B969462846043440F088FCE4E780F87E
:10E570000080F1E79C4E01202BAC0508D84E01200D
:10E58000014B186E2AF0EEBB9C4E01202DE9FF478F
:10E590001E46C368044689469246BDF83070DDF8D1
:10E5A00034804BB3CBB20D2B24D81A4AD556BAF1CE
:10E5B000FF3F23D023683146174A3846CDE9005A39
:10E5C000C04752465FFA89F12079FBF705FC024605
:10E5D00000B10288D3B2314638460393C2F3032315
:10E5E000120B02932368CDE900520C4AC04704B0D5
:10E5F000BDE8F0870025DAE74D1CD8E77B06F6D4A6
:10E6000023683146064A3846C4460C9504B0BDE836
:10E61000F0476047386B05085DAB05086AAB050835
:10E620008EAB05082DE9F041154686B0884619469F
:10E630006A1CBDF830600D9F23D0030900F00F0461
:10E64000174A30464033CDE900450593B847A8B195
:10E650002A4698F80510D8F80000FBF705FC68B1C9
:10E66000028801783046059B0391C2F30321120B07
:10E6700002910021CDE900420A4AB84706B0BDE840
:10E68000F0817306FAD4030900F00F00064ABC4675
:10E690000C904033304606B0BDE8F041604700BF03
:10E6A0009DAB0508AFAB0508D8AB0508084B024683
:10E6B00008498B420AD2184602E01C30884205D233
:10E6C0000388C3F30B039A42F7D1704700207047C9
:10E6D000B82A0608B432060870B50546B0F8090035
:10E6E000FFF7E4FF064B0446284693F86460FFF703
:10E6F00066FD16B1E368184470BDA368FBE700BF70
:10E700009C4E012038B505460C46FFF7E5FF2B79F6
:10E7100003F0E00203F00703602A2AD1052B0CD88E
:10E72000DFE803F0030B0F0B1B1B6A7901239340F7
:10E730000278DBB214B11343037038BD22EA03033D
:10E74000FAE76A790123934002889BB214B113431C
:10E750000380F2E722EA0303FAE701236A7903FA66
:10E7600002F2036814B113430360E6E723EA0203ED
:10E77000FAE7052BE1D8DFE803F0030305050707F7
:10E780000470DAE70480D8E70460D6E770B58588BE
:10E790000B4604460021C5F30B0518462A4640F0F7
:10E7A00075FA6169084A0346914202D3074A9142C9
:10E7B00005D319B11846BDE87040084770BD2A4618
:10E7C000BDE8704040F0EEB9B43206089B3406084C
:10E7D00038B5064C064DAC4206D2A16820461C3422
:10E7E000FFF7D4FFAC42F8D338BD00BFB82A060803
:10E7F000B43206089FED067AF7EE007A60EE870ADB
:10E8000020EE800A70EE277A80EE270A704700BF5C
:10E81000DB0FC940B0EEC07AF0EEE06A86FE876A90
:10E82000B5EE406AF1EE10FA3DD0C6FEC75AC5EE0D
:10E83000867ADFED1E2ADFED1E3ADFED1E4A9FEDE0
:10E840001E5A9FED1E3AB7EE006A9FED1D4ADFED9E
:10E850001D5AE7EEE23AA7EE834AE7EEA34AA7EE97
:10E86000846AA7EEA45AE7EE855AC5EE867AF4EEDE
:10E87000C76AF1EE10FA03D59FED137A77EE677A47
:10E88000F5EEC00AF1EE10FA03D59FED107A77EE9F
:10E89000677AB5EEC00AF1EE10FA48BFF1EE677A7A
:10E8A000B0EE670A7047DFED077AE0E739094E3DC1
:10E8B000E3B59E3E88FA163E45FE7F3F99FB243F16
:10E8C00069A2163EA7DFA834DB0FC93FDB0F494022
:10E8D00091ED056AD0ED017AD1ED036A91ED047AEC
:10E8E00067EEA66AD0ED005A27EE877AD1ED014A8D
:10E8F00067EE867A91ED025A91ED004AA4EEA57A70
:10E9000090ED026AE5EE257AD1ED064AE4EE256A3D
:10E9100091ED075AD1ED085AA5EE067AE5EE867A12
:10E92000E4EE866A80ED017AC0ED027AC0ED006AFD
:10E93000704700BFDFED277AB4EEE70AF1EE10FA78
:10E940000CDDDFED256A9FED257AF0EE407A30EEA2
:10E95000660AF4EEC77AF1EE10FAF6DCDFED207A03
:10E96000B4EEE70AF1EE10FA0CD5DFED1B6A9FED6D
:10E970001D7AF0EE407A30EE260AF4EEC77AF1EE18
:10E9800010FAF6D4DFED187AB4EEE70AF1EE10FAD9
:10E9900014DDDFED107A37EEC00A60EE006A9FEDFD
:10E9A000136A9FED137ADFED137AA6EE867A20EED6
:10E9B000266AE6EE877AA6EE270A7047DFED0E7A22
:10E9C000B4EEE70AF1EE10FAE7D5DFED057A37EE9F
:10E9D000C00AE2E7DB0F4940DB0FC940E4CB164138
:10E9E000DB0F49C0E4CB16C1DB0FC93F92E741B949
:10E9F0009730083C15A82ABEDB0FC9BFFDEEC07AD0
:10EA000017EE903A2033402B00D893E79FED010A90
:10EA1000704700BF00000000D0ED005A9FED2B4A68
:10EA200008B535EE840AFFF7E9FFB0EE405AB0EEC4
:10EA3000650AFFF7E3FFD0ED014AF0EE405A34EEED
:10EA4000840AFFF7DBFFF0EE403AB0EE640AFFF70E
:10EA5000D5FF90ED023AF0EE404A33EE040AFFF79C
:10EA6000CDFFB0EE404AB0EE430AFFF7C7FF25EEF8
:10EA7000236A65EE046AC1ED024A25EE847A25EE2A
:10EA8000005A81ED086A23EE844A23EEE53AB0EE9F
:10EA9000666A65EE805A81ED004AB0EE454A81ED26
:10EAA000053A60EE637AA4EEE56AA4EE874AE4EEE6
:10EAB000E65AC1ED017AA4EE857A81ED046A81ED12
:10EAC000034AC1ED065A81ED077A08BDDB0FC93F45
:10EAD000B7EE001A0022DFED050A10B540F060FA2B
:10EAE0000023836143610362C36110BDF304353FBA
:10EAF0002DE9F04F1F461346894689B013F8011BD4
:10EB0000002900F02B8215468046002609E0404689
:10EB100001361D46C8472B4613F8011B002900F09B
:10EB20008C802529F3D16978302900F0DD80023509
:10EB30000023A1F1300C5FFA8CF2092A4FF0000299
:10EB40005ED96C297DD07829E5D8572967D9A1F1FC
:10EB500058002028DFD801A454F820F0DDED00088B
:10EB600017EB000817EB000817EB000817EB00087D
:10EB700017EB000817EB000817EB000817EB00086D
:10EB800017EB000817EB00081BED000829ED000843
:10EB900017EB000817EB000817EB000817EB00084D
:10EBA00017EB000817EB000817EB000817EB00083D
:10EBB00017EB000813ED000817EB000817EB00082F
:10EBC00017EB000817EB0008FFEC000817EB000834
:10EBD00083ED000817EB000817EB0008DDED0008D7
:10EBE000BEF1050F18D9BAF1050FAAD80A2CA8D181
:10EBF00002EB820215F8011B04EB4202A1F1300C7A
:10EC00005FFA8CF0A1F1610EA1F1410AA1F1370484
:10EC10000928E5D86446EBE7A1F15704E6E761B1BE
:10EC200025297FF478AF25214046C8472B46013679
:10EC300013F8011B00297FF474AF304609B0BDE81A
:10EC4000F08F15F801CBBCF1780F3FF664AFBCF143
:10EC5000570F4DD9ACF1580120293FF65CAF01A008
:10EC600050F821F03FEE000817EB000817EB000802
:10EC700017EB000817EB000817EB000817EB00086C
:10EC800017EB000817EB000817EB000817EB00085C
:10EC90001BED0008F1EE000817EB000817EB000869
:10ECA00017EB000817EB000817EB000817EB00083C
:10ECB00017EB000817EB000817EB000813ED00082E
:10ECC00017EB000817EB000817EB000817EB00081C
:10ECD000FFEC000817EB00089FEE000817EB000898
:10ECE00017EB00083FEE0008A9780123033520E761
:10ECF000BCF1000FA1D0BCF1250F94D00BE757F861
:10ED0000040B0023494600904046FFF7D5F806441F
:10ED100001E757F8043B1E60FDE657F8041B404628
:10ED20000136C9B2C847F6E6D7F800C0BCF1000FFB
:10ED3000C0F2AC8005ACA246BCF1090FE6464FF02C
:10ED4000010108DD01EB81014900BCFBF1F009285C
:10ED5000F8D800293DD08948BEFBF1FBBBF10A0F72
:10ED6000A0FB01C001FB1BEE34BF4FF0300C4FF095
:10ED7000570CC0080929DC4401460AF801CBEAD83F
:10ED800027E038680121092809D901EB81014900F0
:10ED9000B0FBF1F4092CF8D8002900F0E68005ACAE
:10EDA0000393A246754BB0FBF1FBBBF10A0FA3FB2B
:10EDB000013C01FB1B00B4BF4FF0300E4FF0570E6B
:10EDC0004FEADC0C0929DE4461460AF801EBE9D878
:10EDD000039B043700218AF8001029E057F804ABA0
:10EDE0000120BAF10F0F40F2C6800001BAFBF0FC1F
:10EDF000BCF10F0FF9D8002800F0BA8005ACA3468B
:10EE000001E0BAFBF0FCBCF1090F4FF0300E05DD5C
:10EE100058290CBF4FF0370E4FF0570EE64400FB59
:10EE20001CAA00090BF801EBEBD100218BF80010B4
:10EE3000494640460094FFF73FF806446BE657F812
:10EE400004BB0121BBF10F0F40F28D800901BBFB18
:10EE5000F1F00F28FAD8002900F0828005ACA24614
:10EE600001E0BBFBF1F009284FF0300E06DDBCF1EC
:10EE7000580F0CBF4FF0370E4FF0570E864401FB72
:10EE800010BB09090AF801EBEBD1A3E72D21CCF166
:10EE9000000C0DF1150A05AC8DF814104CE757F86D
:10EEA000040B0121092808D901EB81014900B0FBBD
:10EEB000F1F4092CF8D8002952D005AC0393A246EE
:10EEC0002E4BB0FBF1FBBBF10A0FA3FB013C01FB96
:10EED0001B00B4BF4FF0300E4FF0570E4FEADC0C62
:10EEE0000929DE4461460AF801EBE9D8039B71E782
:10EEF00057F8040B002829DB05ACA24609284FF07F
:10EF000001010AD901EB81014900B0FBF1FCBCF120
:10EF1000090FF7D800293FF45DAF0393174BB0FBFF
:10EF2000F1FBBBF10A0FA3FB013C01FB1B0034BF4B
:10EF30004FF0300E4FF0570E4FEADC0C0929DE443B
:10EF400061460AF801EBE9D8039B43E72D214042D3
:10EF50000DF1150A05AC8DF81410CFE70E466CE6DE
:10EF600005ACA24636E7584678E705ACA24630E73E
:10EF700005ACA34659E7D44640E700BFCDCCCCCC86
:10EF800073B5114C06460D460192A06EA0B10F4913
:10EF9000FFF7A8FA3146A06EFFF7A4FA0C49A06E5D
:10EFA000FFF7A0FA0B49019B2A46A06EFFF7A0FDD0
:10EFB0000949A06EFFF796FA94F86C3013B101235B
:10EFC00084F86D3002B070BD9C4E0120ECAB05089A
:10EFD000EAAF0508E1E40008F9AB05080EB400B596
:10EFE00084B0084905AB019001A853F8042B0393A2
:10EFF000FFF77EFD019B00221A7004B05DF804EB60
:10F0000003B0704739DF000800232DE9F0411C46AA
:10F0100082B00746038021460134384627F0B0F815
:10F02000082CF8D1002307F1FC06DFF8608087F890
:10F03000EA301D46C7F8EC30C7F8F030C7F8F430B6
:10F04000C7F8F8301F462A46414601A83446FFF764
:10F05000C5FF032201A911F8013B5BB1013A04F895
:10F06000013BF8D1013504362770082DEBD102B0F1
:10F07000BDE8F08101352046202114443FF006FE12
:10F08000082D06F104062770DDD1F0E77C6B05083A
:10F09000F7B5114E074600230C46304615460F497A
:10F0A0006E3600F86E3F04EB45050D4B002F08BF90
:10F0B00019460C4F3FF0E2FEAC4202D10A4803B0C1
:10F0C000F0BD394634F8022B6846FFF787FF6946E2
:10F0D00030463FF0D3FEEFE79C4E0120FDAB050824
:10F0E00006AC05080FAC05080A4F0120F7B5002350
:10F0F0000B4E044600EB41050A4F06F89F3FAC4219
:10F1000002D1094803B0F0BD394634F8022B6846F5
:10F11000FFF764FF694630463FF0B0FEEFE700BFFF
:10F120009C4E01209DAC05083B4F0120F8B54E1EBA
:10F13000054601F11F04054F16F8012F28463946F0
:10F140000235FFF74BFFA642F6D1F8BD14AC050817
:10F1500002460846531C05D1034B1A681B790A6006
:10F160000B717047014939E798AB05089EAC05085B
:10F1700003685A1C02601970090A03685A1C02606D
:10F180001970704702681146531C0360D31C11F8B4
:10F1900002CB01605178036093781B0443EA01239A
:10F1A000111D43EA0C030160D07843EA0060704708
:10F1B000A0F13003092B07D920F02000413819288D
:10F1C0008CBF00200120704701207047303809288B
:10F1D0008CBF002001207047413819288CBF0020C7
:10F1E00001207047613819288CBF0020012070472A
:10F1F00020280BD0092809D00A2807D00D2805D0CF
:10F200000B3801288CBF0020012070470120704777
:10F21000A0F14103192B98BF20307047A0F1610382
:10F22000192B98BF2038704710B56FF00044024684
:10F23000044404E0B3EB0E0015D1A24214D012F83E
:10F24000013BA3F14100192811F8010BA0F1410C79
:10F2500098BF203300F1200EBCF1190FEAD91B1A18
:10F2600004D10028E9D110BD002010BD184610BD02
:10F2700002B3844610B5841804E0B3EB0E0014D139
:10F28000A44513D01CF8013B11F8010BA3F1410276
:10F2900000F1200E192AA0F1410298BF2033192A4B
:10F2A000EBD91B1A04D10028EAD110BD002010BDF3
:10F2B000184610BD1046704770B5044608460D4606
:10F2C0003DF028FA064602E014F8013F43B120461B
:10F2D00032462946FFF7CCFF0028F5D1204670BD05
:10F2E0001C46204670BD38B507490546FFF7E4FFC8
:10F2F000041E0649284618BF0124FFF7DDFF08B1A8
:10F3000044F00204204638BD19AC0508F1C20508D6
:10F310002DE9F041064686469EF800C070460EF183
:10F32000010EBCF1200FF7D0BCF1090FF4D0BCF1F5
:10F330000A0FACF10B05EFD0ACF10D04B4FA84F474
:10F340006409002CE8D1012DE6D9BCF12B0F3DD08A
:10F35000BCF12D0F39D0102A86463DD04FF0FF3535
:10F360009046B5FBF2F502FB05F7FF43FFB20EF145
:10F37000010E002010E0ACF1300C5FFA8CFC9445DB
:10F3800012DA8542764602D334D1674532D21C4028
:10F390004FF0FF301EF801CBBCF1390FEBD94CF028
:10F3A000200CBCF1600F0BD801B10E602CB3B0F192
:10F3B000004F2BD9DB0729D54FF00040BDE8F08185
:10F3C000ACF1570C5FFA8CFCD9E70124102A00F14C
:10F3D000010E90F801C0C1D1BCF1300F19D04FF02F
:10F3E000FF354FF01008B5FBF2F502FB05F7FF43C0
:10F3F000FFB2BCE708FB00C0CCE70028DEDA13F060
:10F40000010F18BF6FF00040BDE8F0814042BDE839
:10F41000F0819EF801C00EF10106ACF14105604695
:10F42000192D01D80CF1200078280BD04FF0FF35B2
:10F430004FF01008B646B5FBF2F502FB05F7FF43A7
:10F44000FFB294E710229EF802C06FF070450EF1F3
:10F45000020E0F2790468AE701230A22002157E770
:10F4600070B50D461446FEF7BDFF0646A0B1FFF786
:10F47000F3FF40F634039842A8BF1846B0F5617F09
:10F48000B8BF4FF46170A0F561731920B3FBF0F3BE
:10F490002B702378013323703046FEF7A3FF064616
:10F4A000A0B1FFF7D9FF40F634039842A8BF184631
:10F4B000B0F5617FB8BF4FF46170A0F5617319209A
:10F4C000B3FBF0F36B70237801332370304670BDCB
:10F4D0002DE9F04117461E4605464FF47A72002387
:10F4E00038463146454C3DF0D9FD4549454A014431
:10F4F000454882FB01C34FEAE17C0B44CCEB63132C
:10F5000082FB03C24FEAE37C1A44CCEB621284FB19
:10F5100002C44FEAE27CCCEBA40C80FB0C404FEA27
:10F52000EC74C4EBE010C3EB0314A1EB8401A971EC
:10F53000C2EB0211A3EB81036B710CEB4C03A2EB4A
:10F54000C30240F2B55303FB10CC80002A71BCF516
:10F55000896F44DA40F2DA239C4547DCBCF5B77F7B
:10F560002A4BB4BF0022012202EB42014FEA4208BB
:10F5700003EBC10391B2B3F8523008EB020E244CF6
:10F5800004EBCE044FF00B0E163401E034F8023DCC
:10F5900063451FDDBEF1010EF8D11C4B42444FF014
:10F5A000010E03EBC202938F00F5FA600CF1010C1F
:10F5B0004FF47A7285F802E00844ACEB030C314654
:10F5C00000232880384685F803C03DF067FD2A8176
:10F5D000BDE8F0810EF1010E5FFA8EFEE4E7032133
:10F5E00040F296534FF006080A46C6E7022140F261
:10F5F00029434FF004080A46BFE700BFABAAAA2A76
:10F6000080BC92C78988888873B06D16A8030508E6
:10F61000E403050808B50D4BD3E9002352EA030CB7
:10F620000AD10146002340F2011218460B804A809D
:10F630008B808B710B8108BD054909688A1843F1DD
:10F640000003FFF745FF012008BD00BFC8270120C8
:10F65000F41A012090420B462DE9F041B0FBF2F67E
:10F660000446154608D2124A05FB16441846135D97
:10F6700000F8013BBDE8F0819642B6FBF2F706D2F6
:10F680000B4A05FB1767D15D03F8011BECE7BA4293
:10F69000B7FBF2F807D905FB1878054A12F80810ED
:10F6A00003F8011BEDE74046FFF7D4FF0346F2E7FE
:10F6B000846B050830B5684C83B0B4F8D433B3F527
:10F6C0007A7F03D94FF47A73A4F8D433B4F8D633DD
:10F6D000B3F57A7F03D94FF47A73A4F8D633B4F82C
:10F6E000D803B0F57A7F04D94FF47A731846A4F89A
:10F6F000D833B4F8DA13B1F57A7F03D90023194669
:10F70000A4F8DA33B4F8DC23B2F57A7F04D94FF4E5
:10F710007A731A46A4F8DC33B4F8DE33B3F57A7F93
:10F7200002D90023A4F8DE33884202D80021A4F8CD
:10F73000D813934202D30023A4F8DC33B4F8EA23AD
:10F74000B4F8EC339A4202D90023A4F8EA33434BCD
:10F750001B8803B3424DAA78062A43D8414901EBDE
:10F76000820191ED270A2979002940D194F8F413F8
:10F7700007EE903AAB7907EE101AF8EEE77AF8EE5A
:10F78000C76A86EEA77A0BB130EE000AB4EEC70A5C
:10F79000F1EE10FA30DC637A032B14D8C3EB0313B9
:10F7A000314A02EB4302237A032BC4F8FC2312D81C
:10F7B00003EB83012D4A03EBC10302EB8303C4F87F
:10F7C000003403B030BD0023274A6372237AC4F8A3
:10F7D000FC23032BECD90022244B2272C4F8003402
:10F7E00003B030BD29799FED220A0029BED0042A3A
:10F7F00021D8002ACFD021E067EE807ABCEEE77AEC
:10F800008DED017A9DF8042007EE102AB8EEC77A34
:10F81000F4EEC77AF1EE10FA01DD0132D2B2CAB1CC
:10F82000102AA8BF1022D2B28A42134638BF0B4614
:10F8300084F8F433AFE7053A032AACD9F7EE007A3F
:10F8400087EE800A3EF036FC2B88984228BF184687
:10F850002880A0E70122E6E79C4E01208C1F0020B3
:10F86000D8230120A8030508644F0120DC4F0120A4
:10F870006F1203382DE9F04FAD4E85B096F8043481
:10F8800000AFA3F11702022A00F2C582A94BBB60A8
:10F89000DFF8C4A20024A84DDFF8C0C20AF16C0949
:10F8A00050463BE012F0010154D1BEF1140F00F0BC
:10F8B000AE8253084FEA920B03F0773E4FEAD2082C
:10F8C0000BF0333B08F011380EEB0B03D31AA3EB0C
:10F8D000080303EB131303F00F33A5FB038E4FEA6A
:10F8E000DE1ECEEB0E2EA3EB0E0E930303D5BEF160
:10F8F000010F00F08C82BEF1010F0CD95FFA8EFE71
:10F90000BEF1030F00F28382002900F0808212EA28
:10F910000C0F00F07C820C3048451ED090F904E0BA
:10F920000268AEF11E03DBB2012BBBD8817922F055
:10F930004102C37902290260A8BF0221022BA8BF9D
:10F94000022381710021C371037A022BA8BF022315
:10F950000372AEE70134E4B2ABE7013C022C00F2E3
:10F9600056820024022086F87C4412F0A3FA96F80E
:10F970008034022B00F0EA82002800F054836F4BA1
:10F980004FF47A7E96F84D854FF0000C03F5247BFA
:10F990005A88B2F57A7FB3F8462088BFA3F802E010
:10F9A000B2F57A7F9A8888BFA3F846E0B2F57A7FED
:10F9B000DA8888BFA3F804E0B2F57A7F02D9002282
:10F9C000A3F806C099889142B3F85A10B3F85C20A6
:10F9D00098BFA3F804C0914293F86B2002F1FF3264
:10F9E00088BFA3F85AC0632A03D94FF0640283F892
:10F9F0006B2093F86C2003F1660019460132D2B2F5
:10FA0000092A4FF0000288BF83F86CC08D7A01325A
:10FA100010F8014B0631A54238BF00F801CC032A8B
:10FA2000F4D1B8F1010F03F1A40318BF03F81FCC00
:10FA30009B45ADD1424B9B78042B00F0D1822BB972
:10FA40003F4A1388B3F5F07F00F2F781FFF732FEEB
:10FA500096F86715092903D011B13A48FEF70CFC56
:10FA600096F87515092903D011B13748FEF704FC43
:10FA7000B6F88225B6F880351343B6F884251343CB
:10FA80001BB213B10123A6F88635D6F83C352F4AB0
:10FA90001A40002A00F0D682DA0700F149825D049C
:10FAA00040F1CF812A49D6F840250B400A40C6F8DC
:10FAB0003C35C6F8402513F4004200F007820022CE
:10FAC00086F89B2586F8AB25D90440F1098296F883
:10FAD000CB35022B02D1012386F8CB35DFF874B089
:10FAE0005B460BF1780402E006339C420CD01A7896
:10FAF000072AF9D19978DA78914202D35A79002A03
:10FB0000F2D0072019F0FCFE00234FF4806086F845
:10FB10007C3412F0CFF9002800F078820D4DA84611
:10FB200098F8051039B398F8000010B35B461AE056
:10FB30009C4E0120A803050881808080DC4F0120B5
:10FB4000D82301200454012012540120096000022E
:10FB5000F6DFFFFD6C540120A85201208000020056
:10FB600006339C4207D01A788A42F9D15A79002A82
:10FB7000F6D019F0C5FE08F106084445D0D1BC4BBB
:10FB800093F802B0BBF1080F00F0FE8196F84D35F6
:10FB900096F8D123A3F10103032AB3FA83F34FEAC2
:10FBA000531386F8483696F84E35A3F10103B3FA9D
:10FBB00083F34FEA531386F84C36D6F84035C3F337
:10FBC000C03186F84A1602D9002286F8D123A94A04
:10FBD00003EA0201D6F83C351340B27DC6F8401561
:10FBE000C6F83C35002A00F0DB81B6F86036002B01
:10FBF00040F0E381D6F8643613F07F4F02D0002343
:10FC0000C6F86436D6F86C369B4A1A401AB140F2F0
:10FC10000223C6F86C3696F86836013B042B02D9ED
:10FC2000012386F86836ABF1050B944BBBF1030F4B
:10FC300093F890B540F26781BBF1000F20D000230C
:10FC4000FB608B4B6FF007017C60C91A03F1080859
:10FC50000C4604E004EB08035B4580F0F68018F8DE
:10FC6000010B0028F6D00BF0A5FD0028F2D0837917
:10FC70009B07EFD5FB6801227C68002B40F0EB80EE
:10FC80007B4B9B7913B10023794A9371B6F8763692
:10FC900013F00C0F03D1C3F30313022B03D94FF45A
:10FCA0002063A6F87636B6F8783613F00C0F03D139
:10FCB000C3F30313022B03D940F60123A6F87836C9
:10FCC00096F8E52696F8F1369A4200F2268196F8E3
:10FCD000E43696F8F0269A4204D2002386F8E436F9
:10FCE000A6F8E83696F8E62696F8DA379A4202D968
:10FCF000002386F8E6366249FC6001F1780BBC68A7
:10FD000011F8013C4FF0030803EB4303234493F83D
:10FD100098E193F899C193F89A010B461A787245C5
:10FD2000A8BF724603F8012B5A796245A8BF624604
:10FD30005A719A788242A8BF0246B8F101089A70B7
:10FD4000ECD11E318B45DBD1D6F8BC25FC68002AEE
:10FD500000F03D810020012102E00635AC420ED0CA
:10FD60002B78282BF9D16B78043301FA03F3134273
:10FD7000F3D0063522EA03020120AC42F0D108B1EB
:10FD8000C6F8BC253F4D05F108042B4613F8012B9E
:10FD9000072A00F285809C42F8D1EB4688B0FF210B
:10FDA00020226B4618463EF071FF3649034611F893
:10FDB000012B53F82200013079D18C4243F82220E4
:10FDC000F5D1B6F84625DD46B6F844359A4202D359
:10FDD0002D4BC6F84435FF232C4986F80C389AF988
:10FDE0000430142B05D0DAF8002031EA020200F0CA
:10FDF000F4800AF10C0ACA45F1D1254B5A79022A3E
:10FE000001D100225A711437BD46BDE8F08F214858
:10FE10000CF018FFA5E5204A02EBC303BA6093F883
:10FE2000B820002A3FF434ADD3F8BC30002B7FF467
:10FE30002FAD172386F804342AE54FF4F0731380AE
:10FE400004E61C077DD515492DE6FB6800227C6879
:10FE5000002B3FF415AF06494B7C002B7FF416AF07
:10FE60004B79012B3FF40CAF002A7FF409AF0DE76B
:10FE7000D8230120DED9CDFDFDFDFFFF8C1F002022
:10FE8000674F0120EB230120AE014A01010002006F
:10FE9000842A0120A8520120A8030508FE9FFFFD27
:10FEA000EB4688B02022FF2168463EF0EFFE05F8C1
:10FEB000018B08F10108B8F1080F82D005F8018B19
:10FEC00008F10108B8F1080FF1D17AE796F89B150F
:10FED00000293FF4F9ADD90486F8AB253FF5F7AD1D
:10FEE0001A067FF5F4AD96F80434182B06D80122D3
:10FEF0009A405A4B1340002B7FF4E9ADDFF870B104
:10FF00000BF1780400E60023554A1371BBF1000F92
:10FF100000F096800123FB6093E6002296F8E43619
:10FF200086F8E526002B3FF4DDAEA6F8E826D0E6FD
:10FF30004C49D6F840250B400A40C6F83C35C6F877
:10FF4000402598047FF5B7AD4749ACE500283FF45C
:10FF500016AD464B4FF0FF0C90F9045096F8CD14B7
:10FF600003F16C0093F90820AA4204D1013901245D
:10FF700083F808C0C9B20C339842F3D1002C3FF487
:10FF8000FEAC86F8CD14FAE41A469B79002B3FF4B8
:10FF9000FDAD537C012B7FF4F9AD02235374F5E5DD
:10FFA00043F4A02341F4A021C6F83C35B6F86036EE
:10FFB000C6F84015002B3FF41DAE96F85C060BF01A
:10FFC000F9FB00287FF416AEA6F8600612E628209A
:10FFD00019F096FCD6F8BC25BCE686F80C380CE780
:10FFE000D6F83C351E4A23F48053C6F83C35D6F883
:10FFF000403523F48053C6F84035538CB3F57A7FEF
:020000040801F1
:10000000BFF424AD4FF47A7353841FE5D6F83C3522
:1000100023F00063C6F83C35D6F8403523F0006382
:10002000C6F840357AE5D6F83C25D6F8403522F0BA
:10003000800223F08003C6F83C25C6F840359EE4D4
:100040005A4608E7D6F8402543F0080342F0080274
:10005000C6F83C35C6F840251EE500BF004100014A
:10006000D8230120F79FFFFDF6BFFFFD6C53012051
:100070006C5401202DE9F04FA74E83B0A74B4FF0F1
:10008000010AD6F81C28DFF8D08202F2DC52434580
:10009000C6F81C284CD29B46A14BA24D9F1CA04BDE
:1000A0005988002900F01A817A18AA4234BF00202A
:1000B0000120052998BF40F00100002840F00E8182
:1000C000BBF800003C46C0F30B000BE0118814465F
:1000D0000A44002900F00281AA4280F0FF8005292D
:1000E00040F2FC8061888142F0D161798B07EDD1CB
:1000F00023885846DBF8081094F804900193FEF723
:1001000045FBBBF80010B9EB113F00F0EF804FF05A
:10011000000ABBF804100BF11C0B5BF8140CC1F3C4
:100120000B0137F05BF95BF8042CC3451060B6D3C4
:10013000D6F83C357C4DC6F84035FFF79BFB337A4B
:10014000A5F17801794C03EB830203EBC203727AC9
:10015000C2EB021205EB830301EB4202C6F8003446
:10016000C6F8FC2317F060FF4FF0FF33D6F8000409
:1001700063601EF00BFE19F015FC05F5926305F5A2
:10018000A16103E00633994200F0BE801A78002A8C
:10019000F8D19D78D878854202D358790028F1D0DB
:1001A00096F8C8356421227203EB830303EB8303C3
:1001B0009B00632BD8BF6423C6F81438B6F8CC353F
:1001C00001FB03F3632B40F39B801A46C6F81838F3
:1001D0000023574C5749C6F81C38C1F81447C6F8D5
:1001E0002038C6F82438C6F82838C6F82C38C6F89F
:1001F0003028A6F8343886F836381FF063FCB6F895
:100200004A38DFED4D6A05EE903AB6F846389FED74
:100210004B7AF8EEE55A07EE903A9FED490AF8EE70
:10022000E77AB6F8441865EEA65AB6F8383867EE9D
:10023000877A35EE800AC4EDAF7AFDEEC07A17EE0C
:10024000902A07EE901A96F83A18F8EEE77A2032DC
:10025000402A67EE877AC4EDB07A01D8FEF76AFBD0
:10026000FDEEE57A17EE902A2032402A03D8B0EE50
:10027000650AFEF75FFB96F848289FED327A07EE95
:10028000902A9FED2F0AF8EEE77AA7EE870AFDEE97
:10029000C07A17EE902A2032402A3AD8FEF74AFB5D
:1002A00007EE903ADFED286A284BF8EEE77AC6F8B9
:1002B0005418A3EC010A86EEA77A83ED007A2CF09D
:1002C000B9FE14F01BFF224B012250461B6886F832
:1002D0003528C6F81C3803B0BDE8F08FDBF80810ED
:1002E00058464FF0000AFEF751FA12E7019BA11D94
:1002F00058469A1FFDF706FD00287FF40AAF06E76F
:100300000A46C6F8181863E7F27D003A18BF0122C2
:1003100046E79FED100AC3E79C4E0120B82A060865
:100320000040000800800008DC4F0120A0030120ED
:100330001C5401208C1F002088C3E43A17B7D13821
:10034000DB0FC93F35FA8E3CC0C9FB48E856012097
:10035000F41A012000000000B432060838B501226A
:100360001C4B032805461C4C83F81C2720D96A1C0B
:1003700000231A490220D2B24FF0140E5200402A34
:1003800028BF4022C854023301EB030C9A420CF8F8
:1003900001ECF7D8FF2D4FF0FF034FF00E0008BF20
:1003A0000222224482F85838BDE8384013F088BE53
:1003B00000EB800004F5A073257205EBC00003EB91
:1003C0008000C4F800041EF0E1FC1DF003F81DF0ED
:1003D000D5F8CCE78C1F00209C4E0120F45601205C
:1003E000054B0121D3F89C2883F8991842F4001298
:1003F000C3F89C28704700BF9C4E01200368C3F3DC
:100400000D032DE9F041054686B00C46002B3FD187
:10041000384A0120384E0221B242CDE90233CDE9FB
:1004200004011ED3354B9A421AD303F580439A42F6
:1004300022D3334B9A4221D903F580339A421FD9F4
:1004400003F500339A421DD903F500339A421BD9B4
:1004500003F500339A4219D905200AF0C5FCFBE7E1
:10046000034601A902A8039336F03AFF80B14FF08A
:10047000FF3006B0BDE8F0810B46F2E70323F0E75A
:100480000423EEE70523ECE70623EAE70723E8E782
:100490001C4E96F8B438012B02D16FF00100E8E74A
:1004A00001232F68D4F8008086F8B43836F0B8FEFF
:1004B000B0B9154C236923F440732361236943F4D5
:1004C00000732361236943F001032361C7F80080AF
:1004D000BFF34F8F36F0A4FE236923F0010323619D
:1004E000002386F8B4380028D7D12B6804332B605A
:1004F000BFE700BF0040000800400008008000087F
:10050000FFFF00089C4E0120003C02402DE9F04115
:10051000594F8AB03B78B12B6ED1FDF7D5FD80F0F5
:100520000104E4B2554B04F00104554DB3F8A73172
:10053000544EADF80030B54260D3002C00F09A80E4
:100540001022002106A83EF0A1FB4F4B0497DB1BB5
:1005500005934E4B1A69002A05DA4D4A5A6002F19A
:1005600088325A601B69012300250222694604A8CB
:100570008DF8243008953BF01BFE022269464FF6A9
:10058000FF703F4FFDF776FC0446B74245D3002588
:10059000022201A904A8ADF804503BF009FE022292
:1005A00001A92046FDF766FC40BA022202A9C04319
:1005B000ADF8080004A83BF0FBFD079868B106AB56
:1005C000C0F10402294618443EF060FB089818B9AF
:1005D00006A904A8FFF712FF08909DF82430089898
:1005E00023B12A4A136943F000431361B0FA80F043
:1005F00040090AB0BDE8F081012493E7A9881C35C1
:1006000055F8140CC1F30B0136F0E8FE55F8043C24
:100610001B68834218BF01248DE7B7F8048002A944
:1006200004A88DF80D50C8F30B081C3708F1060319
:10063000ADF8083037F81C3CC3F30B021B0BADF8C8
:100640000A2006228DF80C303BF0B2FD062202A9EA
:100650002046FDF70FFC044657F8141C424604A838
:100660003BF0A6FD204657F8141C4246FDF702FC5D
:1006700004468AE70120BCE700400008A8030508FB
:10068000B82A0608B432060800800008003C024080
:100690002301674510B5144CFFF7ECF8D4F81C386B
:1006A00003F2DC53C4F81C38FFF730FF10B9FFF732
:1006B0002DFFA0B10D4B1B78B12B02D1FDF704FD2E
:1006C00010B905200AF090FB094B012100221B689C
:1006D00084F8351884F8BC28C4F81C3810BDFFF71E
:1006E00015FF0028E6D1ECE79C4E012000400008F1
:1006F000F41A012001230B4A10B50B4C82F81C3769
:10070000A375FFF7C7FFFFF7B5FC41F20242FF23D5
:100710000E20A4F8582884F85A38BDE8104013F089
:10072000CFBC00BF8C1F00209C4E012090F887306A
:10073000F7EE002ADFED695A002103EE903A90F8B7
:100740008B3006EE103A90F88930F8EEE33A04EE7A
:10075000103A90F88A30B8EEC66A04EE903A90F8F3
:100760008D3063EEA57A03EE903A26EE256AB8EE58
:10077000C44AF8EEE44AF8EEE33A26EE276A24EE9D
:10078000254A64EEA54A63EEA53A24EE064A64EED5
:10079000A74A63EEA73AF0B5514D062600F1660E62
:1007A000A5F10C0CB7EE005A06FB01F290F886702A
:1007B000AC180244F0EE456A15E0012904F1060484
:1007C00002F10602EED190F8883007EE903A90F8E8
:1007D000903006EE903AF8EEE77AF8EEE66A27EE09
:1007E000A55A66EEA56A237866EE867A07EE103A79
:1007F000B8EEC77A27EE277AFDEEC77A17EE903A61
:1008000066EE847AFA2BA8BFFA2323EAE373137205
:10081000637807EE103AB8EEC77A27EE277AFDEE36
:10082000C77A17EE903AFA2BA8BFFA2323EAE373AC
:1008300053725CF8213007EE903A002BF8EEE77A1D
:1008400049DDA37807EE103A90F88C30B8EE477A7D
:1008500003EE103AB8EEC33A37EE677A23EE253A44
:1008600087EE272AB0EE627AA2EE037A64EEA77AC8
:1008700066EEA36A67EE857A27EE877AFDEEE77A61
:10088000BDEEC77A17EE103AFA2BA8BFFA2323EA77
:10089000E373937217EE903AFA2BA8BFFA2323EA78
:1008A000E3730EF801300131A38807EE903AF8EEB9
:1008B000E77A67EEA67AFDEEE77A17EE903AB3F59F
:1008C0007A7FA8BF4FF47A738F4223EAE373938150
:1008D000BFF673AFF0BDB7EE007AC7E70AD7233C87
:1008E0006005050890F88E306BB3B0F85A308BB1C4
:1008F00090F88F20642102EB8203C3EB0313B3FB58
:10090000F1F3A0F85A30962312FB03F3B3FBF1F393
:10091000A0F85C3043884BB190F88F30642203EB31
:100920008303C3EB0313B3FBF2F34380B0F8463009
:100930004BB1962290F88F3013FB02F36422B3FB85
:10094000F2F3A0F84630704790F821304BB3438B58
:1009500083B190F82230FA22642113FB02F203EBF8
:100960008303B2FBF1F2B3F57A7F4283A8BF4FF461
:100970007A738383838843B1FA2290F8223013FB81
:1009800002F36422B3FBF2F38380C3884BB190F887
:10099000223003EB8303B3F57A7FA8BF4FF47A7359
:1009A000C380704770B50B4C002504F5247694F88D
:1009B000863013B12046FFF7B9FE20460135FFF718
:1009C00091FF3046FFF7C0FF042D04F1A404EED1DF
:1009D00070BD00BFDC4F0120034BD3F8C00808B145
:1009E00005F082BE704700BF9C4E012008B50B4643
:1009F00005490246D1F8C00828B10449FEF778F845
:100A0000BDE80840E8E708BD9C4E0120E1E400088D
:100A1000024B0146D3F8C008FDF764BD9C4E01208F
:100A200008B504460848FFF7F3FFFFF7D5FF074B6B
:100A3000186E13F0C3FA0AF063F8012C01D137F0F5
:100A4000E9FAFBF7C3FC00BF1CAC05089C4E012073
:100A50000048DDE7BDB705080CB4C30607B500D5EF
:100A600061B905A904980191FFF7C0FFFFF7F0FFF6
:100A7000012003B05DF804EB02B070470020F8E7F6
:100A800008B5FFF7C5FFBDE80840E1E710B504462B
:100A90000348FFF7BDFF2046BDE81040F0E700BF68
:100AA00028AC05080948002408B5FFF7EFFFFFF759
:100AB00093FF074B83F8C448C3F8C44983F8C84977
:100AC0001CF02CFE2046FFF7ABFF00BF2DAC050845
:100AD0009C4E0120034B0146D3F8C00808B105F035
:100AE000EFBD70479C4E01200CB407B510F02000FC
:100AF0000BD079B92320FFF7EDFF05A904980191E8
:100B0000FFF774FFFFF7A4FF012003B05DF804EBCB
:100B100002B070470020F8E70FB407B504A951F8F8
:100B2000040B0191FFF762FF03B05DF804EB04B022
:100B30007047154B1B6870B52BB30025134E144836
:100B4000FFF79EFFFFF748FFFCF740FAFCF770FA4B
:100B5000044640B1132013F0B3FAFFF779FF0D48B4
:100B6000BDE870408CE73046FFF7D6FF782D06D8F9
:100B70000135FFF731FF64200AF01CF8E6E725464F
:100B8000FFF766FFF5E770BDBC1A0120E9D705083D
:100B900054AC05086EAC05080FB407B504A951F8AC
:100BA000040B0191FFF722FFFFF752FF03B05DF83E
:100BB00004EB04B070472DE9F041037903F0E00243
:100BC000402A50D004D85AB1202A29D0BDE8F0815B
:100BD000602A4BD0802AF9D182794179254812E0E8
:100BE00003F00703052B16D8DFE803F010151015E6
:100BF0000309D0F805102048BDE8F041CCE7D0F853
:100C0000052051421D48BDE8F041C5E7B0F8072076
:100C1000B0F80510F6E7B0F90720B0F90510F1E7D4
:100C200046790024164D174805EBC605FFF7F0FE80
:100C3000012395F8D071A74202D8BDE8F04107E73B
:100C4000D5F8CC614FEA840856F824204AB113B98C
:100C50000D48FFF7DDFE56F808100C48FFF75CFF63
:100C600000230134E7E741790948C5E70948BDE8B1
:100C7000F04191E7C3AC050874AC05088AAC0508DF
:100C8000A8030508A1AC050833B00508F1C00508A4
:100C9000B2AC0508DAAC05082DE9F04387B0224E66
:100CA000FCF784F9026983890025018804460292D1
:100CB0008268DFF88880019242881C4FDFF88090BC
:100CC000009242681A48FFF767FF15B94046FFF7E0
:100CD000D7FE3B689D4212DA3378052B21D809EB09
:100CE0008303D3F87423B388294601351148009350
:100CF000063636F8043CFFF74FFF062DE5D136F0F7
:100D000091FE81884388CB1A616803FB011105912C
:100D1000FCF7D4F905990246074807B0BDE8F0434F
:100D20003AE70022DFE700BF9C2701208C27012043
:100D3000F2AC05085CAD05086BAD050850AD0508C3
:100D4000A80305080249034801F521610EC923E7FC
:100D50000070F01F88AD050810B5752104461FF01E
:100D60000DF901460948FFF717FF1A2120461FF029
:100D700005F901460648FFF70FFF1B2120461FF02B
:100D8000FDF801460348BDE8104005E79CAD0508A5
:100D9000AFAD0508C2AD050838B50C4D95F8D303C5
:100DA00010F0FD0405D10A48FFF7F6FE2046FFF7D4
:100DB000D3FF95F8D333013B012B06D80548FFF745
:100DC000EBFE0120BDE83840C6E738BD9C4E01204F
:100DD000D5AD0508E0AD0508614B62491A68624B64
:100DE00062482DE9F04F624C93B0624D624FDFF8DC
:100DF000B081B2FBF3F2FFF78FFEB4F8CA294FF4CB
:100E00007A730A20B2FBF3F103FB1122B4F9CC3957
:100E100092B2B2FBF0F25948FFF7BEFE584A594968
:100E20005948FFF779FEFFF713FEA17D574A05EBFE
:100E30008101574B5748D31AD1F88C13A288FFF77A
:100E4000ABFE5548FFF7E4FD94F8CE195348FFF781
:100E500063FE5348FFF7DCFD94F8CF195148FFF7C4
:100E60005BFEFFF7F5FD5048FFF7D2FD00210A4673
:100E700094F8EF334E1C0B4113F0010F08D012B160
:100E80004046FFF7C5FD31463846FFF745FE0122D3
:100E9000072E3146ECD1454E96F86A1506F5EC73EF
:100EA00006F13C02012918BF134693F8DC30032BEE
:100EB00002D03F48FFF730FE3E4B96F86A15A3F587
:100EC000CE72012918BF134693F8DC30012B02D1F2
:100ED0003948FFF721FE374B96F86A15A3F5CE7215
:100EE000012918BF13461B695B7B012B02D93348CC
:100EF000FFF712FEDFF8D480FFF7AAFD0027D4F831
:100F0000D03908F12009DFF8C8B0039358F8041B62
:100F100000295FD0012303FA07FA039B1AEA030FA3
:100F20001CD01AF01F0F19D0254B59F82720D85D77
:100F300052F8202037B12348CDE90412FFF768FDAD
:100F4000DDE904125846FFF7E7FDBAF1020F05D1BB
:100F500096F83D1711B11C48FFF7DEFD0137D5E7C4
:100F60004C1B012056C2050840420F00F3AD050896
:100F70009C4E0120A8030508AEAE050806AE050884
:100F8000000001200008000027AE050800800008CE
:100F9000004000084BAE05087AAE05088CAE050887
:100FA00094AE050896AE05089EAE05088C1F00207D
:100FB000B7AE050864210020BFAE0508C4AE050821
:100FC000AC03012033B00508D2AE05083C07050884
:100FD000CCAE0508FFF73CFD94F8D819D4F8D42915
:100FE00005EB81017D48137AD1F8C813527AFFF7D7
:100FF000D3FD7B497B48FFF78FFD7B497B48FFF79B
:101000008BFDFFF725FD7A4B7A4819684FF47A7308
:10101000B1FBF3F1FFF780FD07A8FEF7FBFA38B14B
:1010200007A90AA83BF0F0F90AA97348FFF774FD75
:10103000FFF70EFDD4F8642A002A00F08A8007EE3C
:10104000902ADFED6E6AB8EEE77AC6EE877AFDEE9B
:10105000E77A17EE903A6A4F37F89C0C58B107EED2
:10106000900ADFED666AF8EEE77A86EEA77AFDEE83
:10107000C77A17EE900AD4F8E41959B107EE901A1E
:10108000DFED5E6AF8EEE77A86EEA77AFDEEC77AC4
:1010900017EE901AB6F87867642ECDE90001314654
:1010A0005848A8BF6421FFF777FD17F89A3C17F856
:1010B000992C05EB830337F8981C5348D3F8DC339D
:1010C000FFF76AFD37F8881C504889B2FFF764FDC6
:1010D000FBF76CFF016921B182684D48120DFFF7E3
:1010E0005BFD4C48FFF794FCD4F840351B0660D5F7
:1010F00017F8683C032B8CBF47484848FFF788FC2B
:1011000094F88034022B26D14548FFF781FC17F86C
:10111000683C042B44D84348FFF77AFC17F8583C46
:10112000002B44D005EBC303D3F834143E48FFF73B
:10113000F3FCFFF78DFC3D48FFF76AFC0126D4F86D
:101140009C483B4F002C38D1FFF782FC13B0BDE820
:10115000F08F13467FE7022010F0CCFE064608B958
:101160003448D2E727F094FE96F9041005EB80008E
:101170000131D0F8F0233048FFF7CEFC94F88334E7
:10118000012B04D12D48FFF743FC2D48BDE7B3796F
:101190002C4805EB8303D3F8F013FFF7BDFCF4E70D
:1011A00094F882340BB92848B6E72848B4E72849B0
:1011B000BCE72848FFF72CFCBBE794FAA4F33846B9
:1011C000B3FA83F306FA03F205EB8303D3F868144A
:1011D00024EA0204FFF7A0FCB4E700BFD6AE05087E
:1011E000E8AE050809AF050817AF05081DAF0508EB
:1011F000F41A012023AF05083DAF05080024744907
:10120000945F012050AF050896AF0508BDAF0508F3
:10121000CCAF0508E7AF0508EDAF0508F9AF050845
:1012200009B0050824D8050851B005086DB00508B7
:101230005DB005080FB0050819B005082DB0050808
:1012400032B0050853BA050836B0050846B005089F
:10125000EBAD050861B005082DE9F04FDFF86C81B2
:1012600099B098F80B30002B00F093804E48002581
:101270004E4EDFF85CB1FFF703FC2F46DFF85491C8
:10128000DFF854A10BA9E8B215F0C8FE9DF8343080
:10129000002B53D0139C54B107EE904A9FED440AA3
:1012A000F8EE677A80EE270A3CF004FF04460B9ABA
:1012B00029465846FFF730FC109A002A6BD002FBF3
:1012C00004F04FF47A73B0FBF3F30993DDF848C0F0
:1012D000BCF1000F61D00CFB04F142F21073B1FBC2
:1012E000F3F1082D98F80B3018BF7F18002B56D05B
:1012F00017984FF47A7E0A2307901598069016984F
:1013000005901198B0FBFEFECDF810E00998B1FBF6
:10131000F3FE03FB1E11CDE902E10999B1FBF3F1E4
:1013200003FB1100BCFBF3F3CDE90010214650464E
:10133000FFF732FC0023B362C6E90D3301354036B6
:101340001A2D9FD198F80B3003B31A4C4FF47A73CF
:10135000194854E91512B1FBF3F3D20854F84C1CA8
:10136000FFF71AFC0A221548B7FBF2F102FB1172D3
:10137000FFF712FC124B1B78432B04D1114854E9A0
:101380001221FFF709FC002344F84C3C19B0BDE8DA
:10139000F08F0D486BE7099298E76146A1E7214677
:1013A0004846FFF7F9FBC5E783B0050878580120E8
:1013B0008096184B945F01202AB105084AB10508B0
:1013C000951B01206EB10508E1B005089C4E012077
:1013D000EBB005088DC00508FAB0050813B529481B
:1013E000FFF716FB284B93F8AD35002B48D0274864
:1013F000FFF746FB16F0A4FB80B1254B254893ED83
:10140000280A8DED010AFFF703FB234B9DED010A2E
:1014100033F89C3C3BBB2148FFF732FB204C214872
:10142000B4F81418FFF778FB94F8103813B31E487B
:10143000FFF726FBB4F818181C48FFF76DFB94F86B
:101440001238CBB11848FFF71BFBB4F81618184830
:10145000FFF762FB94F8113883B1134802B0BDE87E
:101460001040FFF70DBB3CF025FE81B21148FFF79D
:1014700093FBD3E71048DBE70F48E4E70E48EDE7BE
:101480000E48EBE798B105089C4E0120AEB1050867
:1014900008270020B5B10508945F0120CFB10508E9
:1014A0008C1F0020DEB10508FEB105080EB205084C
:1014B00028B20508D9B1050807B2050826EF0508C6
:1014C0000EB403B503AA52F8041B0192FDF758FDB0
:1014D000064BD3F8C0281AB90549986EFDF702F8F3
:1014E00002B05DF804EB03B0704700BF9C4E0120D2
:1014F000BDB705082DE9F04798460B7981460F46A0
:1015000003F0E0041646402C31D10024674DDFF88B
:10151000A081DFF8C09122E03B7903F00703013B93
:10152000042B04D8DFE803F006080B0E2000315D21
:1015300028460AE03157FBE736F81410F8E736F989
:101540001410F5E756F824104046FFF7E5FA7B79CA
:10155000013BA34202DD4846FFF75AFA01347B798A
:10156000A342D9DCBDE8F08756F82410E0E703F089
:101570000703052B58D8DFE803F0030C14161931C4
:101580003578602C5ED045D8002C66D0202C7CD0DD
:10159000E8E796F90050602C54D03BD8002CF5D1E8
:1015A00048E03588EDE7B6F90050F4E7D6F800A03A
:1015B000202C554669D02BD8002CD3D151463C481D
:1015C000FFF7AAFAD7F805108A4518D8B8F1000F26
:1015D000C8D03848BDE8F047FFF79EBA202C3568E0
:1015E00053D015D8002CBDD129463048FFF794FAC6
:1015F000D7F80510A94202DB4B42AB42E6DDFFF70C
:1016000027FA2B463A6848462B49BDE8F04757E78A
:10161000602C17D0802CA5D13178284B2848002980
:1016200014BF31461946D5E7202C2DD007D8002C01
:1016300098D12546B7F90540B7F9076011E0602C4D
:10164000E8D100257B7945FA03F3DB07BDE8F047D5
:101650004CBF1C481C48FFF75FBAB7F80540B7F805
:10166000076029461148FFF757FAAC42C7DCAE4283
:10167000C5DBB8F1000F3FF475AF32462146134881
:10168000BDE8F047FFF748BA00257A79104B03EB25
:10169000C20393F8D0219542B1DAD3F8CC3153F894
:1016A0002500BDE8F047FFF7B3B900BF9EAC0508C1
:1016B00087AC050848B205084EB20508B8D8050839
:1016C000F1C00508EFAC050826EF050863AB050877
:1016D000A803050894AE050813B504460846019210
:1016E0000091FCF7F9FF02462046DDE9001302B045
:1016F000BDE81040FEE60EB403B503AA52F8041B81
:101700000192FDF73DFC054B0549986EFCF7EAFE9A
:1017100002B05DF804EB03B0704700BF9C4E01209F
:10172000BDB7050802460149E5E700BF68B20508F4
:10173000F8B50C4606460846FDF78EFE2021054604
:1017400020463DF0AAFB044618B93046BDE8F840F3
:10175000E8E7114F114E3B7832789A4201D0FBF7FF
:1017600069FD0F4B20461D603AF0D4FF012201466F
:101770002046FBF701FD3B7832789A4201D0FBF717
:1017800059FD20463AF0C6FF2A4601460548BDE805
:10179000F840FFF701BA00BFB81A012094270120D2
:1017A000B41A01207FB205082DE9F0410D4688B03A
:1017B00006460846FDF750FE2021044628463DF027
:1017C0006CFB20B9304608B0BDE8F041AAE7FDF750
:1017D00043FE2246054601460F48FFF7DDF985B175
:1017E000202D2A466946204628BF2022E846FBF7DE
:1017F0003DFD00270646B74208DBAD1B3444002EF2
:10180000EDD1FFF725F908B0BDE8F08118F8010B1C
:101810000137FFF75FF9EEE795B2050810B504460A
:101820000748FFF72DF9FBF7B7FD20B10548BDE8E4
:101830001040FFF725B920460349BDE810405AE79C
:10184000ADB20508B7B20508BFB20508154B53F88D
:10185000403C2DE9F041044688B0F3B11A6804A970
:101860001846D56A6A46A847064688B104AC6D4654
:101870000027DFF83C80013735F8022B34F8021BD3
:101880004046FFF789F9BE42F5DC08B0BDE8F081BB
:1018900005492046FFF72FFFF7E7044908B0BDE8E8
:1018A000F04128E7945F0120E0B20508F8B205088E
:1018B000C6B2050813B50446084601913AF02AFF5E
:1018C000024670B1092804D1019909483DF00BFB8B
:1018D00038B1074B2046074A074902B0BDE810401F
:1018E00009E70349054802B0BDE81040FFF754B9C5
:1018F000646B0508FFB205080AB3050834B3050890
:1019000013B50446084601913AF004FF01990246D6
:1019100068B1042803D109483DF0E5FA38B1074B16
:101920002046074A074902B0BDE81040E3E60349F4
:10193000054802B0BDE81040FFF72EB95C6B050802
:1019400042B305080AB3050852B305082DE9F04370
:1019500000279BB0064608460C463AF0DBFE0546DB
:101960001C22394602A801973DF090F925B3402D7D
:1019700007D040232A46384930461BB0BDE8F04323
:10198000B9E60DF1040804F1400902222146684637
:101990003DF0BDFA0023102209A968468DF80270B7
:1019A000FDF7B6FC099B0DF10202934222D10234ED
:1019B00008F8010BA145E8D100213D220AA80991B0
:1019C0003DF064F9002D3AD0244C257ED5B120227B
:1019D00004F11C0101A83DF02FF998B104F11C019C
:1019E00009A8FDF7A3FB09AB1D4A30461D49FFF7C7
:1019F00082FE04E01A7830461B49FFF77CFE1BB0DC
:101A0000BDE8F08394F86430CBB9C5B901AD174C8B
:101A10000FCD0FC495E80F0084E80F00144B01228E
:101A200009A8A4F1100103F83C2CFDF77FFB114835
:101A3000FFF72CF809A91048FFF7AEF8DFE70C4BC9
:101A400013F83C3C1BB9054B1B7E002BF2D0074919
:101A500009A8FDF76BFBEDE765B305089C4E012077
:101A6000A3B305080AB3050887B30508B84E0120DB
:101A7000945F0120ADB30508BCB305082DE9F74F0D
:101A80003D4F834608460D463AF044FED7F83C9554
:101A90000446B8B9394D0126394F3A48FEF7B8FF28
:101AA00055F8041B49B106FA04F313EA090F02D0F2
:101AB0003846FFF731F80134F2E703B0BDE8F04FE4
:101AC000FEF7C6BF024630492846FDF7D1FB78B97C
:101AD0002A4C2E4D2E48FEF79BFF54F8041B00297C
:101AE000EBD00B78002BF8D02846FFF715F8F4E779
:101AF0002B782D2B11D10135013C4FF0010A1F4BE2
:101B0000002653F8048BB8F1000F09D12A46214969
:101B1000584603B0BDE8F04FEDE54FF0000AEEE7A0
:101B20002246414628460193FDF7A2FB019B00BBDC
:101B30000123B3409A0505D5174803B0BDE8F04F1F
:101B4000FEF79EBFBAF1000F0DD029EA0303134838
:101B5000C7F83C35FEF75CFF41460C4803B0BDE8D2
:101B6000F04FFFF719B849EA03030D48C7F83C35B1
:101B7000F0E70136C5E700BF9C4E01207808050854
:101B8000D3B30508C9B30508E6B005085DB005087C
:101B9000D7B30508E2B30508F3B30508FFB305089A
:101BA00008B405082DE9F74F814608460E4617464A
:101BB00098463AF0AFFD0446E8B9404D4048FEF77C
:101BC000ABFF20460FF0AAFF3B68184206D0204624
:101BD0000FF0B6FF01462846FEF79EFF0134182C91
:101BE000EFD13B6813B93748FEF712FF03B0BDE8E9
:101BF000F04FFEF72DBF024633493046FDF738FB64
:101C00000546A8B92C46314D3148FEF701FF204664
:101C10000FF084FF10EA080F06D020460FF090FF67
:101C200001462846FEF778FF0134192CEFD1DDE795
:101C300033782D2B2AD10136013C012548F08073E1
:101C40004FF0000A019350460FF07AFF2246834678
:101C500001463046FDF70CFB18BB50460FF05EFF07
:101C6000019B03421DD09DB1BAF1180F02D03B6811
:101C700040EA03081748C7F80080FEF7C9FE594636
:101C8000124803B0BDE8F04FFEF786BF0025D5E748
:101C9000BAF1180F02D03D6825EA00050E483D60F4
:101CA000EBE70AF1010ABAF1190FCCD132460B4920
:101CB000484603B0BDE8F04F1DE500BF5CB0050825
:101CC00010B405081AB40508E6B005085DB00508AB
:101CD000D7B30508FFB3050808B40508E2B3050843
:101CE00040F20223004A5DE7085501206FF07F4370
:101CF000004A57E70055012070B5054608461646CC
:101D0000FDF7AAFB0D4B044693F89025904205D2AF
:101D100001460B48FEF740FF204670BD2EB1FF285C
:101D200003D10848FEF738FFF6E7013A064928468E
:101D30004FF0FF34FFF7DFFCEEE700BF8C1F002001
:101D400021B4050832B4050845B405082DE9F04F63
:101D5000074691B082480E46824DFEF71DFF0023D4
:101D600081494024062205F8343C3046012391F88D
:101D7000901545F838DC05F8334C08F087FD0A204B
:101D800008F018FF15F8343C0C2BDAB240F2E4806E
:101D90009DF80C50FE2D30D0FF2D0BBF15240F24C5
:101DA00001260026944240F0D780611E6846C9B2E1
:101DB0002CF020F804F140030DEB030414F8413C2F
:101DC000834240F0C48006F1FF389DF80D305FFA81
:101DD00088F8B8F1010F12D903F01F075C096137C9
:101DE0006248FEF715FE022E6AD0013C042C65D82D
:101DF000DFE804F00B5E606462000226D2E79DF823
:101E00000E701D469DF80F40EAE759486C464FF0AA
:101E1000000ADFF8B891FEF733FEDFF8B4B1554899
:101E2000FEF7F6FD0AF1010A14F8011B4846FEF719
:101E300073FEBAF10C0F49D1FEF70AFE022E4FD005
:101E400064223B464C48B5FBF2F102FB1152C9B289
:101E5000D2B2FEF7A1FEB8F1010F71D8474A484B44
:101E60009DF810104748002914BF11461946464DE9
:101E7000FEF792FE9DF81110444B4548002914BF0F
:101E800019462946FEF788FE022E59D19DF81240C8
:101E90004048FEF7BDFD4CB3FF2C37D00A223E4828
:101EA000B4FBF2F102FB1142D2B2FEF775FE20E064
:101EB0003A48ABE73A48A9E73A48A7E73A48A5E7DE
:101EC00000230DF11F008DF83F309FE7374B03FBD8
:101ED0000AF2B2F1553FA5D85846FEF799FDA1E7A1
:101EE0003A4629463248FEF757FEB7E72846FEF73E
:101EF000C7FD9DF813402F48FEF78AFD44B1FF2C23
:101F000021D021462C48FEF747FE04E02B48EEE79F
:101F10001D48FEF7B5FD0DF1130500241A4E274F9D
:101F2000DFF8688015F8013F7BB1FF2B0CBF3A4604
:101F30004246214601342248FEF72EFE042CF1D100
:101F400011B0BDE8F08F1D48E3E73246F1E71D49C7
:101F50003846FFF7D0FBF3E71B48FEF791FDEFE7AC
:101F60008BB40508945F01208C1F00209CB40508E9
:101F7000A7B40508CDB40508DFB405086BB405089F
:101F800074B4050816B505087BB40508C4C2050875
:101F90002DB5050834B5050848B50508AEB40508E3
:101FA000B6B40508BEB40508EBAD0508ABAAAAAAED
:101FB000FBB4050850B505089EAC05087FB40508BC
:101FC00060B505086BB505087BB5050814AC0508B8
:101FD000B8D805082DE9F84F07460C46DFF8A4806D
:101FE000DFF88490DFF8A0A020463AF093FB064685
:101FF00060B91D4B1D4893F804241D4B03EB82036D
:10200000D3F84815BDE8F84FFEF7C6BD0246414675
:102010002046FDF72DF960B1DFF85CB000255BF8D4
:10202000041BB1B9224638461249BDE8F84FFFF704
:1020300062BB114C114D1248FEF7EAFC54F8041B28
:1020400019B12846FEF768FDF8E7BDE8F84FFEF73E
:10205000FFBC324620460135FDF70AF90028DED1E3
:10206000544689F80454BFE79C4E012084B5050806
:10207000A8030508E2B30508F40805085DB00508E3
:10208000D7B30508E6B0050866C5050838B50D469E
:102090000446052219492846FDF7EAF868B9184BA5
:1020A00093F86C2022B9012183F86D2083F86C101D
:1020B0001448BDE83840FEF7E3BC03221249284625
:1020C000FDF7D6F8A0B90E4D95F86C3063B195F8D0
:1020D0006D304BB10D492046FFF70DFB002385F80D
:1020E0006C3085F86D3038BD0948FEF7C9FCF5E75E
:1020F00020460849BDE83840FFF7FDBA13C205087D
:102100009C4E01208EB505086DC30508A4B50508D1
:10211000DBB50508EFB50508F8B5164C054694F88B
:102120006C307BB194F86D3063B11349FFF7E3FA7B
:1021300028461249FFF7DFFA002084F86C0084F883
:102140006D00F8BD0E4E16F83C7C8FB1207E002845
:10215000F7D10C4DA6F130040FCD0FC495E80F0058
:1021600084E80F000123F37209F0B6FC3846E8E773
:102170000120E6E79C4E0120A4B50508FEB5050840
:10218000945F0120B84E012008B5FFF7C5FF50B19C
:10219000054B01229A75FEF77DFA0448FEF776FC9E
:1021A0000020FEF73DFC08BD9C4E01201CB6050832
:1021B00008B5034610462AB1DB0600D511B1FEF77B
:1021C00065FC002008BDF8B50D4E054696F8643054
:1021D00093B9F8BD25B12388C3F30B039D4204D006
:1021E000A288D4E902013CF0DDFC1C34BC42F1D3EE
:1021F000002386F86430ECE7024C034FF6E700BF9B
:102200009C4E0120B82A0608B43206082DE9F04F8A
:10221000164685B01A468246019130460021334C5D
:10222000FFF7C6FF4FF0000906F0100305460293C2
:10223000FEF7D2FB2379019A03F01803934203D0EF
:10224000002A48D1182B46D14FF00D0B274B0BFB22
:102250000933B3F80900FCF729FA80462046FBF75A
:10226000AEFF0746D8E90221024401442046FBF7AD
:102270005FFF80F001012A460390C9B23046FFF7A4
:1022800097FF0546DDE9022302B123BB174A0BFB8A
:1022900009FB52F80BB0B2060FD573B95946144872
:1022A0000393FEF739FCD8F808202146039B5046DB
:1022B0003A44FFF71FF9FEF7CBFB59460D48FEF7EE
:1022C0002BFCD8F80C20002321463A445046FFF757
:1022D00011F9FEF7BDFB09F1010940F22D230D3480
:1022E0009945A5D105B0BDE8F08F00BF841B050856
:1022F00023B6050824B605080149FFF7FCB900BF5D
:102300002EB6050838B50C46054615492046FCF79B
:102310008BFF30B9FEF746FB1248BDE83840FEF7A8
:10232000AFBB11492046FCF77FFFA0B90F4A82F8E6
:10233000C60182F8CE0182F86A0282F8720282F83F
:102340000E0382F8160382F8B20382F8BA0382F809
:10235000F1030748E1E72846BDE83840CCE700BF75
:102360003DB6050843B605085EB605089C4E01203B
:1023700066B605082DE9F043064687B008460C46C8
:102380003AF0C8F9082844D1671E03AD073429463E
:102390003A46A84612F8010FFCF740FF01F8010B7E
:1023A000A242F7D10023DFF880908DF8143017F89F
:1023B000010FFCF733FF05F8010BC1B2484601914C
:1023C0003CF06BFD20B1019928463CF066FD28B138
:1023D0003046FFF791FF07B0BDE8F083A742E6D192
:1023E000104940461DF004FB0E4808230E4910F822
:1023F000012B013B11F8014B02F118026A4402F86B
:102400000C4CF4D103A909488DF81430FEF7C4FB35
:10241000E1E70028E8D0304607B0BDE8F043FFF719
:1024200081B900BF2854012048AB050882B60508D1
:102430002DE9F74F4FF0000B064601AA08462E493A
:102440005D463CF0E5FB01270446DFF8BC80DFF881
:10245000BC90DFF8A4A01CBBBBF1000F28D1274C17
:10246000002D44D029462648FEF796FB94F86430A8
:102470000BB903F01DFFFCF7ABF9002384F86D30B6
:10248000FEF790FA15B12846FFF79DFE9FB1304642
:10249000FFF742FE78B1FEF7FDF80020FEF7C0FA24
:1024A000BBF1000F0AD02046FCF7D6FF85B2C5B9B4
:1024B0003046FFF721FF03B0BDE8F08F41462046CC
:1024C000FCF7FAFE80B949462046FCF7F5FE0028E5
:1024D000EED05F4601AA514600203CF099FB04462D
:1024E000B9E74FF0000BF5E74FF0010BF2E70548B5
:1024F000FEF7CCFABFE700BF2BAC05089C4E0120CD
:1025000092B60508B5B6050889B605084AC2050899
:1025100007B5009313460A460249FFF7ECF803B0EB
:102520005DF804FBCBB6050820B10078B0FA80F066
:1025300040097047012070472DE9F34106460846DF
:10254000FFF7F2FF0D46074670B1002401A92046AF
:10255000013434F059FB01463046FFF7EDFF122CF1
:10256000F4D102B0BDE8F0810846FCF775FFC4B2B3
:10257000112C6DD8681C3A4DFBF734FF8046D0B95A
:10258000384B03EB4403197B8A1E51425141354BB2
:1025900003EB44031A7BAA5C002952D05B7B192011
:1025A00040F2EE2100FB031321462F4802B0BDE8A4
:1025B000F041FEF7F1BA017828463CF06EFC78B1A4
:1025C000032C2A49A0EB050394BF0022012202EB51
:1025D00042020A4452FA83F393F8B875032F04D1E8
:1025E000304602B0BDE8F04186E64046FBF7FAFE11
:1025F000F8B1022FF4D1FCF72FFF40F6CA0280B2E7
:10260000184B904203EB4403A8BF104640F2EE2261
:102610009042B8BF10461922A0F2EE20B0FBF2F0B3
:102620005873BB1E594259410E4B03EB44031F73B1
:10263000ADE7022FF5D1304602B0BDE8F041FFF71B
:1026400071B821460A4802B0BDE8F041FEF7A4BACD
:1026500011233A460749304602B0BDE8F04157E73A
:1026600028800508945F0120E4B60508A803050842
:10267000F4B6050801B705082DE9F04F024691B000
:1026800008460B46FFF750FF044628B1104611B02C
:10269000BDE8F04FFFF746B84FF0FF322746264619
:1026A000DFF8E082DFF8E092DFF8E0A2CDE9082071
:1026B000A24A126E92F83810CDE90E02CDE90C1044
:1026C000CDE90A0007AA9E4918463CF0A1FA054642
:1026D00004944DB9089A0C9FBA4262D19948FEF70A
:1026E0005BFA11B0BDE8F08F062F12D8DFE807F0D3
:1026F000041E2328454C510051462846FCF7DCFDBA
:1027000078B14FF4806001240FF0F4FB90F90430AD
:10271000089307AA8A49002001373CF079FA054658
:10272000D7E72846FCF798FE0890F2E72846FCF722
:1027300093FE0990EDE72846FCF7D5FD0A90E8E7FF
:10274000284639F0E7FF4146024605902846FCF747
:102750008FFD18B3059A49462846FCF789FD0646C1
:102760000028D6D02846FCF777FE04280646D0D9A4
:1027700001467548FEF710FAB3E72846FCF76CFEF1
:1027800000230C900F93C4E72846FCF765FE0D90DC
:10279000BFE72846FCF7A7FD0E90BAE70123049394
:1027A000B7E7DFF8EC8151B2434613F9010B8842D9
:1027B00008D00135092DF8D1002101316348FEF719
:1027C000EBF98EE701216248FEF7E6F900237AB2C1
:1027D00018F9011B8A4200F00C810133092BF7D153
:1027E0003A460121E9E7A7F1140253425341059308
:1027F00008AD002303F10108EB68A3BB95F900B015
:1028000058460FF043FBD5F804A020B1D0F8009053
:10281000B9F1000F5ED1BAF1000F19D14FF4614345
:102820004FF0010A6B60AB680BB90323AB60002368
:10283000D5F804905846029319462A7ACDE90092B9
:102840001A4611F057FBE86028B94146414891E724
:102850004FF0000AE7E74A464146BAF1000F37D089
:102860003D48FEF759F9B8F1020F05F110054FF098
:102870000103BFD1059BDDF83C800B9D53B1374868
:10288000FEF7FEF8D8F800301B6A1BB12A4634491F
:1028900040469847049B002B4ED03249324B142FB0
:1028A00018BF19463148FEF777F9142F09D1049B58
:1028B00003B936B12B68DB691BB132462C49284677
:1028C0009847002C66D100224146284634F050F942
:1028D0002848C6E7C5F80C90BAF1000F25D041464C
:1028E00025485246FEF718F95146484602F090FE38
:1028F000D5F808A0BAF1000F0FD099F8042092453E
:102900000BD0534641461D48FEF706F9D9F8003072
:102910005FFA8AF148469B699847D9F82C30002B1A
:10292000A1D00023C9F82C309DE7D9F808204146F2
:102930001348FEF7F1F8DBE70B49B3E79C4E0120A3
:102940002BAC05083FB7050827B7050883B805086D
:1029500058B7050864B7050880B7050837B80508F3
:102960001156010809B7050866C5050860B80508CD
:1029700009E50008A4B70508C0B7050812B805089E
:10298000EDB7050821B705081CB4050816B70508FA
:10299000660905081C4F0026DFF874904FF0030A03
:1029A00004F0E4FC052008F005F999F89035B342ED
:1029B00089D917F801BBBBF1000F15D0584608F0B4
:1029C000F9FE044680B1584604F0ECFB08B1A0F8CB
:1029D00006A001210490F7F753FFA379049813F0A0
:1029E000010F03D0F7F7DEF90136DEE7F7F7D4F988
:1029F000FAE73A4602210548FEF7CEF8099B002B7C
:102A00003FF4F1AE0023F2E6E023012058B70508B9
:102A10008C1F002010B5044608460B46FFF784FDC6
:102A200028B9032208491846FCF722FC28B90748B0
:102A3000FEF72CF80120FDF7F3FF20460449BDE81E
:102A40001040FEF758BE00BF95B8050899B80508B4
:102A5000EFB505082DE9F74F05460846FFF764FD79
:102A60000B46044618B9334A92F8307027B9284605
:102A700003B0BDE8F04F3FE42646DFF8C880DFF83A
:102A8000C89001AADFF8C4A018462B493CF0C0F852
:102A900010B904F079FC08E056B901220146284635
:102AA000FFF72AF9421C04461BD103B0BDE8F08FA2
:102AB000FCF7D2FC2F28834636D80FB104F056FC21
:102AC000BBF1060F14D01D4901235FFA8BF291F878
:102AD0009015E0B207F0DAFE002759464846FEF7A7
:102AE0005BF801AA1449002001363CF091F8CFE7C9
:102AF000DAF840351B0113D5FF2C0FD0E1B2284680
:102B0000FFF724F9E8E701372846FFF71FF90B4BD9
:102B1000F9B293F890258A42F5D8DDE70027F6E769
:102B20000748FDF7ADFFD7E72F2241462846FEF7BD
:102B3000E2FDD6E7945F01202BAC05088C1F002036
:102B4000BBB80508DBB80508CAB805089C4E0120CB
:102B50002DE9F04F064685B008460B46FFF7E4FC2A
:102B6000044628B1304605B0BDE8F04FFEF7DABDA7
:102B700003AA3049184627463CF04AF8A0460546C5
:102B8000DFF8C090DFF8C0A0DFF8C0B05DB92A4B15
:102B90003A46A1B2186E35F031F868BB2749304685
:102BA000FEF7A9FD28E0B8F1000F06D0B8F1010F3B
:102BB00025D03046FEF7B6FD1EE0284639F0AAFDC6
:102BC0004946024601902846FCF752FB50B3019A51
:102BD00051462846FCF74CFB30B3019A594628462B
:102BE000FCF746FB10B3019A28461549FCF740FB59
:102BF000F0B13046FFF780FB05B0BDE8F08FBB1E9B
:102C0000294630465A425A41FFF776F8421C04469C
:102C1000F2D003AA0749002008F101083BF0F8FFB1
:102C20000546B3E74746F4E70127F2E70227F0E756
:102C30000327EEE72BAC05089C4E012007B90508D9
:102C400004B90508FBB80508FEB8050801B9050870
:102C50002DE9F74380460846FFF766FC0B4605461C
:102C600028B14046FEF75EFD03B0BDE8F08301AA3F
:102C70002D4918462F463BF0CBFF2E460446DFF881
:102C8000A8907CB9022DECD1A7F57A73B3F57A7FC1
:102C900021D94FF4FA634FF47A7224494046FFF782
:102CA00037FCE1E74DB1012D10D001AA49460020C3
:102CB00001353BF0ADFF0446E3E7012221464046E3
:102CC000FFF71AF8431C0646EFD1CDE72046FCF784
:102CD000C3FB0746E9E7164DB8B2D5F830385B6854
:102CE0009847FF2EBCEEC00A0CD1F8EE407A95F85A
:102CF0009025104BA24213DC10EE101A0E48FDF77F
:102D00004BFFB1E70D4BF8EE407A10EE102A31463A
:102D100003EB86030A48C3ED0D7AFDF73DFFA3E7F9
:102D20000134E3EC017AE5E72BAC050815BA050898
:102D30008C1F0020C85F012032B90508945F012074
:102D400025B90508F8B507460846FFF7EDFBC8B1F9
:102D50001F4B5E690136304634460EF0F1FE0546E3
:102D6000F0B90134192CA8BF002420460EF0E8FE6B
:102D70000546A8B9B442F4D138461649BDE8F84032
:102D8000FEF7B9BC0846FCF767FB04460EF0D8FE18
:102D9000054628B921461048BDE8F840FDF7FCBEBD
:102DA0000B4B5C6111F056F92A4621460B48FDF7A2
:102DB000F3FE182C09D80A480C2101FB040090F8F6
:102DC000C805BDE8F84011F07BB90020F9E700BF65
:102DD000A003012041B9050855B905086BB90508DC
:102DE000A803050838B50446114D0846FFF79CFBBB
:102DF00068B1104B93F900104B1C06D10E4B197A99
:102E00000E48BDE83840FDF7C7BEC9B2F8E708462E
:102E1000FCF722FB032804D8C0B2FDF79FFA29462D
:102E2000E3E7204603220649BDE83840FEF763BCCD
:102E300066C50508A00301209C4E012084B9050841
:102E400094B9050838B50446114D0846FFF76CFBE8
:102E500068B1104B93F901104B1C06D10E4B597AF7
:102E60000E48BDE83840FDF797BEC9B2F8E70846FE
:102E7000FCF7F2FA032804D8C0B215F0C9F92946C4
:102E8000E3E7204603220649BDE83840FEF733BC9D
:102E900066C50508A00301209C4E012080B90508E5
:102EA0008FB90508444B2DE9F74FDFF824A10546FB
:102EB0001A7A88468AF800205A7A93F864308AF899
:102EC00001200BB903F0F4F900263C4CFBF780FC21
:102ED000B1460D23394A4146734352F803B0584670
:102EE000FCF7EAF9002841D0B9F1000F01D0FDF755
:102EF000AFFD59463248FDF70FFE00222146284615
:102F0000FEF7EAFBFDF7A4FD237903F01803082B75
:102F100045D0102B48D02046FDF74DFE274A0D2303
:102F200003FB0623B3F80900FBF7C0FB0746D8B143
:102F30002046FBF744F90090D7E9022102440144FE
:102F40002046FBF7F5F878B9594601901D48FDF782
:102F5000E3FD019AB96828461346009A0A442146BF
:102F6000FEF7C8FAFDF774FD09F10109013640F2D8
:102F70002D230D349E42ACD10020FFF724F9FF230E
:102F80008AF800308AF80130B9F1000F11D14246B9
:102F90000D49284603B0BDE8F04FFEF7ACBB0B4926
:102FA0002846FFF71FFFB6E708492846FFF74AFF04
:102FB000B1E703B0BDE8F08F9C4E0120841B0508EB
:102FC00028B60508AFB90508E2B3050866C50508C7
:102FD000A00301202DE9F74F074608460E4639F0B9
:102FE00099FB044620B1012825D132782A2A22D122
:102FF000B24E00254FF00D0BDFF8E092B24640F2E2
:103000002D28AF48FDF73CFD0BFB05F34846013585
:103010005AF80310FDF780FD221E3146384618BFCE
:1030200001220D36FEF758FBFDF712FD4545EBD1A9
:1030300003B0BDE8F08F3D2130463BF02EFF002865
:1030400000F0368101460A4611F8014D202CFAD0D5
:10305000921B0130814610F8011B2029FAD05FFA3B
:1030600082FA4FF00008DFF854B20D235246304682
:1030700003FB08F10BEB01045BF801100091FCF776
:10308000F7F80546002857D10099084639F042FB69
:10309000824551D1267906F0E001402900F0CB802D
:1030A0000ED8002956D0202900F09D803846854949
:1030B000FEF721FB204603B0BDE8F04FFDF77BBDD6
:1030C000602900F091808029F0D1484639F022FB38
:1030D000E3790546A679DB070CD52046FBF7FCFA19
:1030E0000378014633B12A4648463BF0FCFE0028EF
:1030F00040F0D880002D00F0D580AE42C0F0D280E4
:103100000D23204603FB08B393F805A0FBF7E4FA70
:10311000324600213BF0BAFDAA452CD82A466A491E
:1031200048463BF0E0FE30B32046FBF7D5FA2A468E
:1031300049463BF037FD1EE008F1010840F22D231F
:10314000984592D132466149384603B0BDE8F04F08
:10315000FEF7D1BA06F00703042B1CD10B460A2256
:103160004846FCF7D5F8D4F80530014683429DD394
:103170002046FBF7C7FA0D23554803FB08F85BF818
:103180000810FDF7C9FC00222146384603B0BDE80F
:10319000F04FFEF7A1BA052B0FD101230A224846B2
:1031A000FCF7B6F8D4F8053001468342FFF67EAF4F
:1031B0005B4283423FF77AAFDAE74846FCF74CF9C7
:1031C000B4F80550B4F8071016F0050FAAB28BB288
:1031D00001D02AB20BB29042FFF668AF98423FF797
:1031E00065AF0146C4E765793A4A002602EBC5059A
:1031F000B246334695F8D0210092009AB24202D9E5
:10320000BAF1000F03D0002B3FF450AFB3E7D5F86D
:10321000CC1151F8260060B149460193FCF704F83F
:10322000019B30B94FF0010A31462046FBF76AFA9C
:1032300053460136E1E706F007066379013E009345
:10324000009BAB4297DD4846814610F8013B202B9E
:10325000FAD02046FBF740FA8246042E04D8DFE875
:1032600006F0031010161F004846FCF7F5F80AF8A0
:10327000050048462C213BF010FE013500F1010904
:10328000DEE74846FCF7E8F82AF81500F1E70023E6
:103290000A2200214846FCF73BF84AF82500E8E7F7
:1032A0000123F5E732460C493846FEF724FAFDE6DD
:1032B0003146384603B0BDE8F04FF3E5841B0508FE
:1032C000BFB905080DBA0508B8D80508E2B3050866
:1032D00002BA0508A8030508D2B9050828B60508EA
:1032E0002DE9F04F914689B00C461A4600218046E0
:1032F0004D46FEF75DFF00270646DFF8E0B0B9F166
:10330000000F69D02946062220463BF095FC002894
:103310003246404613BF012100214FF0010A4FF011
:10332000000AFEF745FF0646287811F0BBFE07901D
:1033300010B3687911F0B6FE079B4FF461714FF03E
:10334000190C5B79EA780793AB781CFB021295F8AD
:1033500001E01CFB0313297900B14079CDF804E0AA
:10336000CDE90232079B5A46CDE90410009351463D
:103370003B464046FDF7B8FB207811F093FE0790DE
:1033800010B3607911F08EFE079B4FF461714FF01E
:10339000190C5B79E2780793A3781CFB021294F86E
:1033A00001E01CFB0313217900B14079CDF804E062
:1033B000CDE90232079B5A46CDE9041000935146ED
:1033C0003B464046FDF748FB013706340635142FCF
:1033D00095D109B0BDE8F08FCA46CDE71BBA050804
:1033E0002DE9F041064686B008460F46FFF79CF8E7
:1033F000054638B100235C4901201A4606B0BDE8F5
:10340000F0416DE70846FCF727F81328044600F35F
:10341000A28006268DF81750544D4643781CFAF7C3
:10342000E1FF074670B1FCF717F8C0B211F050FE8B
:1034300040B1AB19027983F8D0259DF817300133DC
:103440008DF817303846FAF7CDFF074668B1FCF71C
:1034500003F80D2809D8062303FB045383F8D1058C
:103460009DF8173001338DF81730DFF8FC80B11C60
:103470000DF1170238464144FBF7F2FFFAF7B2FFAD
:10348000074668B1FBF7E8FF012809D8062303FBCC
:10349000045383F8D4059DF8173001338DF81730A5
:1034A0003846FAF79FFF80B1FBF7D6FFC0B211F0A4
:1034B0000FFE50B10623027903FB045383F8D52590
:1034C0009DF8173001338DF817309DF8172006232B
:1034D000042A2FD103FB04530022A3F8D42516F0AD
:1034E00061FA06234FF4617603FB045595F8D00585
:1034F00011F0D8FD95F8D32595F8D275192380469B
:1035000095F8D50513FB076713FB026611F0CAFD9A
:103510004379214698F80520039395F8D43514484B
:103520000097CDE9016395F8D135FDF735FB06B07D
:10353000BDE8F081052A05D103FB0453002283F87E
:10354000D525CCE7062ACAD0002308EB060248F8A6
:1035500006309380C3E713232A460649304606B057
:10356000BDE8F041FEF7D4BF6C5401209C4E012011
:103570001BBA050834BA05082DE9F04F174689B083
:103580001A460C46002181463D46FEF711FE3A4E92
:1035900007F16C038046DFF8E8B0079394F9041054
:1035A0000023364A92F90800884260D001330C3279
:1035B000092BF7D10C35079B0C349D42EED109B095
:1035C000BDE8F08F29460C2220463BF035FB002851
:1035D0004246484613BF012100214FF0010A4FF037
:1035E000000AFEF7E5FDEA7995F90430804606EB1E
:1035F000820251464846D2F8F02304922A7A06EB1A
:103600008202D2F8F0230392AA7906EB8202D2F862
:10361000F02302926A7906EB8202D2F8F02301923B
:103620002A6800925A46FDF75FFAE279514694F90A
:103630000430484606EB8202D2F8F0230492227A44
:1036400006EB8202D2F8F0230392A27906EB820203
:10365000D2F8F0230292627906EB8202D2F8F023CC
:103660000192226800925A46FDF7F6F9A2E7002F70
:10367000A8D1BA46D9E700BFA80305086C530120BA
:103680003ABA05082DE9F04707468AB00846FEF722
:103690004BFF044638B10023544901201A460AB0B2
:1036A000BDE8F04768E70DF11C0807904E1CC8E91B
:1036B00001000846FBF7D0FE4C4B40B21A4693F986
:1036C0000410814200F08A8001340C33092CF6D1B9
:1036D000002425463046FAF785FE064638B1013506
:1036E00000230A22EDB21946FBF712FE07904FF0B5
:1036F0000009DFF800A13046FAF774FE064640B331
:10370000FBF7AAFE3A49002251F804CBD3B2604538
:1037100003D00132102AF7D100230AEB8302D2F83A
:10372000F023904215D1B9F1020F1FD0B9F1030F68
:1037300021D05A1EB9F1010FD2B212D00B2A03D8F0
:103740008DF821300135EDB209F10109B9F1040F0D
:10375000D1D1052D15D838460AB0BDE8F047FDF7A0
:10376000E1BF042AF0D88DF82230EBE7052BEBD827
:103770008DF82430E6E79A1E0D2AE5D88DF823301F
:10378000E0E798E807001B4B84E807009DF823203A
:10379000002103EB82020846D2F8F02304929DF840
:1037A000242003EB8202D2F8F02303929DF822201A
:1037B00003EB8202D2F8F02302929DF8212003EB62
:1037C00082030D4AD3F8F0330193079B00939DF9D0
:1037D0002030FDF741F90AB0BDE8F0870C23012540
:1037E0008DF8200003FB042474E700BFA8520120D9
:1037F00098070508A80305083ABA05082DE9F04F0F
:103800008BB00C460021074608921A46FEF7D0FC02
:103810000026089D4FF019094FF46178DFF8A4B035
:103820000990089B002B49D029460A2220463BF0EC
:1038300003FA0028099A384613BF012100214FF0EE
:10384000010A4FF0000AFEF7B3FC2A8909903346BB
:1038500006925146EA88384605922A790492EA7817
:103860000392AA7819FB028202926A7819FB0282FB
:1038700001922A7800925A46FDF736F9228933469A
:103880000136514606923846E2880A350592227979
:103890000492E2780392A27819FB02820292627883
:1038A00019FB0282019214F80A2B00925A46FDF786
:1038B000D3F81E2EB5D10BB0BDE8F08FDDF820A0F7
:1038C000DCE700BF57BA05082DE9F04380468BB00E
:1038D00008460F46FEF728FE044638B10023654926
:1038E00001201A460BB0BDE8F04387E70846FBF716
:1038F000B3FD1D28054600F3B3800A268DF8274046
:103900004643781CFAF76EFD044630B1FBF7A4FD80
:103910009DF8273001338DF827302046564CFAF7B2
:1039200061FD074668B1FBF797FD0D2809D80A230A
:1039300003FB054383F854009DF8273001338DF8CD
:103940002730DFF83091711C0DF1270238464944C9
:10395000FBF786FDFAF746FD074668B1FBF77CFDED
:10396000222809D80A2303FB054383F857009DF852
:10397000273001338DF827303846FAF733FD0746F4
:1039800068B1FBF769FD0D2809D80A2303FB05433D
:1039900083F858009DF8273001338DF827309DF8C3
:1039A0002730062B0CD0002309EB0602404649F8CD
:1039B000063053601381FDF7B5FE0BB0BDE8F08310
:1039C0000A260023384606FB0546A6F85A30A6F814
:1039D0005C30FAF707FD074640B1FBF73DFD9DF867
:1039E0002730A6F85A0001338DF827303846FAF709
:1039F000F9FC58B1FBF730FD0A2303FB0543A3F89C
:103A00005C009DF8273001338DF827301B4B4FF0B9
:103A1000FF324FF461705A600A2202FB0542B2F88D
:103A20005C300693B2F85A30059392F858300493FC
:103A300092F857300393192392F8561013FB0101A3
:103A4000029192F8551013FB0103002101930846DF
:103A500092F854300A4A00932B46FCF7FDFFACE77E
:103A60001D232246074940460BB0BDE8F043FEF750
:103A70004FBD00BFE85F0120945F0120A00301203B
:103A800057BA050834BA05082DE9F04F804691462B
:103A90001F460C4616464FF0000BDFF820A12DED17
:103AA000088B95B094ED008AB5EE408AF1EE10FADD
:103AB0007DD0D4ED019A94ED029AD4ED038AB9F148
:103AC000000F49D0D6ED00BA96ED01BAB4EE6B8A7C
:103AD000D6ED02AA96ED03AAF1EE10FA6CD1F4EE3F
:103AE0004B9AF1EE10FA67D1B4EE6A9AF1EE10FA41
:103AF00062D1F4EE4A8AF1EE10FA0CBF01210021E6
:103B00003A460D46404681F00101FEF751FBB0EE0A
:103B10006B0A074611A8FAF771FCB0EE4B0A079042
:103B20000EA8FAF76BFCB0EE6A0A06900BA8FAF73B
:103B300065FCB0EE4A0A059008A8FAF75FFC059903
:103B4000069A079B039040460291294601925246ED
:103B500000935B46FCF7C8FFB0EE480A11A8FAF7DD
:103B60004DFCB0EE690A05460EA8FAF747FCB0EE28
:103B7000490A06900BA8FAF741FCB0EE680A0590D6
:103B800008A8FAF73BFC069B059A002103904046E3
:103B90000292524610341036CDE900535B460BF1C9
:103BA000010BFCF759FFBBF1080F7FF47BAF15B099
:103BB000BDEC088BBDE8F08F0021A1E77ABA0508BB
:103BC0002DE9F74F07460D46DFF8A8A1DFF8A8B1A9
:103BD0002846FEF7A9FC064638B100235D490120BE
:103BE0001A4603B0BDE8F04F4EE70522514628467D
:103BF000FBF73EFBA0B9584B0022C3F88021C3F865
:103C00009021C3F8A021C3F8B021C3F8C021C3F8A4
:103C1000D021C3F8E021C3F8F02103B0BDE8F08F54
:103C200004224E492846FBF723FB04462846002C75
:103C300044D1FAF7D7FB80460028EED038F06AFD71
:103C4000474BC2B253F8049BB9F1000F07D12A4683
:103C50004449384603B0BDE8F04FFDF74CBD494636
:103C600040460134CDE90023FBF702FB0646DDE9BF
:103C700000230028E6D1374A0346002115460133C8
:103C800042F8101B082BFAD10BEBC404D4F8BCC0CB
:103C9000BCF1000F03D094F8B8E0764505DB494647
:103CA0003148324DFCF778FF92E70CEB061305EB39
:103CB000061401360FCB84E80F00EEE7FBF7CCFBD0
:103CC000072804463DD82846FAF78CFB064658B329
:103CD000FAF740F9204B012503EB041383ED600A4A
:103CE0003046FAF77FFB064638B1FAF733F91A4B3C
:103CF000013503EB041383ED610A3046FAF772FBDA
:103D0000064638B1FAF726F9134B013503EB0413D5
:103D100083ED620A3046FAF765FB38B9384603B0DE
:103D2000BDE8F04FFDF7FEBC0546D9E7FAF712F9FA
:103D30000948032D00EB041484ED630A3FF44DAFF2
:103D4000ECE7072332460A49384603B0BDE8F04F96
:103D5000FEF7DEBB14610120945F01208EBA0508D6
:103D6000F4080508E2B3050893BA050866C5050816
:103D700034BA050821B70508A80305082DE9F74F4F
:103D800092460C461A46002181465646FEF710FA26
:103D900000258046DFF864B0BAF1000F2CD0314620
:103DA000042220463AF048FF00284246484613BF06
:103DB0000121002101270027FEF7FAF973888046C8
:103DC0005A46019339463AF82530484600932B4627
:103DD000FCF78AFE63885A46394648460193043602
:103DE00034F8043B00932B460135FCF735FE042DD7
:103DF000D2D103B0BDE8F08F5746EBE79DBA050876
:103E00002DE9F34105460846FEF78EFB0C460746B2
:103E100038B10023334901201A4602B0BDE8F04111
:103E2000ACE731492046FBF7FFF9034668B92D4A54
:103E30004FF47A704FF4FA610133108051800432EC
:103E4000042BF9D102B0BDE8F0812046FBF704FB5A
:103E50000328064641D82046FAF7C4FA074670B14F
:103E6000FBF7FAFA4FF0010804463846FAF7BAFAB7
:103E700048B9284602B0BDE8F041FDF753BC40F216
:103E8000EE248046F1E7FBF7E7FAB8F1000FF0D037
:103E9000A4F2EE2240F2DC539A4203D8A0F2EE22C2
:103EA0009A420AD940F6CA0340F2EE220F49284648
:103EB00002B0BDE8F041FEF72BBB0D4B00210D4ACF
:103EC00003EB8603A3F80042A3F802023346CDE9D0
:103ED00000400846FCF7C0FDB4E703233A46064914
:103EE000E5E700BF9461012021B70508AEBA0508D7
:103EF000945F01209DBA050801B705082DE9F04F30
:103F00008FB08946174600211A4606460024FEF760
:103F10004FF90DF1240B0546DFF86CA059F8243059
:103F2000594602A8029332F0D3FD57B357F8243014
:103F30003046029A039393422A4613BF012100217F
:103F40004FF001084FF00008FEF732F904A90546CA
:103F500003A832F0BDFD04A9234652460091304625
:103F60004146FCF7C1FD23460134524641463046E6
:103F7000CDF800B0FCF770FD202CCFD10FB0BDE81C
:103F8000F08FB846EFE700BFBCBA0508F0B50746AA
:103F900089B008460E46FEF7C7FA054638B1002339
:103FA000194901201A4609B0BDE8F040A6E70846C5
:103FB000FBF752FA1F2804461DD83046FAF712FACA
:103FC0000146204629F0A0F978B103AE0E483146EB
:103FD00000EB840032F07CFD23460C4A294628463B
:103FE0000096FCF739FD09B0F0BD384609B0BDE8D0
:103FF000F040FEF781B91F232A460549384609B02B
:10400000BDE8F040FEF784BAA4610120BCBA0508FF
:1040100034BA05082DE9F04F924685B00C461A4691
:10402000002181465546FEF7C3F800268046DFF89A
:104030006CB0BAF1000F2FD02946042220463AF086
:10404000FBFD00284246484613BF012100210127FD
:104050000027FEF7ADF8EB7880465A4602933946C2
:10406000AB78484601932B8800933346FCF73CFD20
:10407000E3785A463946484602930435A3780193BB
:1040800034F8043B009333460136FCF7E5FC102E70
:10409000CFD105B0BDE8F08F5746E9E7C6BA0508AD
:1040A000F0B5074685B008460E46FEF73DFA0546D0
:1040B00038B100231C4901201A4605B0BDE8F04084
:1040C000A8E70846FBF7C8F90F28044623DC30466A
:1040D000FAF788F90146204629F08EF8A8B104F1D4
:1040E0002002124B2946284603EB820393F8132241
:1040F000029293F812220192B3F810320C4A009304
:104100002346FCF7A9FC05B0F0BD384605B0BDE874
:10411000F040FEF7F1B80F232A460649384605B0AD
:10412000BDE8F040FEF7F4B924620120945F01205D
:10413000C6BA050834BA05082DE9F04F87B0144611
:104140001A46054603910021FEF732F84FF00008A9
:104150000646DFF820B106234FF0000903FB08F7FD
:10416000C037039BDB5D0493002C7FD0E35D2846C2
:10417000049A05939A42324613BF012100214FF061
:10418000010A4FF0000AFEF713F8059B06465A464F
:1041900051462846CDE900934346FCF7A5FC049B15
:1041A0005A46514628460137CDE9009309F10109E5
:1041B0004346FCF751FCB9F1060FD2D108F10108D2
:1041C000B8F1060FC7D1E427DFF8A8B0039BA7F129
:1041D000E40913F807A0002C4AD0E35D32462846D4
:1041E0009A45049313BF012100214FF001084FF0BD
:1041F0000008FDF7DDFF049B06465A464146284667
:10420000CDE900930623FCF76FFC01370623194A1A
:1042100041462846CDE9009AFCF71EFCEF2FD5D188
:10422000039B93F8EF70ACB194F8EF8032462846C8
:10423000474513BF0121002101240024FDF7B8FFE9
:1042400000230C4A2146009328460723CDF804801A
:10425000FCF74AFC0023074A21462846009307231F
:104260000197FCF7F9FB07B0BDE8F08FA24696E78F
:10427000A046CAE7D8BA0508F0B5054687B0084693
:104280000B46FEF751F9044638B100231C490120C2
:104290001A4607B0BDE8F0404EE703AE194F02AA38
:1042A000184918463AF0B4FCB8B1032C04D128469A
:1042B000FDF738FA07B0F0BDFBF7CEF802AA46F8D2
:1042C000040B3946002001343AF0A2FCECE73246F8
:1042D00021460D48FCF760FCECE7032CE7D1059B79
:1042E000DDE903461A4601933146E0B228F0CEFFDD
:1042F000019B0028EBD12846FDF7FEFFDAE700BF5F
:10430000A46101202BAC0508D8BA05082DE9F04FAF
:1043100089B000260C46002107921A460746B2468D
:10432000FDF746FF4FF01909079D4FF46178DFF85C
:1043300094B00690079B3BB32946062220463AF0EC
:104340007BFC0028069A384613BF012100214FF05C
:10435000010A4FF0000AFDF72BFF6A7906903346F9
:1043600019FB02825146384605922A7919FB0282CE
:104370000492EA780392AA7802926A7801922A78E3
:1043800000925A46FCF7B0FB62793346013651463B
:1043900019FB0282384606350592227919FB028202
:1043A0000492E2780392A27802926278019214F861
:1043B000062B00925A46FCF74FFB0A2EBAD109B0E1
:1043C000BDE8F08FECBA05082DE9F04F074689B03B
:1043D00008468B46FEF7A8F8044638B10023544936
:1043E00001201A4609B0BDE8F04F8FE7514B08464F
:1043F00093F8F0A693F8F19693F8DA87FBF72CF888
:104400000928054600F38B8006268DF81F404A4C8C
:1044100046430BF10100F9F7E5FF834658B1FBF77E
:104420001BF80D2807D8A31983F800039DF81F3047
:1044300001338DF81F305846F9F7D4FF834668B131
:10444000FBF70AF8824509D3062303FB054383F8EB
:1044500001039DF81F3001338DF81F305846F9F7DE
:10446000C1FF824668B1FAF7F7FF484509D806232D
:1044700003FB054383F802039DF81F3001338DF8D9
:104480001F305046F9F7AEFF814668B1FAF7E4FFF6
:10449000804509D3062303FB054383F803039DF8F6
:1044A0001F3001338DF81F30DFF88480311D0DF18E
:1044B0001F0248464144FAF7D3FF9DF81F20062A01
:1044C0000BD0002308EB0602384648F806309380EC
:1044D000FDF728F909B0BDE8F08F02FB05424FF463
:1044E0006170192392F8051313FB0101059192F8ED
:1044F000041313FB010300210493084692F80333CD
:10450000039392F80233029392F80133019392F8E5
:1045100000330A4A00932B46FCF79EFADAE7092398
:1045200022460749384609B0BDE8F04FFDF7F0BF15
:10453000946201209C4E0120945F0120ECBA050892
:1045400034BA05082DE9F04F144689B00F461A46D3
:1045500000210646FDF72CFE0546002C00F0D58014
:1045600022783B789A42024630460DBF4FF0010850
:104570004FF0000801210021FDF71AFE23780546BF
:10458000994A41463046FCF7AFFA3B784146964A95
:104590003046FCF761FA002C00F0B98062783046B2
:1045A0007B789A422A460DBF4FF001084FF0000871
:1045B00001210021FDF7FCFD637805468B4A414649
:1045C0003046FCF791FA7B784146884A3046FCF742
:1045D00043FA07F1CA0304F1CA0B4FF0020904932E
:1045E0004FF0000A822305933B78534500F39180F6
:1045F000002C00F0F28097F8EA30304694F8EA2078
:104600009A422A460DBF4FF001084FF000080121E1
:104610000021FDF7CDFD94F8EA300546744A414685
:104620003046FCF761FA97F8EA304146704A304666
:1046300007F1EC09FCF710FA002C00F0D08004F12F
:10464000EC034A4604F1FC014FF001089A4633F8A6
:1046500002CB32F8020B844518BF4FF000088B42A2
:10466000F5D188F001012A463046C9B2FDF7A0FD18
:10467000082105465046FAF739FD5E4A0346414691
:104680003046FCF731FA97F8EA104846FAF72EFD63
:10469000584A034641463046FCF7DEF9002C00F04C
:1046A000A0804FF0FC094FF0010807EB090104EB73
:1046B0000900FAF7B9FD09F10409002818BF4FF005
:1046C0000008B9F58E7FF0D188F001012A46304606
:1046D000C9B2FDF76DFD082104F1FC00F9F722FFD6
:1046E000454A034641463046FCF7FEF997F8EA1082
:1046F00007F1FC00F9F716FF3F4A034641463046F2
:1047000009B0BDE8F04FFCF7A7B9A0463DE7A046C9
:1047100059E7059B3B440693002C5CD0059B06980B
:10472000234419460793FAF77FFD049B1A789BF8F8
:1047300000309A424CD1B0FA80F84FEA58184B46F4
:1047400009F11002F85AE15A0233884218BF4FF0BB
:1047500000089342F6D188F001012A463046C9B2DA
:10476000FDF726FD627804EB090105469BF8180069
:10477000FAF78EFC02909BF8003041461F4A304603
:104780000193079B00930AF10103FCF7ADF9049B29
:1047900007EB09017A780AF1010A187E0BF1010B87
:1047A0000793FAF775FC079B4146049A09F1100933
:1047B000029030461B7801320193069B04920093CD
:1047C00053460E4AFCF748F9059B093305930BE75E
:1047D0004FF00008B3E7A046D9E7A04623E7A0467C
:1047E00051E7A04682E700BF05BB050817BB0508D7
:1047F00045BB05085DBB050874BB05082CBB050857
:104800002DE9F04F8FB004460846B04902AA3AF0AD
:10481000FFF9064640B903460246AD494120FFF77D
:1048200091FE0FB0BDE8F08FAA49FAF7FDFC0746EC
:1048300020BB02AAA5493AF0EBF9FAF70DFE0828C9
:10484000054606D908233A46A3492046FDF760FEEF
:10485000E7E7A24C94F8F036834202DC84F8F05685
:10486000DFE7064604F5DE673146384621F088FC6E
:10487000013694F8F036B342F6DCEFE7984930465B
:10488000FAF7D2FC0546E0B902AA90493AF0C0F91D
:10489000FAF7E2FD0828064603D908232A4691497B
:1048A000D3E78E4C94F8F136834202DC84F8F1664B
:1048B000B7E728460135314632F0E2F8082DF8D145
:1048C000F4E789493046FAF7AFFC074600BB02AA75
:1048D0007E493AF09DF90028A3D0FAF7BDFD0828DB
:1048E000054603D908233A468049AEE77B4C94F845
:1048F000DA37834209DD014604F5DE6021F08AFCE7
:10490000294604F5DE6021F093FC84F8DA5788E745
:1049100077493046FAF788FC054618BB06AE6F4B60
:10492000DFF8A8910146B0461022304693F8DA77B6
:104930003AF0ACF9BD4202AA80F20E81494600204D
:104940003AF066F910B93A466A490EE1FAF784FD81
:10495000013528F8020BEDE7674C96E80F0084E874
:104960000F005EE765493046FAF75EFC0546002811
:104970003BD15A4B0DF11808074693F8DA97464693
:104980004F4502AA51494FF0000080F2F2803AF000
:104990003FF9014610B94A465949E6E0B2464FF0A0
:1049A000000B032230463AF0B2FA304637F0B2FE3E
:1049B000584502D801370436E2E79AF800000BF1B7
:1049C000010BFAF72BFC0AF8010BEEE74A464D49BA
:1049D000CBE0414620460135043408F104080322A7
:1049E00021F0B8FBAF42F4D11BE747493046FAF754
:1049F0001BFC0546002840F0AC80384F02AA334922
:104A000097F8F0863AF004F900283FF40AAFFAF775
:104A100023FD461E01D4B04503DC434601223B4939
:104A200013E72A4902AA00203AF0F2F801460028CA
:104A30003FF4F7AE4FF000080DF10C09082203A86F
:104A40008DF81480CDE903883AF061FA03A837F0B5
:104A500061FE40451CD802AA1C4900203AF0D8F853
:104A600000283FF4DEAE90F800A04FF0000897F861
:104A7000F196DFF8A8B04D4502AA14494FF00000A6
:104A80007EDA3AF0C5F8024658B94A4620496CE049
:104A900099F8000008F10108FAF7C0FB09F8010BCA
:104AA000D4E7002D40D11378303B092B3CD919496C
:104AB0000192FAF7B9FB019A90B310465946FAF7FA
:104AC000B3FB019A002838D013494EE02BAC0508FF
:104AD0008C5501208BBB050891BB05089C4E01201D
:104AE0009CBB0508A5BB0508B3BB0508BFBB0508F3
:104AF000D1BB0508C0BC050878560120FBBB0508E2
:104B0000E0BC050807BC050825BC05082ABC05084B
:104B100000BD0508FEAB05083DBC050836BC050810
:104B20004FF001084FF0FF3510460192FAF794FC60
:104B30000028019A03DA214917E0A846F2E70EABF4
:104B400003EB4503013523F8200C94E74A461C4942
:104B50000BE032461B4908E01B4900203AF058F8A8
:104B600000283FF4F9AE3A4618492046FCF7C3FD49
:104B700057E63AF04DF800287FF428AF144C31E79F
:104B80003AF046F80028E1D106EBC600114C0822A5
:104B900003A982303744204421F0DCFA5046FAF76A
:104BA0003DFB87F8BA0704EB061006A96A0002303D
:104BB00039F0F8FF87F8D28733E600BF72BC0508EA
:104BC00087BC0508AABC05082BAC0508DDBB050899
:104BD000885601208C5501202DE9F04F0F46914653
:104BE00089B0002187EA09099846139A06460025EC
:104BF000FDF7DEFA6FEA09030446DFF880900693BA
:104C000028460CF08BFF129B184230D0069BDFF831
:104C100070B0034014BF4FF0010A4FF0000A049334
:104C200010EA0703284614BF4A465A4605930792DE
:104C30000CF086FF4346079A514603900090304699
:104C4000FBF752FF049B22463046B3FA83F1490931
:104C5000FDF7AEFA039B059A04460093514643467E
:104C6000002A14BF5A464A463046FBF7F5FE013586
:104C7000182DC5D109B0BDE8F08F00BF88BA05086E
:104C800025BD050837B504460846019137F042FDB9
:104C90000199054602462046FAF7EAFA70B9625DC4
:104CA0001046FAF7A5FA00B932B901352C4420466E
:104CB00001340378202BFAD003B030BD0020FBE78D
:104CC0000329F0B5054685B00C46164614D80B4F9F
:104CD0003970FBF7BDFE0A492846FEF783F82246E5
:104CE000084901A8FAF77AF901AB324608212846AB
:104CF000FDF78CFAFF233B7005B0F0BDA003012047
:104D000066C5050884B905080329F0B5054685B0D0
:104D10000C46164614D80B4F7970FBF799FE0A49DA
:104D20002846FEF78FF8224608496846FAF756F9F2
:104D30006B46324610212846FDF768FAFF237B7048
:104D400005B0F0BDA003012066C5050880B90508BF
:104D500010B5114B86B0114904460493104B11480D
:104D60000393114B114A0293114B0193114B009382
:104D7000114BFBF7D1FEFBF76BFE10491048FBF718
:104D80000BFF3CB10F4A1049104806B0BDE8104077
:104D9000FBF702BF06B010BD6CBD050836BD0508A7
:104DA00071BD050841BD05087BBD05082CBD050882
:104DB00084BD050817AF0508AB4E012090BD05085E
:104DC00098BD0508646B05085C6B0508A9BD05085E
:104DD0000120BDE72DE9F04F3E4C87B00A46002187
:104DE0000646FDF7E5F905903B4A2378608802EB1B
:104DF0008303D3F8E4A7F9F759FC8368C1680493E7
:104E0000364B93F86420002A4BD0DDF810800491D3
:104E1000002721796279049B07FB012213F8029095
:104E2000B8F1000F3FD018F802504D45059A3046B2
:104E300007F1010713BF012100214FF0010B4FF0D3
:104E4000000BFDF7B5F905907DB305F00F022D09B4
:104E500053465946403502923046214ACDE9007505
:104E6000FBF742FEB9F1000F2AD009F00F024FEA1A
:104E7000191953465946029209F140023046CDE9CC
:104E80000072174AFBF7E8FDA279012A38BF012218
:104E9000BA42BEDC0834134BA342A5D107B0BDE82B
:104EA000F08F9046B4E74546BFE7B8F1000FD9D080
:104EB00053460D4A594630460097FBF715FED1E799
:104EC0007306E1D45346084A594630460097FBF72B
:104ED000C3FDD9E79C0A0508A80305089C4E0120DC
:104EE000D6BD05088C0B0508ECBD050838B50C4B84
:104EF0000C4603EBC0050B4895F8F42603EB820340
:104F0000D3F8E417FBF708FE95F8FA3633B1611CC5
:104F10000548C9B2BDE83840FBF7FEBD38BD00BF4B
:104F2000A8030508F1C005089DAC050873B50E4639
:104F300011490546FAF778F918B93070012002B026
:104F400070BD2C78602C8CBF613C413C072C10D884
:104F5000013501230A2201A92846FAF7D9F9019B54
:104F60009D4206D00F2804D8013440EA041434705E
:104F7000E4E70020E3E700BF98AB05082DE9F04F18
:104F8000714D0A460021824605F1800B2DED028B02
:104F90008BB0FDF70DF9814600266C4B93F8644009
:104FA000AB7AB34200F393801035AB45F4D140F2B5
:104FB0001620F9F77BFBD0E902530CB12C461D46B5
:104FC0000DF1100B002715220021584639F05EFE26
:104FD0002E78002E43D069783046039105F034FFD7
:104FE00095F9023008EE100A5A1C029353425341BD
:104FF000002C00F0A6800022039914F802C0A0182B
:10500000B44540F09A8090F90280029A424540F0FF
:10501000928042788A4208BF0123012203F00103F3
:105020000BF807204A4683F0010150460393FDF731
:10503000BFF8039B81464CB1454A18EE101A304622
:10504000CDE900A24246F9F7EDFA039B414A18EE7A
:10505000101A3046CDE900A2029AF9F7E3FA0137B7
:105060000335152FB4D16CB304F13F06384FDFF888
:10507000E4801BF8013B02930BBB2078F8B194F954
:10508000022001321BD0617805F0DEFE05464A465B
:1050900001215046FDF78CF894F90220029B294625
:1050A00081462078CDE900A7F9F7BCFA2078029B69
:1050B0004FF0FF322946CDE900A8F9F7B3FA0334DF
:1050C000B442D6D10BB0BDEC028BBDE8F08FE888BE
:1050D000F9F7ECFAD0E902230CB114461A46297A02
:1050E0006B7A06FB013312F903800CB3E756B8451F
:1050F0004A4650460DBF012300230121002102939F
:10510000FDF756F8029B814644B1114A31462846C4
:10511000CDE900A23A46F9F739FA029B0D4A314629
:1051200028460136CDE900A24246F9F72FFA34E7C6
:105130004FF0FF37DBE700236FE703323F2A7FF4AE
:105140005CAF4FF0FF386DE7B80301209C4E0120A3
:10515000E90A0108590A01082DE9F04F80468BB091
:1051600008460D4637F0D6FA024670B3A5492846E0
:10517000FAF77EF8044640BBFBF76AFCA24DA34851
:10518000A34FFBF77DFCA34E1420DFF8D48231F04F
:105190008BFCE11004F0070238460131FBF7BCFC40
:1051A0002B7F6A7F06EB8303D3F8E4174AB19A4852
:1051B000FBF7F2FC01342435102CEAD10BB0BDE82A
:1051C000F08F4046FBF7E8FCF4E7284605AA934930
:1051D00039F01EFD054620B901464120FFF7CEFEFD
:1051E000ECE78F49FAF720F820B98E494046FCF7E2
:1051F00082FAE3E78C4E0827002431682846FAF744
:1052000013F8002808BF3446013F06F11006F4D118
:1052100054B986492846FAF707F828B12A4684493E
:105220004046FCF768FAC9E7002005AA7B498DF8DB
:10523000130039F0EDFC0646002C3BD080B1FAF7A4
:105240000BF9451E09D4A37A9D4206DAE2684AB1F9
:10525000012303FA00F0104204D132467549DFE71A
:10526000754EFAE7E0880027F9F720FA73490397AB
:1052700091F86410D0E90232002908BF1A46217A59
:10528000637A05FB013302EB030B12F903A005AAB5
:105290006249002039F0BCFC8146A0BB012368496B
:1052A00044B39BF900202046CDE900312946F9F7A7
:1052B0006DF983E768B10DF11301FFF737FE28B1EF
:1052C0009DF81350284601F06DFF20B932465D4924
:1052D000A6E7594EFAE72846A346F4F7A9FD824609
:1052E000284605F09DFD03902846254606F062FA03
:1052F0000746CCE7CDE90031524639469DF8130008
:10530000F9F790F95AE74649F9F78EFF064658BB78
:10531000ACB1EDB24C4F72B229462079F4F75CFD86
:1053200000283FF44BAF02883146037838460136F7
:105330000093C2F30323120BFBF72EFCEBE7424C66
:1053400072B279793868F4F78FFD00283FF436AFF0
:10535000028831460378204601360093C2F30323C6
:10536000120BFBF719FCEBE738494846F9F75CFFED
:1053700010B34846FAF770F8064642B26CB1E9B28B
:105380002079F4F729FDC8B9CDF800906B1C22688C
:105390002F494046FCF7AFF910E779793868F4F700
:1053A00063FD58B99DF813302A491A09CDF80090C9
:1053B00003F00F034032ECE74FF0FF3606AF304604
:1053C0003946F9F7C5FE08A95046F9F7C1FE56451A
:1053D00048D076B24CB18BF8006008AB00976A1CDD
:1053E00021681D48FBF7D8FBE8E69DF81320039BD6
:1053F00011091A489E7002F00F0208AB4031009765
:10540000F0E700BF00BE05088000012005BE0508CA
:105410001BBE0508A80305089CC305082BAC05089E
:10542000E6B005082CBE0508B803012040BE0508FB
:1054300044BE050853BE050866C505089C4E0120FC
:10544000590A010863BE050875BE05081CB40508A5
:1054500096BE0508B9BE0508E1BE050804BF0508EB
:105460005DB0050834B108AB6A1C21680648FBF73B
:1054700093FBA3E69DF8132008AB0448110902F042
:105480000F024031F3E700BF2CBF050847BF0508F6
:10549000224BB0F5FA6F1A680346A8BF4FF4FA63BF
:1054A000B3F57A7FB8BF4FF47A73D20416D540F2C1
:1054B000DC52904215D040F2DB5207EE903A904217
:1054C000F8EE677A1FD8DFED166A9FED167A77EE51
:1054D000E67A9FED150AA7EE870A7047B0F57A7F46
:1054E00002D89FED120A704707EE903ADFED106A7E
:1054F0009FED107AF8EE677A9FED0F0A77EEE67A65
:10550000A7EE870A7047DFED0D6A9FED0D7A77EE03
:10551000E67A9FED0C0AA7EE870A7047DC5301205C
:1055200000007A44D62000C000E082440000000061
:1055300000407A44661000400000404200A0BB4496
:10554000D62000400000834410B584464FEA810E07
:10555000102312F4004F4FEA420214BF0E24072416
:10556000013B92B2CCF80040F444F2D100EB81123E
:105570008C010351122042F8213010BD10B5844631
:105580004FEA810E0424130B013C4FEA021203EB95
:10559000430392B203F11803CCF80030F444F2D183
:1055A00000EB01130A018450062043F8214010BD8E
:1055B000704700BF704700BF034B00EB400003EB98
:1055C000C000407C704700BF3C07002000231D2125
:1055D0001E22017042708370C3707047704700BF15
:1055E00000207047704700BF0020704701207047BF
:1055F000704700BF704700BF704700BF704700BFD3
:105600009FED010A704700BF0000000000207047B6
:1056100003681B691847094B002230B593F9004015
:1056200001325D7804330119062ACD7213F8025C49
:10563000055513F8014C8C75F0D130BDD0370508F5
:10564000002383700370C37043707047D0F8FC3040
:105650004BB1D0F88C31D0F814211B685B689A42AA
:1056600005D3D01A7047D0E907239A42F9D2C0680F
:105670001044C01A704700BFD0E9091291420ED3FE
:105680008A1AD0F80011036981B1D0F88811013B62
:10569000096849680A4493420BD9981A704703690C
:1056A00019448A1AD0F800110029EED1013B981A4A
:1056B00070470020704700BFD0F8003113B190F858
:1056C000A4017047D0E90903181AB0FA80F0400924
:1056D000704700BFD0F8FC20034610B472B1D0F878
:1056E0001421C1685C69881A013A205C08BF0A4627
:1056F0005DF8044BC0B2C3F814217047006A5C69BE
:10570000411C205CDC68C0B2A14238BF0A465DF88B
:10571000044B1A62704700BFD0F8A83103B1184794
:10572000704700BFF8B590F8BD31012B1CD0002A9E
:10573000164619DD05460F460269436AD41AA86960
:105740003946B4421844A8BF34462246361B39F0C5
:1057500029FA686A2A6927440444002EB4FBF2F34C
:1057600002FB13436B62E9DCF8BD00BF70B5094C66
:10577000236873B10546002606E099681A681E730F
:1057800021609047236823B15A681846AA1A002A54
:10579000F3DA70BDE873012070B5204C2378012B3B
:1057A00000D070BD1E4B1B68002BFAD01D4D2B681E
:1057B00028465B6898470028F3D01B4B1B4E1A689D
:1057C000338892889A4219D31949002228460968D9
:1057D0004968EA622A6803FB01F1D3689847338875
:1057E000144A013352683380002ADAD01168938852
:1057F0004A69134218BF1B048B6170BD0D4B002218
:105800005B682270002BCCD00B491A6809789B8802
:10581000890748BF1B04936170BD00BF9827012012
:10582000BC1A0120C01A01209027012096270120D0
:1058300088270120FC1A0120081B012008B5294BEC
:105840001B68DB041ED5B5EE400AF1EE10FA26D037
:10585000DFED257AB4EEE70AF1EE10FA1FD49FEDE2
:10586000237AB4EEC70AF1EE10FA2AD870EE677AFE
:105870009FED1F7A9FED1F0AA7EE870A38F01AFCEA
:1058800080B208BDDFED187AB4EEE70AF1EE10FA47
:105890000BDA9FED190A38F00DFC80B208BD9FEDC0
:1058A000170A38F007FC80B208BD70EE677A9FEDEA
:1058B000147A9FED140AA7EE870A38F0FBFB80B23A
:1058C00008BDDFED117ADFED116A70EE677A9FEDAA
:1058D000107AA7EEA67AB0EE470A38F0EBFB80B25A
:1058E00008BD00BFDC5301200000404200E08244BC
:1058F00066BEFFBE0060BB4400007A440080BB442B
:1059000038DFFF3E00407A440000834466BEFF3E1D
:1059100000A0BB446D4B1B782DE9F04F87B0002BE6
:1059200000F0CE806A4D4FF000086A48A968FBF786
:1059300033F969686848FBF72FF9684B6848DFF866
:10594000D8A1D3E90031C91A664B1A68B1FBF2F24B
:10595000FBF722F9FBF77CF86348FBF791F8634803
:10596000FBF78EF8624B5FFA88F41B78A34221D8CC
:10597000604C0025604FFBF76BF82646013556F862
:10598000041B3846FBF7C8F8162DF7D101255A4EEF
:10599000FBF75EF823466168013530461B68043426
:1059A000C91AFBF7B9F8162DF4D107B0BDE8F04FCE
:1059B000FBF74EB8514B14264FF03C0B671C03EB22
:1059C000840306FB045693ED000A38F073FB96F847
:1059D0001EE081B2B6F80E901EF0010F80B214BF27
:1059E00052222D221EF0020F0490504614BF542361
:1059F0002D231EF0040F07EE903A14BF56232D23DB
:105A00001EF0080F009317EE903A14BF4FF0430CAE
:105A10004FF02D0C1EF0800FCDF804C014BF4FF0D6
:105A2000530E4FF02D0EB1FBFBF10591642101FBEC
:105A300009F1CDE902E13946FBF76EF8B37FDB07E8
:105A40003AD55C232E4A6343D118D05891ED010A10
:105A500070B1B8EE400ADFED2B7A20EE270A07EE90
:105A6000900AF8EE677A80EE270A38F023FB00B23E
:105A7000642290FBF2F102FB11022348FBF74CF881
:105A80001421224808F1010801FB075701FB0454C7
:105A9000F988628A0491218B02F003039208039132
:105AA000E18A0291A18B0191A18A009119214B43B6
:105AB000218AFBF771F855E71548FAF7A9FFDFE7E8
:105AC000144807B0BDE8F04FFAF7DABFC80100206C
:105AD000FC0C002068BF050878BF0508D41600201C
:105AE0008FBF0508141C0120BCBF050818C005089D
:105AF0001C250020A80D0020C8C005084456002021
:105B0000040E002000401C4691C00508A6C00508F0
:105B10009DC00508CCC0050874C005082DE9F84FE4
:105B200006460C461E4D37274FF00008DFF87890E8
:105B3000DFF878A02046FCF7F7FCD5F800B048B9AC
:105B400021465846F9F7B8FB20B921466868F9F7AD
:105B5000B3FB80B15846FAF75BFF696811B1504654
:105B6000FAF7DAFFA96811B14846FAF7D5FF4FF006
:105B70000108FAF76DFF013F05F11005DAD1204663
:105B8000FCF7D2FC48B9B8F1000F06D122463046E6
:105B90000449BDE8F84FFBF7AEBDBDE8F88F00BF84
:105BA000E8370508F4C00508EEC00508E8C0050898
:105BB00070B504680546236A1B6943B1236AD0F8AF
:105BC00094001B69984701282AD002280DD0236A27
:105BD000DA699AB9586958B399692162BDE8704089
:105BE000C3E9052239F0ECB92362236ADA69143378
:105BF000002AF9D1236ADA69002AEBD0216A14332A
:105C000094F824200E7B2362F6B2DAB996B92846BE
:105C1000F4F73AF828460121BDE87040F3F7B4BF25
:105C2000236A01462846143B2362F3F7ADFFCEE713
:105C3000206270BDAB68002BE9D09A881968120405
:105C40008A61E4E700212846F3F79EFF002384F8E9
:105C50002430002EDBD0EDE738B58569002D3DD02E
:105C60002C68236A1B7B5BBB204636F0F5FC236A5D
:105C70005B680BB3236A5A68236A22F01F025B68D1
:105C8000216A886803F01F0100F11F03194421F005
:105C90001F01BFF34F8F00290ADD02F120031144D9
:105CA0000F488B42C0F85C221A4603F12003F8D15A
:105CB000BFF34F8FBFF36F8F2846BDE8384077E7BB
:105CC000AB68002BD0D01A6820469B88936136F0D1
:105CD000C3FC236A5B68002BCCD1EDE738BD00BF65
:105CE00000ED00E038B5846904B938BD2568284660
:105CF00036F0B2FC2B6A1B7B1BB92046BDE838404E
:105D000056E7A368002BF8D01A6820469B88936159
:105D1000BDE838404CE700BF8160F5F7C7BE00BF63
:105D20000171F5F7C3BE00BF38B5D0F8A8310446FD
:105D30000D460BB19847B8B1636AA269D554636A3E
:105D400021690133D4F800218B4228BF002363620C
:105D500022B12046BDE83840F6F75AB8D4F82021E1
:105D6000136843F08003136038BD00BF90F8BD2175
:105D7000012A0AD0D0F800210AB1F6F749B8D0F8C4
:105D80002021136843F08003136070472DE9F84F1A
:105D9000AD4C80462379DB072DED028B6BD5AB4BE9
:105DA0006579AB4E1F88012D56D0022D35D0002DC0
:105DB0003ED094ED068AF37B33B1B38923B1A54B72
:105DC0001B78002B40F0CB80A279337A632B06D866
:105DD000022D00F0DD80217C002940F0ED8095420D
:105DE0009D4BB0EE487ADFED9D6A38BF1546B27B19
:105DF0001D70D4E90A31E3625B1A07FB03F307EE77
:105E0000903AF8EEE77AA7EEA67A84ED067A002AB1
:105E10005FD1BDEC028BBDE8F88F6389BB42C8D26D
:105E20008F4B012594ED068A1B686571E361C2E71B
:105E3000A389BB4219D38A4BE1691A68F37D521AD0
:105E400003EB830303EB8303B2EB830FB1DB012589
:105E500094ED068A6571AEE7E389BB4280F08680E7
:105E60002389BB4201D2002565717D4B94ED068AE2
:105E70001B68E3619FE76579DFF8D091EB1E012B8A
:105E800032D9B9F80800C0F30B0037F06FF90928D0
:105E900040F3A7806E4EB9F80070F3889F4203D399
:105EA0003288BA42BFF47FAFB7EB430F3FF77BAF07
:105EB0000323DFED6C7A674A6371B0EE678AA371E2
:105EC0000023C4ED067A137023816381A381E381EB
:105ED0007EE0012D7ED0022D9BD10720BDEC028BF0
:105EE000BDE8F84F0EF0ECB8594EB9F80070F388E1
:105EF0009F4202D33288BA4202D2B7EB430F63DD2E
:105F0000B9F80800C0F30B0037F030F9092873DD49
:105F10000022357D6271A271002D70D04D4B1D7035
:105F20002B46154699B2B288738812FB01F213FB17
:105F300001F3717C92B29BB28A422281638140F26A
:105F4000B980521A92B28B42A28140F2B1805B1AA0
:105F50009BB2E381642363740023636123E711F040
:105F600091FA002841D10222A2712EE73C4BE1694F
:105F70001A68337E521A03EB830303EB8303B2EBFD
:105F8000830FFFF616AF022594ED068A657112E7BE
:105F9000207C88B90121C4F8148080462174C3F1A3
:105FA0006403314908FB03F381FB0301DB17A3EB17
:105FB000A1536433637412E760692C49A8EB0008AD
:105FC0008845ECDB63740AE7032D7AD194ED068AE9
:105FD0000325F0E6BDEC028B0820BDE8F84F0EF07B
:105FE0006FB8B9F800701A4EDDE6337C83422CBFDF
:105FF00001220022A271E8E6032DE7D0D9E632881B
:106000001B4BDFF850A01B68B7FBF2F2013293F98B
:106010006C10082A28BF0822D3B28AF80030002961
:1060200080D091423FF47EAF124991F800E00EF12A
:10603000010101F003018E453FF474AF4FF0FF3CC6
:106040004FF0A40B22E000BFE8730120FC5E0120AA
:10605000E0530120FB5E0120FA5E0120ACC527372A
:10606000F41A0120000000006BCA5F6B8096980054
:106070009C520120A44E012018B93CEA2C0C28BFE8
:106080008C46013101F003018E4515D012480BFBFF
:10609000010090F96C008242EED18C465FFA8CF0E0
:1060A000FAF75CF99AF80030B9F80070657939E7C9
:1060B00000234EE7002246E7BCF1FF3F3FF432AF3A
:1060C000ECE7B9F80800C0F30B0037F04FF80928E7
:1060D0003FF7E1AE6DE600BFDC4F01202DE9F04750
:1060E000694CA36820469847002869D0B4F90E305F
:1060F00004F14805A17D06EE903AB4F91030092963
:1061000007EE103AB4F91230F8EEE66A07EE903A6C
:10611000B8EEC77A4FF00103F8EEE77AC4ED126AE1
:1061200084F8543084ED137AC4ED147A4AD0574F72
:10613000284619F033FDBB8D002B4CD1544B1B6806
:106140005B0770D4BB6AD4ED127AB3F90220D4EDA8
:10615000135A06EE102AB3F90420B3F9003007EE03
:10616000102AB8EEC66A00EE103AD4ED146AB8EE02
:10617000C77A484DB8EEC00A3B8835EEC66A464E2F
:1061800036EEC77A05F1080837EEC00A84ED136AC7
:1061900084ED147A84ED120A53B9A84506F10C0671
:1061A00005ED010A0CD03B88B5EC010A002BF4D0B8
:1061B00030460C3638F0ECFEA84505ED010AF2D168
:1061C000BDE8F087314F04F12001284619F0AAFC00
:1061D000BB8D002BB2D0D7F828C02846DFED2F6A40
:1061E00000252F49ACF102020CF10406B3F5C87F7B
:1061F0001CD0D1ED007AB8EEE77AD0ED007AE0EC71
:10620000016A77EE877AFDEEE77AE1EC017A22F80F
:10621000025FB242EAD1012B0CD0013BBB851C4B83
:106220001B685B078ED530F043FB8BE7B0EE667AD8
:106230000D60E2E71B48DFF874E0816BB4F80C8076
:10624000C831194E8EFB01A9C917D0E90C20C1EB4A
:10625000E911C832C830A1EB0801ACF804108EFB7C
:106260000281D217C2EBE112ACF800208EFB002EA7
:10627000C017C0EBEE10ACF80200B581F581738158
:10628000FAF738FABB8DC8E7AC2600207826002044
:10629000DC530120F82600207C26002000000000AE
:1062A00018740120E8730120185401201F85EB5158
:1062B00038B5074C074DAC4203D3074B01221A7087
:1062C00038BDA288D4E9021038F06CFC1C34F2E727
:1062D000B82A0608B4320608004F0120224B30B518
:1062E00083B09A7901906AB393F82630DFED1F6A84
:1062F00007EE903A1E4B1F4CF8EEE77A1D7886EEBB
:10630000A77A84ED187ADDB11B4BDDED017AB3F885
:106310004630F8EE670ADFED197A00EE103A60EECB
:10632000A70AB8EE400AF8F765FA04F12003002145
:1063300003EBC5021960083303ED010A9A42F9D153
:1063400003B030BD0E4A12681201F9D593F8263019
:10635000DFED066A07EE903A064BF8EEE77A86EE36
:10636000A77A83ED187AEBE7D823012055555540DD
:106370001C25002044560020E8730120BD378635D7
:10638000DC530120A54B1B78002B00F0B2802DE9D7
:10639000F04FA34D83B095F80491B9F1010F02D0ED
:1063A00003B0BDE8F08F9F4B9F4C1B6893F834708F
:1063B000002F6ED09D4B0022DFED9D6AA64694ED26
:1063C000187A904693F800B040F6FF7A67EE266A96
:1063D0009FED986A2B46984E019200941CE000F4C1
:1063E0007061B1F5006F00F0B38000F29380B1F5F9
:1063F000806F00F0DB80B1F5C06F7BD1C0B24CF094
:10640000080C988283F81EC0013214330EF1040E7A
:106410000236D2B2BA422AD093F81EC09889BCF193
:10642000010FDCD1504500F0D080C0F30801400AD4
:1064300001FA00F081B2002900F0BF807F4C80B2E9
:10644000BBF12D0F04EB5101B1FBF0F000F0D78050
:106450004FF6FF718842D7D007EE900A0199F8EE07
:10646000E77A014480B2019167EEA67AB3E0009C1E
:10647000B8F1000F0DD0DDED017AB8EE677A07EEC6
:10648000908AF8EE677A27EE267AC7EE276AC4ED7F
:10649000196ADFF8B4A16A4A9AF80030A26613B309
:1064A000684E0027DFF8788106F14C09B8F80E3005
:1064B000304694ED180A013707EE903A08F11408B7
:1064C0000836F8EEE77A27EE800A38F089FD9AF868
:1064D0000030D4ED1A7ABB42A9EC010A87FEC00A4B
:1064E00084ED1A0AE2DC022385F8043103B0BDE82A
:1064F000F08F7047B1F5007F31D14CF0020CC1B282
:1065000083F81EC093F81FC019828C45BFF47CAF7E
:10651000D87779E7B1F5406F13D0B1F5606F06D148
:10652000C0B26CF07F0C988383F81EC06CE7B1F5A5
:10653000206F14D1C0B24CF0200C188383F81EC019
:1065400062E7C0B24CF0400C588383F81EC05BE792
:10655000C0B24CF0100CD88283F81EC054E75045EE
:1065600046D0C0F30801400A01FA00F081B221B31D
:10657000324C80B2BBF12D0F04EB5101B1FBF0F0B6
:1065800049D04FF6FF7188423FF43EAF07EE900AC4
:106590000199F8EEE77A014480B2019167EEA67A9C
:1065A0004CF0010CD88183F81EC017E0C0B24CF04B
:1065B000040C588283F81EC026E7BBF12D0F7FF430
:1065C00023AF4FF0FF3131801EE7BBF12D0FF0EE0E
:1065D000467A08D00020D88183F81E9008F101087F
:1065E000CEED007A10E74FF0000100203180F2E795
:1065F000BBF12D0FF0EE467A08D00020D0E74FF621
:10660000FF71308088423FF4FFAE25E74FF0000174
:1066100000203180C4E73080B3E700BFC80100200C
:10662000FC0C0020BC27002044560020951B0120B4
:106630000000704200000000981B0120C0270900E4
:10664000FFFF7F7F645600201C25002070B41A4C89
:106650001A4BA4FB02425209A3FB0243DB0803EBE3
:106660008303A2EB430390F858205FFA83FC624552
:106670001ED09A00046800EB830346689D68641B83
:1066800004601D6B751B456000259D601D6380F8CF
:1066900058C08318013404609A6801329A6029B99D
:1066A0004268013242601A6B01321A6370BC704753
:1066B00004689A00EDE700BF1F85EB51CDCCCCCC30
:1066C00010B5437B04468268581C6073D154627BCA
:1066D000237B934200D802B910BD2368D4E901019D
:1066E00098470023637310BD427B42B1036810B525
:1066F0000446D0E9010198470023637310BD704739
:10670000084B024602201968B2EB910F4FEA910341
:1067100007D25B0840009A4280B202D2FF28F8D923
:10672000704770474C1B01200139032930D81E4B9C
:1067300001EB810C024610B403F1480403EBCC03D7
:1067400004EBCC044FF0010C046003F1480480F822
:1067500088C093F8480002281CD0C9B21348C1EB86
:10676000011150F83110D96471B10221604683F8EB
:1067700048104FF48071A18102F110014C325DF894
:10678000044BC3E91812704700205DF8044B7047B2
:106790000020704793F8552060465DF8044B624432
:1067A00083F85520704700BFE8730120F8210120CD
:1067B000954B2DE9F04FDFF864B285B04FF0010939
:1067C0004FF0000A1D469BF80030022B0CD00AF156
:1067D000010A09F101090BF1280B0535BAF1040F83
:1067E000F1D105B0BDE8F08F95F90320511C00F000
:1067F000E680D2B201924FF00C0C4FF008085FFA1D
:106800008AF1AE46012A50B225D800247F4D1CFBE8
:106810000087234634B10133172B1CD015F81C4FC9
:10682000002CF8D16E788E42F5D1EE59002EF2D0C0
:10683000774D6F6801342435BE4214D0102CF8D146
:10684000734B13F8083C33B9714B4FF0140003F845
:10685000079C03F8080C0132019BD2B29A42D1D9AD
:106860007546002429E0E4B2694D671E07EBC706B0
:1068700005EB8606357F039506F11C050295039D01
:10688000002DE8D1C3EBC303029A00EB400075462C
:106890009B0096465D4A07F0070703EB800386F8E6
:1068A0001D90204637721344CBF81060DB68F3600C
:1068B00014238EF80030F3F7E5FB95F904104B1C18
:1068C00000F09680C9B201914FF008085FFA8AF390
:1068D00001294FFA81FC20D80C224C4812FB0C866F
:1068E00000220132172A18D010F81C7F012FF8D18E
:1068F00047789F42F5D18759002FF2D0BE46002637
:10690000434F786801362437864526D0102EF8D1BB
:106910003F4A12F8082C002A6ED00131019AC9B200
:106920009142D5D9002C46D02423394A601E002636
:1069300003FB0020CBF81460CBF81000F3F7FEF84F
:106940005846F3F7CFF83346324620463149F3F73D
:10695000ADFB01238BF80C3039E7F0B22C4F00F17E
:10696000FF3E03900EEBCE0007EB800000F11C060B
:10697000077F0296002FD0D103466046039E0EF09B
:10698000070E9C46C2EBC20300EB40001F4A9B006F
:106990008CF808E08CF81D9003EB80033046CBF8B0
:1069A00014C01344029ADB68CCF80C301323137024
:1069B000F3F768FB3CB90023CBE9043307E7012375
:1069C0000022019317E7DBF81400F3F7B7F8DBF8C0
:1069D0001000F3F7B3F85846F3F784F83B463A460D
:1069E00030460D49F3F762FB01238BF80C30EEE6DD
:1069F00001230021019367E7054A4FF0130002F8D5
:106A0000079C02F8080C88E73063012078F5040839
:106A100080000120E55C0108595C01083074012008
:106A200030B40568EFF3118C102383F312880368E8
:106A30001B6AEBB18B6804460A461BB1D36914325A
:106A4000002BFBD12B6A6BB1986838B9934209D0FF
:106A5000186828B15B6898680028F7D01433F3E70A
:106A6000C3E900415FFA8CFC8CF3118830BC70479D
:106A70005FFA8CFC29628CF3118830BC38F0A0BA24
:106A800030B593B0002304468DF807100DF10601D0
:106A90008DF806200DF1070501228DF818300395B9
:106AA0008DF82C208DF840201193CDE9073103A9F2
:106AB000CDE90432CDE90932CDE90C33CDE90E330D
:106AC000FFF7AEFF2268136A002BFCD113B030BD74
:106AD00010B592B08C46044609920DF107020A9354
:106AE00000230392012203A98DF807C005928DF8B7
:106AF0002C208DF8402004938DF818301193CDE9A7
:106B00000733CDE90C33CDE90E33FFF789FF226857
:106B1000136A002BFCD112B010BD00BF2DE9F04F5D
:106B2000056885B02C78012C0AD0022C03D12C6A80
:106B3000002C00F0C8800026304605B0BDE8F08F7C
:106B400095F90450032DD4BF00260126B5F1FF3F6F
:106B500008BF46F00106002EEDD11F4605EB4503A8
:106B6000DFF838834FEA45095B0108EB030A143369
:106B700043440293DAF81430002BDDD0FF29944609
:106B80008646027900F0D9809AF85500202840F016
:106B9000CE80B8B2002F00F0E8819AF85470012F2F
:106BA00000F0C5808AF854409B46B64C276806E042
:106BB0002368A3EB070EBEF1190F00F2AB81DBF8DF
:106BC000183013F4004AF3D1530009EB050B00977A
:106BD0000A4608EB4B1B03932223CBF838C08BF8F3
:106BE00055304023CBF848A08BF856300A23CBF819
:106BF00058A0ABF83E00DDE9020131F0ADFC002801
:106C000040F01A82BBF83E309BB2FF2B40F201826B
:106C1000DBF81410FF239C48ABF83C304B689B4AD0
:106C20000340039803431A434A6009EB050B984A53
:106C30004FF0FF0CDFF868E208EB4B1ADAF81400AB
:106C400004E02168C91B0A2900F22C81836913F032
:106C50000403F6D0416ADAF838301970BAF83E30D9
:106C6000BAF83C10013B01399BB289B2AAF83E3018
:106C7000DAF83830AAF83C100133CAF83830BAF8DC
:106C80003E309BB211B9002B40F05581BAF83E302E
:106C90009BB2002BD2D13946029831F04BFD00282F
:106CA00045D1DAF8143020217A4C08EB4B18D96121
:106CB00001265A6822405A608AF8551088F8540014
:106CC0008AF8560038E741F080010126FFF700FFFF
:106CD00032E72268521A0A2A00F28A80986910F074
:106CE0002000F6D01022DA612022DA619A69970733
:106CF00001D500229A629A69D40703D49A6942F0B6
:106D000001029A615A684D44624C002108EB451813
:106D1000202022405A60D8F8583088F8541043F0A8
:106D20000403C8F8583088F8550088F856105A4AB5
:106D3000138801339BB21380FEE69AF85510202980
:106D4000F5D19AF854100129F1D08AF854404D4CED
:106D5000216804E02068401A192800F2DB80986955
:106D600010F40040F6D109EB050EBFB2520008EB5B
:106D70004E1ECEF838C04FF0220CCEF848008EF8E8
:106D800055C04FF0100C8EF856C0CEF85800AEF833
:106D90003E70BEF83E0080B2FF2840F2288158685D
:106DA000394F3840394F10430743FF20AEF83C00BD
:106DB0005F6009EB050A4FF0FF0B964608EB4A1798
:106DC000FB8F9BB2002B00F0FB807B6908E09A6987
:106DD00012F0200276D12068401A0A2800F28B8037
:106DE0009A69520714D49A69D2063FF577AFEEE755
:106DF0004D44202208EB4518D8F8583088F8540044
:106E00001343C8F8583088F8552088F856008EE7A4
:106E1000586ABB6B1870FB8FB88F013B01389BB26F
:106E200080B2FB87BB6BB8870133BB63FB8F9BB220
:106E3000002BC5D00028C3D1D7F814C003E02268C6
:106E4000521A0A2A2ED8DCF8183013F08003F6D034
:106E5000FB8F9BB2FF2B40F28D80DCF80430A7F84B
:106E60003CB023F07F7323F4583323F47F7323F073
:106E7000030343EA0E0343F0FF7343F48033CCF87B
:106E800004309DE784270120009800FC0024FF8146
:106E9000009C00FC00E800FE0C5F0120382001206F
:106EA0000000FF014D44202108EB4518D8F8582078
:106EB00088F854300A43C8F8582088F8551088F8E4
:106EC000563034E79869400702D5B88F00289FD123
:106ED00020204D445A4C0022D86108EB45185968CF
:106EE00021405960C8F8582088F8542088F8550087
:106EF00088F856201BE74D449446202208EB45189D
:106F0000D8F8583088F854C01343C8F8583088F877
:106F100055200CE74D442021002208EB4518D8F8F5
:106F2000583088F854200B43C8F8583088F855106A
:106F300088F85620FBE6DAF8140003E02168C91B44
:106F40000A29AFD8836913F08003F7D0BAF83E302E
:106F50009BB2FF2B24D9436803991340AAF83CC085
:106F60000B4343EA0E03436090E64FF40073CAF804
:106F70005830DCE6FB8FDCF804009BB220F07F7019
:106F8000BB87DBB220F458304EEA034320F47F7015
:106F900020F00300034343F00073CCF804300FE704
:106FA000BAF83E3003999BB2AAF83C30DBB241EA12
:106FB0000343416811400B4343F00073436065E6AF
:106FC000029831F0B7FB00287FF4B1AE7B69202135
:106FD0001B4C08EB4A18D96101265A6822405A60B6
:106FE00087F8551088F8540087F85600A4E5BEF8D5
:106FF0003E00DFF854C080B25F68AEF83C00C0B21B
:1070000007EA0C0742EA004038430E4F07435F602F
:10701000CFE6BBF83E30039A9BB2DBF814100A4867
:10702000ABF83C30DBB242EA03434A680240134308
:10703000044A1A434A60F8E58BF854A077E600BF8B
:1070400000E800FE00240082009800FC30B5002318
:1070500093B0012204468DF818300DF10705119305
:107060008DF8071003A90A928DF82C208DF8402086
:107070000395CDE90432CDE90733CDE90C33CDE9F1
:107080000E330DF10B030993FFF7CAFC2268136A54
:10709000002BFCD19DF80B0013B030BD036810B578
:1070A0009B68044698470122FF236273A37310BDB7
:1070B000036810B504461B689847012123682046E1
:1070C0009B689847E37B0133E37310BDF0B583B051
:1070D00004460D461646089F0193384635F01AFBC4
:1070E000216828443246E672A07220468E692946FD
:1070F000019BB44603B0BDE8F040604703689B6A5B
:10710000184700BF03685B6D03B11847704700BFA5
:107110000368DB6C03B11847704700BF002310B54C
:10712000C373044642748A6C016003730AB1194642
:1071300090472368012120469B689847FF212368D8
:107140000122A173DB6C62731BB12046BDE81040C5
:10715000184710BD70B54FF6FF7C0E4D0E4C4FF02A
:10716000010E0E490E4E00234CFA03F20EFA03F004
:10717000013312F0010F03D00C60083121F8040C28
:10718000102BF1D104F58064B44202D035F802CF5F
:10719000E9E770BD30F90408000002400424012032
:1071A0000018024010B50409013C052C16D80D4A00
:1071B00000F00F0332F8141041FA03F212F001024A
:1071C0000ED0012098400138084035F0CFFF064B23
:1071D000064A1B5D184402EBC00010BD002010BD24
:1071E000104610BD30F904083CF9040804240120BD
:1071F000F8B50B4F97F8343083B10A4C0025A668D8
:1072000001353079FFF7CEFF18B1217DF279F2F721
:10721000B9FF97F83430A034AB42F0DC0120F8BD60
:10722000B01E0020FC07002038B50C46054600784B
:10723000FFF7B8FF611C0446C9B210B14123C17108
:10724000837120466978F3F71BFBAB7820461BB1AE
:10725000BDE83840F2F7A0BDBDE83840F2F7A2BD66
:107260002DE9F041FFF79EFF0C4B054600241F68F7
:107270000B4EBC4201DBBDE8F08104EB4403F05C43
:1072800003EB0608FFF78EFF854204D121464046F6
:10729000BDE8F041C8E70134EBE700BF806301209F
:1072A00050630120054B53F8203033B11A689B8896
:1072B00051690B4218BF1B0493617047FC1A0120EF
:1072C0000E4B012210B40E4C93F800C002FA00F3EA
:1072D00054F8200003EA0C0351B1003B18BF01230E
:1072E00018B1016882883BB18A615DF8044B704730
:1072F000B3FA83F35B09F3E71204F5E7081B0120F7
:10730000FC1A012070B5392086B0FFF74BFF054607
:1073100010B140F23E23C380124C4FF400710222A0
:107320000026236B104843F004032363236B059668
:1073300003F0040300930323CDE9011201A9009A8D
:10734000CDE903632CF0FEFAA36832460E2123F048
:107350007843284643F0E043A36006B0BDE87040A0
:10736000F2F7DCBF003802400008024010B5054CBF
:1073700023681B6998472368002283F836209A63A4
:1073800010BD00BFBC27002010B5084C236893F83F
:10739000352012B1DB68984700B910BD044A0121BD
:1073A0002368126883F836109A6310BDBC2700204A
:1073B000F41A01200D4A02EBC00310B593F8ECE07B
:1073C00093F8ED408EEA010C644500D110BDD3F86E
:1073D000E830C0002BB11C688E459B8808BF1B0499
:1073E000A361104480F8EDC010BD00BFE873012018
:1073F000F8B5114E0124114D522716F8010BFFF775
:10740000D1FE0022202118B1C4718771F2F7BAFEB3
:1074100015F8010BFFF7C6FE4FF0530C0022402178
:1074200020B1C47180F806C0F2F7ACFE0134E4B2BA
:10743000052CE2D1F8BD00BF00700120F46F0120DF
:1074400003681B68184700BF03682DE9F0415F6AB5
:107450001FB13B46BDE8F041184704460D461646AD
:1074600000E023689B6820469847B042F9D3002E7D
:1074700008DD2E442368204615F8011B1B68984739
:10748000AE42F7D1BDE8F08103685B68184700BFE2
:1074900003689B68184700BF0368DB68184700BF94
:1074A00003685B69184700BF03689B6A03B118470C
:1074B000704700BF0368DB6A03B11847704700BF1D
:1074C00003689B6A10B5044682B023B1CDE900126F
:1074D0009847DDE900122046FFF7B6FF2368DB6A14
:1074E00023B1204602B0BDE81040184702B010BDDD
:1074F000E6E700BF014B1868F4F706BDEC1E00205C
:10750000014B5868F4F700BDEC1E0020014B986851
:10751000F4F7FABCEC1E0020014BD868F4F7F4BC79
:10752000EC1E0020014B1869F4F7EEBCEC1E0020A5
:10753000014B5869F4F7E8BCEC1E0020154B1B8882
:107540005BB9154A154B12781B688AB17BB11A6872
:107550009B8800B91B0493617047114BD3F81C2121
:107560002AB150B9D3F80821106083F81901704787
:1075700080F00100002BEAD1F9E7B3F820C1012126
:10758000084AD3F80801B2FBFCF20A41026083F812
:1075900019117047266301202C6301202863012004
:1075A000E873012040420F0030B4EFF31183102242
:1075B00082F312880B484FF0E0210B4DDBB20268DA
:1075C0000A4C013202608A692A600022C4F8242130
:1075D0000A6983F31188064A1368013330BC1360CB
:1075E000704700BFF41A0120101C0120E87301202D
:1075F0008427012010B4EFF31181102383F3128844
:107600004FF0E0229469136913F4803F0D4B03D0CF
:107610000120C3F8240194690B4AC9B21068D3F859
:10762000242181F31188094B02444FF47A701968C0
:1076300000FB01F31B1B5DF8044BB3FBF1F300FBF4
:1076400002307047E8730120F41A0120141C012055
:107650002DE9F04FDFF8F48183B0784AD8F8043090
:10766000147801912BB19A88A507196858BF1204A4
:107670008A61D8F800202AB19188E407156848BFCC
:107680000904A96101386E4E6E4CC7B26E4DDFF829
:10769000C0B133B119689B884869034218BF1B0405
:1076A0008B6132B1116893884A69134218BF1B0479
:1076B0008B610120DDF804A0FFF740FF7368C3F37E
:1076C0000803002B40F0AE80EFF31183002B40F055
:1076D000A9804FF0E0202368816922689342FAD1A3
:1076E0002A689142F7D8DBF800C04FF47A7000FBAB
:1076F0000CF2511AB1FBFCF100FB03197368C3F3E0
:107700000803002B40F08B80EFF31183002B40F037
:1077100086804FF0E02C2368DCF818002268934242
:10772000F9D12A689042F6D8DBF800104FF47A724B
:1077300002FB01FEAEEB0000B0FBF1F002FB030028
:10774000A0EB0903B3F57A7FD8D3BAF1010AB5D11A
:10775000D8F8043033B11A689B8851690B4218BFBE
:107760001B049361D8F8003033B11A689B885169C3
:107770000B4218BF1B0493610020DDF804A0FFF743
:10778000DDFE7368C3F30803002B4FD1EFF31183C1
:10779000002B4BD14FF0E02023688169226893428F
:1077A000FAD12A689142F7D8DBF800C04FF47A701A
:1077B00000FB0CF2511AB1FBFCF100FB03197368DA
:1077C000C3F3080343BBEFF311832BBB4FF0E02C53
:1077D0002368DCF8180022689342F9D12A689042A5
:1077E000F6D8DBF800104FF47A7202FB01FEAEEB24
:1077F0000000B0FBF1F002FB0300A0EB0903B3F5BE
:107800007A7FDCD3BAF1010ABBD1013FFFB2FF2F6F
:1078100010D0D8E900233CE7FFF7ECFEEDE7FFF7D7
:10782000E9FE8DE7FFF7E6FE814667E7FFF7E2FE38
:107830008146C4E703B0BDE8F08F00BF081B0120FC
:1078400000ED00E0F41A0120101C0120FC1A0120B8
:10785000141C0120124B5B68C3F30803F3B9EFF368
:107860001183DBB90F4A4FF0E02C10B40E4C1368B3
:10787000DCF8180011688B42F9D121688842F6D8EB
:107880000A4A4FF47A71146801FB04F2121AB2FB2F
:10789000F4F25DF8044B01FB03207047AAE600BF39
:1078A00000ED00E0F41A0120101C0120141C01203E
:1078B0002DE9F04FDFF8E8A29AF828212DED048B8E
:1078C000022A95B0CDE9020215D110F06DF99AF8AF
:1078D0000430DC0740F12C83A04B1B68002B00F028
:1078E00005839F491A6809789B88C8079D4D58BF32
:1078F0001B049361FBE201239B499A4281F88C307F
:1079000040F007819AF875329FED987A07EE903A29
:107910009AF80430F8EEE77A13F0010F944B67EE13
:10792000877A0493FCEEE77A17EE904A40F0B18430
:10793000029B1C44CAF87C42DAF8BC110029C0F250
:107940000A839AF88132002B00F06083894B0593FB
:10795000049B1B685D0700F16A844FF0004300261A
:107960000DF1340B1193DAF898320F96B3420D965D
:10797000129610960E9645DD9FED7F8A7F4F804DC3
:1079800008E0B9F12C0F40F271810136DAF8983233
:107990009E4237DA17F8014B04EB440C630015F8EC
:1079A0001C9060460193012309F01F024FEA591E03
:1079B00005EB4C0C03FA02F214AB4FEA40086046A8
:1079C00003EB8E034FEA8E0153F80C3C1340D8D0E2
:1079D0000AEB0103D3F8BC3112EA030900F0768107
:1079E0000FAB0FA9013653F82E3023EA020341F8FA
:1079F0002E305BF82E3013434BF82E30DAF89832E5
:107A00009E42C7DBDAF89C32002B2DDD5D4E002450
:107A10005B4D4FF0010816F8010B14AF5A460FA941
:107A200000EB4003013405EB430318465B794FEA52
:107A3000531C03F01F0307EB8C0C08FA03F35CF8EC
:107A40001C7C5CF814CC3B4203EA0C0C14BF0123F1
:107A50000023BCF1000F18BF83F0010311F01AFFDF
:107A6000DAF89C329C42D6DB0DF13B010DF1330379
:107A70000C4613F8012F11F8010F9C4282EA000214
:107A80001A70F6D1404B9BE8030083E80300049B87
:107A9000DAF8BC211B6802F480109AF8701203F423
:107AA0008003034314BF012300238AF876320029A0
:107AB00040F03884354B1B78002B00F03D84DFF814
:107AC000E490970740F13681059B1B689E0740F1C3
:107AD0003681BAF87832DD0740F17786022034F03B
:107AE00059FA9AF80430D90740F14281DAF8BC31EA
:107AF0001A0640F13881BAF878120F0500F140817A
:107B00004FF4006034F05CFABAF87812DAF8BC315D
:107B100036E19AF82931002B40F014829AF84C3162
:107B2000002B00F0E38100239AF84D418AF84C3194
:107B3000029B002C40F0FA82002B00F00C859AF892
:107B40004E31002B01F02A83114F4FF001089FEDB9
:107B5000118A114EA7F12409104D35E0FC1A0120BD
:107B6000081B0120951B0120445600200024744965
:107B7000DC5301206C5801208096984A88760120B9
:107B80006C540120A4760120A475012064580120C2
:107B90003875012000007A449461012028540120A6
:107BA000E8730120A82600205946DAF8303148460B
:107BB0009847032C40DD01349AF84EB10436A7EC07
:107BC000010A5C4580F2E884072C2B6BD4BF15F8C2
:107BD00004B05FFA84FB002BE6D0DAF83031594666
:107BE000484698476A8B0AEB4B03A98BB3F8983148
:107BF0009A4200F2B28407EE901A07EE103AF8EEBD
:107C0000677AB8EE477AC7FEC77A08FA0BFB2B6B88
:107C10001BEA030F05D0DAF8C03113F4807F00FEB1
:107C2000270ABCEEC00A032C10EE103A9BB200EEFD
:107C3000103AB8EE400ABEDCB5EE400AF1EE10FA9A
:107C4000B9D0338806EE903A7388F8EE666A07EE8C
:107C5000103AB8EE477A30EE660A37EE667A60EE92
:107C6000087A87EE870A30EE080AA4E708F10208CE
:107C700005EB080115F808204C78A24221D29CF8A7
:107C8000011040F2833E4FF0190C40F633080AEB26
:107C90008101D1ED767A1CFB02E1FDEEE77A17EE69
:107CA000902A4245A8BF4246B2F5617FB8BF4FF463
:107CB00061728A4205DD1CFB04E39A42CCBF0023BB
:107CC00001235A460FA911F0E5FD5EE608F102080E
:107CD00005EB080315F808E093F80180C6451CD2AF
:107CE0009CF801304FF0190C0AEB8303D3ED767A40
:107CF00040F28333FDEEE77A1CFB0E3E40F6330C78
:107D000017EE903A6345A8BF6346B3F5617FB8BFED
:107D10004FF46173734500F35081C8465144D1F864
:107D2000B4321A4200F0C18043465A460FA911F0FE
:107D3000B1FD2AE6A74BDB78002B7FF4C5AE01200E
:107D400034F028F9DAF8BC315C077FF5C7AE0120C2
:107D500034F020F9BAF8783298073FF5C2AE022025
:107D600034F02EF9BDE69B4AD278002A40F05285C5
:107D70004FF4006034F00EF9BAF87812DAF8BC313A
:107D8000954A8E07526840F0EC803AB193480478E7
:107D90001068A407928848BF12048261904A42F298
:107DA0001070D2F880211061DA0007D49AF804200C
:107DB000570703D522F004028AF80420059A1268B6
:107DC00012F00A0F13D01E0740F1BF834D0740F198
:107DD000C784DC0640F10682BAF87822100500F16B
:107DE0000182510641F156809A0500F108829E06F3
:107DF0004FF4807040F1F38134F0E2F8794B1B7856
:107E00000E2B00F00482082B00F001829AF8043057
:107E100013F0010F744B1B6800F0DD8101228AF81A
:107E20006224002B00F0598327F03CFE9AF80430BE
:107E3000DD0700F15283049BDAF8BC211B6802F4D1
:107E400080726A4903F08053134391F8282214BFCB
:107E5000012300239A4202D00022C1F84022634A43
:107E60000224634D82F8283299F800308AF82841BC
:107E7000002B45D1FFF7EEFC029BC3F101031E1856
:107E800037F0BAF8039A0AEB82039200D3F864340D
:107E9000B0EBA31F01D0830198118642524440F3F6
:107EA0008880B601C2F864642AE0FFF7D3FC07EECD
:107EB000900AF8EE677AF4EEC87AF1EE10FA3FF520
:107EC00064ADB8F1000F7FF460AD63000122494852
:107ED000234415F81330590903F01F0302FA03F382
:107EE00050F82120134340F821304EE5404D002446
:107EF000DFF814918AF8284199F80030002BB9D0A6
:107F00002B78472B08D103993B4A0AEB8103D3F81E
:107F100064349B1122F811300AEB8404D4F8640411
:107F2000801115B0BDEC048BBDE8F04F37F02CB8D4
:107F300010F0A2FB9AF80430D907D7D42C4D0CF0DE
:107F400061FAD4E7DAF838310AF5967098470023D9
:107F50008AF82931E2E59AF80430DF073FF5F1AC01
:107F6000F4E43AB11D4804781068A507928858BF18
:107F700012048261214ADFED226AB2F8442007EE42
:107F8000902A204AF8EEE77A527986EEA77A07EE31
:107F9000902A134AD2F88001F8EE677A67EE277AC2
:107FA000FDEEE77A17EE902A0A2AB8BF0A2202618C
:107FB000FAE6013BC2F86434A2E740F2833E4FF098
:107FC000190C1CFB08E84345CCBF4FF000084FF0EC
:107FD0000108A3E6AC560120FC1A0120081B012071
:107FE00078580120A0520120545F012044560020FF
:107FF000951B01209C760120981B0120AC260020B7
:1080000000247449E0560120A8260020B948BA4A45
:10801000848AC08A06EE904A02F1100407EE100A24
:10802000F8EEE66AB8EEC77AF2EC017A9B08F4EE55
:10803000E67A63F07F00F1EE10FAF4EEC77AC8BF7B
:10804000C3B2F1EE10FA48BF43F040039442EBD1C3
:108050009AF882229A4200F02C870022AAF8842201
:108060008AF88622A54A8AF882321278002A00F01D
:1080700016875F2B00F059846F2B00F032870023A6
:10808000CAF888329AF80430D9073FF55FAC9AF8FD
:108090008632002B7FF45AACBAF98432322B7FF748
:1080A00055AC974B1B6813F0600F7FF44FAC954BAA
:1080B00001221B788AF88622934201F00782DAF8BF
:1080C000C03113F400727FF441AC9AF88232572B1E
:1080D00001F0C882049909684F0702D55A2B00F0B5
:1080E0009A805D2B01F05E835E2B01F054835B2B45
:1080F00001F04A83562B01F0A3839AF88232972B22
:1081000001F01784BAF87822960741F0BB83A3F1F7
:10811000B702072A01F29F83DFE812F0960B9D0B4E
:108120009D0B9D0B790C9D0B720C3C0C002B00F0F1
:108130001282013C744D8AF84D41DAF83C31002B33
:1081400000F0F98198470446FFF784FBDAF85C22D7
:10815000031BA21A059300F0EE81CAE99742029927
:10816000DAF86432CB1A05998B42C8BF13462A78D5
:10817000DFED666A3E2A029ACAF864224FF6DC7284
:1081800000F0A4829A4240F2B631A8BF1A468A4251
:10819000B8BF0A4607EE902A9B1AB8EEE77AB3FA00
:1081A00083F35B09C6EE877A8AF86832584B1A80E7
:1081B000CAED9B7A574B1B68DE0400F1E2820298FD
:1081C00010F01AFF00283FF492AE0124DFF850911E
:1081D0008AF8284190E6002B7FF426AE2BE633F098
:1081E000D9FE0BE6402033F0D5FEDAF8BC319A0513
:1081F0007FF5FDADBAF8782217053FF5F8AD13F01D
:10820000A9FE002840F00687DAF8BC31EFE54020EF
:1082100033F0C0FEFAE59AF89032002B01F0C183EA
:1082200001238AF890228AF891323B4B05939AF801
:108230009232DBB19AF80430DC0717D52D4B9AED5A
:10824000757A9B8A07EE903AF8EEE77AB4EEE77A11
:10825000F1EE10FA0ADDDAF8BC3113F0010207D1B1
:108260008AF892223222AAF8942201E0DAF8BC318C
:10827000980440F163829AF896322BB99AF89032BA
:1082800013B93223AAF8943201238AF89632FFF701
:1082900064BB1D68E9067FF54BAB204B187815F0E1
:1082A0004FFA00287FF444ABEA043FF541AB9AF85B
:1082B0007632002B7FF43CABBAF878321B053FF5E1
:1082C00037AB0FF0B9FF0D4B1B78002B01F0388254
:1082D000002841F054822CB1DAF87C32029A9A429A
:1082E00001F2A68210200BF0EBFE01238AF8803207
:1082F000FFF722BB28540120B0750120A8030120FC
:1083000038570120D4270120951B012000247449EF
:10831000F85E0120DC5301206C5801201763012016
:10832000A826002014200BF0CBFE8F4BDAF8BC21DE
:108330001B78002B7FF4C3AB002A04DA9AF80430D0
:10834000D9077FF5BCAB9AF8C431DFF840B2874A51
:1083500001931268DBF8003009925A1C00F0E585A1
:10836000DFF82C92824A002B08921268079240F3A1
:10837000CF800025CDF828907E4CDFF81882A946E2
:1083800021790A23012713FB017308EB030218F874
:1083900003005578A84280F0AF8001EB810240F6DF
:1083A000330E192640F2833C18F8123008EB4202D3
:1083B00016FB00C00AEB8303D3ED767A8B00FDEE4B
:1083C000E77A069317EE903A7345A8BF7346B3F564
:1083D000617FB8BF4FF46173834240F38D80D278E0
:1083E00016FB05C6644D013AB34202EB4200284435
:1083F00090F8885302FA07F07EDC002D7CD02368C9
:10840000079EF31A002B03DB06F5FA7367712360EE
:10841000019B002B72D0584B02441A4492F88933C6
:10842000002B6BD18B000B4408EB43010B79043319
:10843000DBB20AEB830393ED727A504B5B8A03F154
:10844000C80107EE901AF8EEE77AB4EEE77AF1EE9B
:1084500010FA00F3AB81C83B07EE903AF8EEE77AEA
:10846000B4EEE77AF1EE10FA40F1A885637992F85C
:108470008A23002B42D0534241F20241404A0693E4
:1084800011800221FF2050540E200BF019FE6A1EAD
:108490001F2A00F2B983DFE812F0CC029F02C30367
:1084A0006C024C048D0363032A037E0463043304CB
:1084B000B7036C02C7048D0363032A030F040B0484
:1084C0000704EA03F7021304B703CC02BC049F02BB
:1084D000BA04B703F702B60499042A4B1B78002BA1
:1084E0007FF4A9AC254B93F82130002B3FF4A3ACCB
:1084F00017200BF0E5FD9EE40023236009F101093C
:10850000DBF8003008349945FFF63AAFDDF82890E3
:10851000019B002B40F0A881089BDAF840241B68DF
:108520009B1AB3F5FA6F02D40023CAF84434DAF880
:10853000BC21FFF7C6BADAF86022002A7FF40FAE3A
:10854000DAF86432029AD31A11E6042033F022FDDD
:10855000DAF8BC313DE40C4DEFE507EE902AF8EE79
:10856000677AFFF752BB00BF645801209852012080
:10857000F41A0120BC760120D037050828540120C8
:10858000F456012008270020951B0120A403012098
:10859000A8260020E85F0120DAF8BC319AF8C491DF
:1085A00013F0400309F00109049318BF4FF00009CC
:1085B0009C4B8AF8C59108931B680693BBF1000F8A
:1085C00000F0FB85984B0024AA8B1B880792069A23
:1085D00009EE903A6B8A954F02F5967209EE103AC1
:1085E000934E97F80380F8EE699A6B8BB8EE499A30
:1085F00001924A460997D9464746DFED8E8A9FED9C
:108600008E8A06F1480598469346BBF1000F39D093
:108610008A4B03EB8400D0ED007ABCEEE77A17EECC
:10862000103A98B240452DD3079B98422AD8019B17
:108630002B6077B3032C2FDCBB460134C7FEE87AEE
:108640000435C7FE887A4C45E6EC017ADDD1D9467F
:10865000099F089BB9F1000F00F0BC801A683B69C4
:10866000FA60002B00F0DB84D31A3A6A9A4280F257
:10867000BF800123724A87F82530136823F0040372
:108680001360B5E087B1032C06DC032C49FE897A20
:10869000D3E7049B002BD0D0E0B217F067F907EEC8
:1086A000900AF8EE677AC8E7049B002BF4D128689B
:1086B000069B181A0028C0F2E983032CECDC4FF06B
:1086C00000034FF0000B8AF8C531E5E79A4240F20B
:1086D000B6315C48A8BF1A468A42B8BF0A4680FB3A
:1086E0000361059E07EE902A94B29A1ADB17B8EE42
:1086F000E77AC3EBA10380FB0601F017B2FA82F21E
:10870000C6EE877AC0EBA1004F495209A1FB046174
:1087100047F6FF768AF86822B3424FEAD101A8BF34
:108720003346B042A8BF3046484E3380484B708035
:10873000B280F180CAED9B7A1C803BE59AF89032BA
:10874000002B3FF40AA99AF8043013F001037FF4D8
:1087500004A98AF8903201238AF89132FFF7FDB814
:10876000042033F02DFCBAF96034364A82FB031240
:10877000DB17C3EBA203AAF85834DAF8BC31FFF7D1
:1087800028BBDAF8BC31DC073FF519AD9AF80430A4
:10879000D8077FF514AD9AF870221AB943F0020396
:1087A0008AF8043004200FF0F3F808E592F88A33D1
:1087B0006279002A3FF4A2AE264A0693002B00F00D
:1087C000D8872549116004215CE6012033F0F8FBCD
:1087D000FFF784B91B681A49FA683B619B1A0A685B
:1087E00042F004020A607A689342C8BF87F8259075
:1087F0001A4D2B78282B07D1DAED757A134BFDEE45
:10880000E77A17EE902ADA809AF8583201338AF81C
:10881000583292E4044AD279022A7FF4A9AAFFF7D7
:108820006AB900BFF41A012060540120AC5601203F
:10883000B075012000A00C4500803B443875012034
:108840003857012067666666CDCCCCCC981B0120DA
:10885000F85E0120F456012002140214951B012039
:108860000080BB446F12033BDAF8D032002B7FF755
:1088700053AE5FED058A4FF0000B1FED068ADFF85F
:10888000DC82B04ECDF81C90AE4B012213F82B5079
:108890000A2313FB052308EB030118F8032048788B
:1088A000824236D205EB850340F633014FF0190CB6
:1088B00040F2833718F8134008EB43031CFB0272A5
:1088C0000AEB8404D4ED767AAC00FDEEE77A0194ED
:1088D00017EE904A8C42A8BF0C46B4F5617FB8BF32
:1088E0004FF46174944214DDDA781CFB0070964FEB
:1088F000013A844202EB4202CCBF002401243A44F4
:1089000092F88893B9F1000F08BF0024002C40F0C2
:108910008D82002373800BF1010BDAF8D03204361C
:108920009B45B1DBDDF81C90F6E5BAF98432B3F56E
:10893000FA7FFFF60BA89AF88632002B7FF406A880
:10894000CAF8883201238AF886329AF8043013F084
:10895000010400F0D2859AF870221AB943F002039C
:108960008AF8043003200FF013F8784B0593FEF7D4
:10897000EFBF099B069A9E7A164486F308069E72FC
:10898000734B5A79002A40F0F5850D2D00F059817E
:108990005A79099B06995E7A0E4486F308065E7240
:1089A000002A40F0BD856B4F386801236A4A137076
:1089B00015F064FC00230C2D6371089B1B6840F0CC
:1089C0004B81DAF840249B1AB3F5FA6F3FF596AD68
:1089D0000023CAF8443491E5099B069A9E7916440F
:1089E000642EA8BF642626EAE6769E71584B5A7913
:1089F000002A40F002861B2D00F023815A79099B42
:108A00000699DE790E44642EA8BF642626EAE6762F
:108A1000DE71002AC7D09AF83C341C2211960A3B1A
:108A2000ADF84C20012BBED811A90D2018F082FA08
:108A3000B9E7099B069ADE781644FF2EA8BFFF26E9
:108A4000012EB8BF0126DE70414B5A79002A40F052
:108A50004486192D00F0F580099A069916790E447E
:108A6000FF2EA8BFFF26012EB8BF012616715B7925
:108A7000002B98D09AF83C341A2211960A3BADF894
:108A80004C20012B8FD8CFE7324F06993868304BF6
:108A9000468A5A790E44B6F5FA6FA8BF4FF4FA66C3
:108AA00026EAE6764682002A40F046851E2D00F032
:108AB000C98086895A79069B1E44B6F5FA6FA8BF0D
:108AC0004FF4FA6626EAE6768681002A3FF46DAF17
:108AD0009AF83C341F2211960A3BADF84C20012B2A
:108AE0003FF662AF11A90D2018F024FA5CE7194F88
:108AF00006993868164B067C5A790E44C82EA8BFD2
:108B0000C82626EAE6760674002A40F06485112D10
:108B100000F09880867A5A79069B1E44C82EA8BF1A
:108B2000C82626EAE6768672002A3FF43EAF9AF817
:108B30003C34142211960A3BADF84C20012B3FF631
:108B400033AFCFE7AC770120D03705086C58012050
:108B5000842A01209C52012058570120E85F0120FF
:108B6000AD4F06993868AD4BC67B5A790E44C82E76
:108B7000A8BFC82626EAE676C673002A40F0978585
:108B8000102D5FD0467A5A79069B1E44C82EA8BF86
:108B9000C82626EAE6764672002A3FF406AF9AF81F
:108BA0003C34132211960A3BADF84C20012B3FF6C2
:108BB000FBAE97E7984F06993868984B867B5A79B1
:108BC0000E44C82EA8BFC82626EAE6768673002A79
:108BD00040F025850F2D35D0067A5A79069B1E4424
:108BE000C82EA8BFC82626EAE6760672002A3FF4F9
:108BF000DCAE9AF83C34122211960A3BADF84C20B8
:108C0000012B3FF6D1AE6DE7834F0123844A3868CC
:108C1000137015F033FB00236371089B1B68D0E6CB
:108C2000099B069A5E781644642EA8BF642626EA3D
:108C3000E6765E700FF0F8F9784B5B79002B40F028
:108C40008D84754F38680123754A137015F016FB33
:108C500000236371089B1B68212D3FF4B2AE714A5B
:108C6000CAF8445456601A46CAF84034ABE6099B29
:108C7000069A5E791644FF2EA8BFFF26012EB8BFC4
:108C800001265E71654B5B79002BDAD09AF83C3493
:108C9000152211960A3BADF84C20012BD1D811A911
:108CA0000D2018F047F9CCE75B4F5C4B386831E793
:108CB000594F5A4B386865E7574F584B38688BE720
:108CC000554F564B38685A7990F87D60069B1E4484
:108CD000642EA8BF6426012EB8BF012680F87D60EF
:108CE000002AB0D09AF83C34172211960A3BADF80E
:108CF0004C20012BA6D811A90D2018F01BF9A1E7D3
:108D0000454F464B38685A79867D069B1E44C82ECF
:108D1000A8BFC82626EAE6768675002A93D09AF878
:108D20003C340B2211960A3BADF84C20012B89D81C
:108D3000E1E7099B069ADE7A164486F30806DE729E
:108D4000364B5B79002B3FF47CAF9AF83C3405221C
:108D500011960A3BADF84C20012B3FF672AF9EE70F
:108D60002D4F2E4B38685A79467D069B1E44C82EDF
:108D7000A8BFC82626EAE6764675002A3FF463AF08
:108D80009AF83C340A2211960A3BADF84C20012B8C
:108D90003FF658AFAFE7204F204B38685A79067D31
:108DA000069B1E44C82EA8BFC82626EAE67606758E
:108DB000002A3FF448AF9AF83C34092211960A3B46
:108DC000ADF84C20012B3FF63DAF94E7124F134B0B
:108DD00038685A79068B069B1E44B6F5FA6FA8BF11
:108DE0004FF4FA6626EAE6760683002A3FF42BAFB4
:108DF0009AF83C34202211960A3BADF84C20012B06
:108E00003FF620AF77E7044F044B386851E6034B39
:108E1000F4E5024B20E600BF9C520120842A012089
:108E20005857012050040120974BB1E51879B6F945
:108E30000270043007EE107AC0B2B8EEC77A0AEBBF
:108E400080078000D7ED727A0690F4EE477AF1EE53
:108E500010FA3FF460AD92F88903012800F0E78032
:108E6000DA8810B9002A40F0C581089BFDEEE77A48
:108E70001B68DAF840249B1AB3F5FA6F02D400237A
:108E8000CAF8443417EE903A738044E5D6ED007A80
:108E9000FFF7D3BB402033F093F8FFF7A6B911F0EA
:108EA000010300F093808AF887220FF0A5FEFFF7F8
:108EB000E9B8764ABAF9845212689068744A82FB1B
:108EC0000042C01747F6FF74A0EBA216921134447B
:108ED000A5423FF7C7A8121A2A44AAF88422FFF72E
:108EE000C1B8DAF8C0319C053FF5C9A8BAF9843297
:108EF000B3F5FA7FFEF62AAD9AF88632002B7EF49F
:108F000025AD01228AF886229AF80420D00700F1C4
:108F1000E0830FF071FEDAF88832002B00F01C8439
:108F200000238AF88632FEF711BD0023DFF8749122
:108F30000127584C98461D46574E1193CBF80030E8
:108F4000CAF8D0321293ADF84C3089F800701BE0AB
:108F5000E378013B03EB4303334493F88933012B5C
:108F60001CD0DBF800300AEBC3010133C1F8D42276
:108F7000CBF8003081F8D88281F8D97208F1010865
:108F80000A34B8F11E0F15D020460A2211A935F077
:108F900053FE0028F2D0E288002AD9D0DAF8D03285
:108FA0000AEB8302013382F8C483CAF8D032A2F8F4
:108FB000C653E3E7DBF80030FFF7D4B90123637150
:108FC000079B03F5FA732360FFF798BACAE9A23347
:108FD0009AF80430DE077FF55AA84D0605D42F4ACB
:108FE00092F82520012A7EF4B1AC9AF8872201324A
:108FF000D2B2032A8AF887227EF6A8AC9AF87022A9
:109000001AB943F002038AF8043004200EF0C0FCC1
:10901000FFF738B80A200BF053F8FFF7F5B82049EE
:109020003A610A6842F004020A60FFF71EBBB9F118
:109030000C0F92F88A3300F0C380FDEEE77A4FF40C
:109040009667B7FBF3F317EE902A9142A8BF11463B
:10905000B1F5617FB8BF4FF46171A1F56171B1FBEA
:10906000F3F7A9F10C03FFB2162B3ED8DFE803F0AB
:109070007C3D3D3D3D3D3D3D3D3D3D3D1C3D3D3D02
:109080003D3D3D3D3D665D00842A01204056002067
:10909000D34D6210E85F0120D0370508AC5601209F
:1090A00038570120A8260020A24BC82F19683B463C
:1090B000A8BFC8230A7FD8B2934216D09B1A9E4AF3
:1090C000087748BF0733DB100133DBB20A935379CB
:1090D000002B40F017830A9B002B40F05C82069B1C
:1090E0005344D3ED727AFDEEE77A019B2B4408EBF3
:1090F00043035A7812B99B78302B02D08F4B012250
:109100001A70089BB9F10C0F18BFB9F1210F1B6839
:109110003FF4AFAE002C3FF4ACAE894ACAF8449499
:1091200057601A46CAF84034A5E69AF84B34BB4259
:10913000DBD0022FD9D88AF84B74D6E7814B781C44
:1091400093F820208242D0D0C0B20328CDD883F833
:10915000200024F031FE24F0B3FD069B5344D3EDF0
:10916000727AFDEEE77AC0E7774A5378BB42BCD00B
:10917000032F98BF57705378744AC3EB031302EB65
:109180004303734A13600EF04FFF6B4A5379002B71
:1091900040F0C7827B1CDBB20A939CE7DAF8BC3153
:1091A0006C4983F040099AF8C4210B68C9F380190F
:1091B000089109EA02098AF8C591674FFFF749BA91
:1091C000614A1179002900F09381C821FDEEE77A08
:1091D00040F6330317EE900A8342A8BF0346B3F567
:1091E000617FB8BF4FF46173A3F56173B3FBF1F70F
:1091F000FFB2BAE71B8907EE102A77EEE87A06EE8F
:10920000903AB8EEC77A09F1FF33F8EEE66A66EEF7
:10921000886AA7EEA67AFDEEC77A17EE904A1F2B52
:1092200000F2E982DFE813F02A01FF00C604E9003A
:109230009E04C0009A005A0066044E043604E702F9
:10924000E9003404C0009A005A0031042E042B04B3
:1092500012042000CC02E7022A01CA02FF00C80261
:10926000E7022000C502EA02B4F5FA6F17EE907A21
:10927000304BA8BF4FF4FA672F4A196827EAE777FF
:109280004F825179002940F04D84B9F11E0F0CD066
:10929000B4F5FA6F19685279A8BF4FF4FA6424EA5A
:1092A000E4778F81002A40F05184AA002A4408EB19
:1092B0004202517811B99278302A02D01F4A012116
:1092C0001170186814F0DAFF069B7C1C534418BF19
:1092D0000124D3ED727AFDEEE77A12E7C82C17EE7F
:1092E000907A144BA8BFC827134A196827EAE77772
:1092F0000F745179002940F06083B9F1110FD4D077
:10930000C82C19685279A8BFC82424EAE4778F7260
:10931000002ACAD09AF83C24142111970A3AADF8D1
:109320004C10012AC1D811A90D20019317F002FE9B
:10933000019BBAE79C520120842A01205857012042
:10934000500401200C550120A44E0120644F01203F
:1093500098520120F41A0120AC560120C82C17EEB7
:10936000907AB84BA8BFC827B74A196827EAE777A9
:10937000CF735179002940F00984B9F1100F94D0CE
:10938000C82C19685279A8BFC82424EAE4774F7220
:10939000002A8AD09AF83C24132111970A3AADF892
:1093A0004C10012A81D8BEE7C82C17EE907AA54B45
:1093B000A8BFC827A44A196827EAE7778F735179AD
:1093C000002940F01084B9F10F0F3FF46EAFC82CA4
:1093D00019685279A8BFC82424EAE4770F72002ADA
:1093E0003FF463AF9AF83C24122111970A3AADF882
:1093F0004C10012A3FF659AF95E7099B84F3080703
:10940000914A9F725379002B40F00184B9F10D0FFE
:1094100007D084F308075379099A5772002B40F05C
:10942000DF82884B41E7642C17EE907A099BA8BF36
:109430006427854A012FB8BF01279F715379002BFC
:1094400040F0F683B9F11B0FEBD0642C5379099AE5
:10945000A8BF642424EAE477D771002BE1D09AF8FE
:109460003C341C2211970A3BADF84C20012BD8D874
:1094700011A90D2017F05EFD724B16E7FF2C17EEB9
:10948000907A099BA8BFFF276F4A012FB8BF012719
:10949000DF705379002B40F0C182B9F1190FC0D0B1
:1094A000FF2C099BA8BFFF24012C2746B8BF01272A
:1094B0001F715379002BB4D09AF83C341A221197BB
:1094C0000A3BADF84C20012BABD8D1E75F4B93F8AA
:1094D000743293423EF4F3AD5D4B1B78032B3EF4A4
:1094E00035AA5C4B5B7A002B7EF4E9ADFEF72EBA11
:1094F0004FF49661B1FBF3F168E60F200AF0E0FD4E
:10950000BAF88432544AFA3B8AF88642AAF884327E
:10951000136823F060031360504B0593FEF718BAED
:109520009AF83C340E2211960A3BADF84C20012BE0
:109530003FF639AAFFF778BA9AF83C241E21119613
:109540000A3AADF84C10012A05D811A90D200B9349
:1095500017F0F0FC0B9B3868FFF7A8BA9AF83C3478
:10956000032211960A3BADF84C20012B3FF669AB64
:10957000FFF795BB9AF83C240D2011960A3AADF8F6
:109580004C00012A3FF601AA11A90B9317F0D2FC57
:109590000B9BFFF7FAB90A9B4FF0020C304A4FF0D1
:1095A000140E5B0002EB0C00402B28BF4023991ED9
:1095B000013B014482F800C0023202F801EC914202
:1095C000F8D1274A23F001030E201344FF229A709A
:1095D0000AF076FD83E59AF83C24112111960A3AA7
:1095E000ADF84C10012A05D811A90D200B9317F0E6
:1095F000A1FC0B9B3868FFF78ABA9AF83C241B2120
:1096000011960A3AADF84C10012A3FF6F4A911A9B7
:109610000D200B9317F08EFC0B9BFFF7ECB99AF81B
:109620003C240F2111960A3AADF84C10012A05D8B6
:1096300011A90D200B9317F07DFC0B9B3868FFF7E9
:10964000C9BA00BF9C520120842A0120D8270120DA
:10965000FA5E0120E0530120385701206C580120A8
:10966000F4560120BE4B42F21071BE4A1B8B01FB27
:1096700003F39168B3FBF1F3C2F8D431C2F870334D
:10968000049B1B681A063AD4B74B05931B685B070B
:109690007EF55EA9B54A0021002311600A21B44A73
:1096A0001370B44A1180B44A1380FEF751B99AF886
:1096B0003C24102111960A3AADF84C10012A05D825
:1096C00011A90D200B9317F035FC0B9B3868FFF7A1
:1096D00057BACAF88C32FEF739B99AF83C241921E6
:1096E00011960A3AADF84C10012A3FF6B2A911A919
:1096F0000D200B9317F01EFC0B9BFFF7AAB91FF070
:1097000061FBC1E79AF83C34182211970A3BADF887
:109710004C20012B3FF6DFAC11A90D2017F00AFCFD
:10972000D9E49AF83C340C2211970A3BADF84C204E
:10973000012B3FF62FAD11A90D2017F0FBFB29E5FA
:1097400000283EF4CFAD9AF88032002B40F07781AC
:10975000DAF8BC11FEF7F5B8884B1B68B3F5805FEB
:109760007EF4F4A89AF87432002B7FF4D9ABFEF79C
:10977000EDB841F2024111800221FEF783BE029B47
:109780001C44CAF87C42DEE70120F6F7E7FD764B81
:109790000593FEF7DDB80220F6F7E0FD724B059366
:1097A000FEF7D6B80020F6F7D9FD6F4B0593FEF70C
:1097B000CFB8734B734A6BE5724A46E6714A6FE65F
:1097C000642C6F4B6F4AA8BF642419685279012C2E
:1097D0002746B8BF012781F87D70002A3FF465ADA8
:1097E0009AF83C24172111970A3AADF84C10012A37
:1097F0003FF65BAD97E54FF0FF3712E6B4F5FA6F31
:109800005F4B604AA8BF4FF4FA641968527924EAA2
:10981000E4770F83002A3FF448AD9AF83C242021D6
:1098200011970A3AADF84C10012A3FF63EAD7AE5A1
:1098300002200EF075F900238AF88032FEF77CB81A
:10984000F6F758FFFEF759BC01200EF0E1FC464B3D
:109850000593FEF77DB89E2B7DD09AF882329D2B22
:1098600074D09AF88232AE2B6BD09AF88232AD2B3C
:109870003D4B05937EF46CA8FF21002026F0F4F800
:10988000FEF766B800249AF8932211941AB103F0F7
:10989000C002802A16D1A3F1B702072ADBD801A1A2
:1098A00051F822F0299901085798010857980108A2
:1098B000579801082199010857980108179901083C
:1098C000D5980108F6F716FF274B8AF893420593BF
:1098D000FEF73EB80123ADF844302B4BBDF84440B1
:1098E0009989BDF94620214428489981D9890A449B
:1098F000DA8101238AF8933241F202430380FF2385
:1099000083700E200AF0DCFBBAF88432FA3BAAF826
:109910008432FFF705BB4FF6FF73ADF84430DCE748
:109920000123ADF84630D8E74FF6FF73ADF8463067
:10993000D3E7174B4FF4C8729A850B4B0593FEF78C
:1099400007B80121002026F08FF88EE70021FF20C4
:1099500026F08AF885E70021012026F085F87CE7CB
:109960006C5201208C1F00206C580120D063012014
:10997000D4630120D6630120D86301203857012029
:109980009C520120842A012018540120F456012001
:109990007826002002200EF03BFCAE4B0593FDF72D
:1099A000D7BF9AF8923283F001038AF8923213B348
:1099B0000B200AF085FBFDF7C9BF9AF83C14112073
:1099C00011970A39ADF84C0001293FF696AC11A960
:1099D0000D200A92019317F0ADFA0A9A019B8CE4CC
:1099E0009AF83C340E2211970A3BADF84C20012B1B
:1099F0003FF617AD3CE50C200AF062FBFDF7A6BF71
:109A000003200EF005FC934B0593FDF7A1BF00204A
:109A10000EF0FEFB8F4B0593FDF79ABF9AF83C348E
